:20000000004B00209D4C0100FDC90110FDC90110FDC90110FDC90110FDC90110FDC9011081
:1C002000FDC90110FDC90110FDC90110FDC90110FDC90110FDC901103BCA0110A4
:20003C00000105090004081000040810020402010101010902000120181A18182C34041E41
:20005C00000C0E020B040B0A070800110F00A6AAACA4A9A9A399B19ABCB6A8313117191AD6
:20007C0021241B1D1F31313331313118191A22311C1E20313134310000000500BD00B70068
:20009C00B100BC001C003000380008003801020000010002020200030401000200000000FF
:2000BC000501000706010003070800000F0101FF10080000180800002202000038C40D0089
:2000DC00C80000008100000032000F0100C50D00900100004000000096000501952B0D006D
:2000FC00C80000002200000032000F020000000002000000020000000A00000002000000A7
:20011C000200010000000000000000000000000000000000000000000000000000000000C0
:20013C000E000000C003000080070000000F0000001E0000003C00000078000000F000007A
:20015C0000E0010000C003000080070000000F0000001E0000003C00000078000000F00087
:20017C000000F00001017101010101011101010131010101010180010001100161013B0081
:20019C001400630173017201620143010001130106013D0135000401120100010001000193
:2001BC00000104010401330133013C014401320136000001000165010001350081010001A4
:2001DC000501820183010001660100010001080109010302710230016002110270020102E6
:2001FC000202020280020002100261023A0041006302730272026202430200021302380021
:20021C000002000204021202000200020002000204020402370037003C0244020002390063
:20023C000002000265020002350281020002050282028302000266020002000208020902E6
:20025C000304710402046004110470040204020401040204000410046104000414046304FC
:20027C00730472046204430400041304060400040004040412040004000400040004510418
:20029C006400000400040004440400040004000400046504000435048104640005040004DE
:2002BC0083040004660400040004080409040000360001000600000000000000000F0000C0
:2002DC0000000000000000000000000000000300FFFF00000403FFFF0000FFFF0F00E80304
:2002FC000005401F0330000100000000FF3F0F0008000E0000000000000000000300010FD4
:20031C000000090100000000000000000000000000000000000000000000000000000000B7
:20033C0000000000000000000000000000000000AD0000010001363601010001020100017F
:20035C000301000104010606080400000C0100340D01000F10040101140100FF16080000B9
:20037C0020020000220100FF23010001240100FE250100082602000028010001290100012A
:20039C002A0200002C01000F2E0200003001000131010008320200FF340100073501024056
:2003BC00360100003701000138010001390100FF3A01000F3C0200FF3E01010F3F01000127
:2003DC004001041F41010001420100FF43010080440800004E0100084F01000F5001000100
:2003FC00510100FF5201000A5301008754010001580400005C04000060040000640400007A
:20041C00680400006C0400007004000074040000780400007C040000800100FF81010001F9
:20043C0082010001830101023545251502030504FFFFFFFFFFFFFFFF9A1000000000000031
:20045C00000000000000000000000000000000000000000000000000000000000000FAFA8C
:20047C00140000000000000000000001000001010000000000000000000000000000000049
:20049C00000000000000000000000000000000000000000000000000000000000000000040
:2004BC0000000000000000000000000000000000000000780008020030000A00000800005C
:2004DC000000000000000804FA000000FFFFFF000C1100000000000000001D1100000000B2
:2004FC00000000002E010F000000FA0000002F0100000000FA000000300100000000FF004E
:20051C000000310100000000FF000000320100000000030000003301000000000300000021
:20053C0034010000000001000000350200000000FFFF0000370200000000FF0000003902C1
:20055C0000000000FF0000003B0200000000FFFF00003D0100000000FF0000003E010000C9
:20057C000000010000003F0100000000010000004001000000000700000041200000000074
:20059C0000000000610200000000FFFF0000630800000000000000006B0800000000000000
:2005BC000000730800000000000000007B080000000000000000830205000000580200003D
:2005DC008501000000001000000086020000000032000000880200000000320000008A0267
:2005FC00000000000A00000000C137010000910A010002BF560000007784010001BF560017
:20061C00000077840100039DED0000007784010004E5830100007784010001F78301000153
:20063C00F183010001778401000177840100017784010000095501000177840100017784DA
:20065C0001000177840100017784010002F783010002F18301000277840100000955010032
:20067C000277840100027784010002013B01000277840100041B480000007784010003F7C8
:20069C0083010003F183010003BF56000003BF5600000377840100039DED00000377840187
:2006BC000000095501000377840100037784010004F783010004F183010004BF56000004AC
:2006DC00BF56000004BF560000041B4800000477840100047784010004DF830100000955A4
:2006FC0001000104052900000300000000040000E5F7010083F90100D7F90100F1F3010093
:20071C0055F40100CDF8010059FA0100BFF90100A9FA0100F1F2010011F5010065F90100B2
:20073C00F9F8010065F50100B5FA0100CDFA010095FA010081FA01003BFA01002DFA01006E
:20075C00CDF6010067FA0100A5F901000DFA010095F60100D7FA0100452401003D63010047
:20077C0001F00100B9F5010029F10100F5F9010045550100757901005D790100B5F40100A7
:20079C008D8101007F81010051F60100000000000000000023830100318001000DF7010087
:2007BC000000000000000000000000000000000000010400003333333333333333333333E7
:2007DC00333333333303010F00000000000000000000000000000000FFFFFFFFFFFFFFFFF3
:2007FC00FFFFFFFFFFFFFFFFFF4648546573740000000000000000000000000000000000B8
:20081C00000000000000000000000000D9070000010000001C0B000008000000FE060000A8
:20083C0001123456789ABCDEF000000000000000000000000000000003007100300160005E
:20085C00110070003102200350048000070010006100000014006300730072006200430058
:20087C000000130006000000000004001200000000000000000004000400370037003C0279
:20089C004400000000000000000065000000350081000000050000008300000066000000EF
:2008BC00000008000900010371030103010301030103010322030203010300031003000338
:2008DC00000300030003000300030003420300032403060300030003040312032503230302
:2008FC002503230304030403000300030003440300030003230300036503210035038103BC
:20091C0000030503000300030003000325032303080309038F0000008F0001008F0002008F
:20093C008F000300900000018F00010190000002900000038F0001048F0000058F000804FF
:20095C008F0000048A000006510000007F0001003F0004003F0002003F0001007F00020042
:20097C007B756E6B6E6F776E2D696E7374616E63652D6E616D657D007B656D7074792D69C3
:20099C006E7374616E63652D6E616D657D00C0467B7374617469632D696E7374616E636579
:2009BC002D6E616D657D00C000000102030410000810182004040810181C10040810181CF2
:2009DC0000000000080000000000000020000000400000006000000000000000060000002D
:2009FC0002000000860000008200000006088080070880800D2007C00E2007C01400C08077
:200A1C00024000800300C0800108C0801E08C08009400080084000800A400080FE000000AD
:200A3C00B9120100C13401001D7A010089A80000ADBD00001B840100E130010065C70000C7
:200A5C00218401000D17010000000000FFFFFFFFFFFFFFFF000000000000000001010101B3
:200A7C0000C201000300000000000000001000400600000015000000FF000000000000002A
:200A9C000302FFFF482D002040000000000000007BC80110C5BC0110D9B2011033C20110DA
:200ABC00BDAD0110C1B101106DBA011065BB01101DC00110FFFFFFFFC409000000000000FC
:200ADC000000000001003A0100000000000000000000000065D60000D93801000000000071
:200AFC0000000001010100003C0A000010290020880A0000000000000000000000000000A6
:200B1C00000000000000000000000000000000000000000000000000C33B3D3A5D3A713A02
:200B3C00A10A8F3A0F3BB309495E850A2F3B853B001610160E18151C02120324185803027C
:200B5C0010025800010000000000000000000000000001000000FF7FC82C0020840B0000EC
:200B7C000000000000000000004002400B00000027000000FF00000041B5011095A6011053
:200B9C0015B8011000BE040A00BE0208FFFFFFFFFFFFFFFFFF00000000000000ED79010069
:200BBC006D3F010006000500000001020101FFFF000000400F000000B18B000000000000D3
:200BDC0000000000D1C0011061AD01100A000000D01B002031680100FB84010051CA0000EE
:040BFC00B9830100B8
:201000003C000000000000000000000034100000000000000000000001000000000000004F
:1C10200000000000000000000000000001000000000000000800000000000000AB
:20103C003400000000000000000000006810000000000000000000000100000000000000E7
:14105C00010000000000000000000000080000000000000077
:2010700030000000000000000000000098100000040000000000000001000000FFFFFFFF87
:10109000FF00000001000000080000000000000048
:2010A0002C0000000000000000000000C4100000040000000000000001000000FFFFFFFF2F
:0C10C000FFFFFFFF080000000000000020
:2010CC0038140000E410000095A1011091A70110A1C2011009B2011041B80110A5BC011078
:0810EC0085BC01102E0000007C
:2010F400280000000000000000000000141100000000000000000000FFFFFFFF0000000093
:081114000800000000000000CB
:20111C00341400003011000065C2011069C101101BC2011091BA011005BC0110E5BB0110EA
:04113C00300000007F
:20114000341400005411000071C20110A5B6011099BF011045B60110B5BA011025BC01104B
:04116000310000005A
:201164002400000000000000000000008011000000000000000000000000000008000000AE
:041184000000000067
:20118800240000000000000000000000A41100000000000000000000000000000800000066
:0411A8000000000043
:2011AC00240000000000000000000000C8110000000000000100000000000000080000001D
:0411CC00000000001F
:2011D00000000000B81C002004000000000000000000000020000000701000003000000037
:2011F0001C110000C01C00200400000000000000000000000C00000030130000180000004B
:2012100040110000C81C0020040000000000000000000000240000004813000018000000CE
:2012300000000000D01C002004000000000000000000000010000000A01000002C000000A2
:20125000CC100000D81C0020040000000000000000000000200000006411000024000000D1
:20127000FFFFFFFFE01C00200400000000000000000000002800000088110000240000005D
:20129000FFFFFFFFE81C0020040000000000000000000000580000003C1000003400000042
:2012B000FFFFFFFFF01C002004000000000000000000000010000000601300001800000057
:2012D000FFFFFFFFF81C00200400000000000000000000001C000000AC11000024000000CD
:2012F000FFFFFFFF001D002004000000000000000000000038000000F4100000280000003D
:20131000FFFFFFFF081D002004000000000000000000000054000000001000003C000000D8
:1813300018000000000000000000000040130000080000000000000032
:1813480018000000000000000000000058130000080000000000000002
:18136000180000000000000000000000701300000800000000000000D2
:0813780002000000B80B0000A8
:041384000100000064
:0413880000000E0053
:04138C0000000F004E
:041390003200000027
:041394000100000054
:041398002C1C0020E9
:04139C00000200004B
:0413A000FD830100C8
:0413A400FDC901106E
:0413A8000000000041
:0413AC00000000003D
:0413B0000800000031
:0413B4000000220013
:0413B800341A0020C3
:0413BC00010000002C
:0413C000441C0020A9
:0413C400080000001D
:0413C8000000000021
:0413CC00000000001D
:0413D0000000000019
:0413D400080000000D
:0413D8000000000011
:0413DC00000000000D
:0413E0000100000008
:0413E4002C1B00209E
:0413E80006000000FB
:0413EC0001000000FC
:0413F00014190020AC
:0413F40000000000F5
:0413F80000000000F1
:0413FC0000020000EB
:0414000000000000E8
:021406002900BB
:021408000100E1
:02140A002500BB
:02140C003000AE
:02140E003100AB
:021410002E00AC
:021412000100D7
:0114140001D6
:0814180003000000940B00002A
:081420000000000000000000C4
:0414280000000100BF
:04142C0000000300B9
:0414300083C4011060
:041434003C14000064
:041438003C14000060
:04143C0000000000AC
:041440009000000018
:041444009000000014
:0414480000000000A0
:04144C00441C00201C
:041450009D7F01007B
:041454002000000074
:04145800600B000025
:04145C00AC0A0000D6
:0414600009C30110AB
:0414640077480100C4
:04146800CB4F010065
:04146C0095C801100E
:0414700097C8011008
:041474000000000074
:041478005F0B000006
:04147C0094090000CF
:04148000AC090000B3
:041484007C090000DF
:0214880008005A
:02148A00090057
:02148C0001005D
:02148E0000005C
:01149000015A
:041494000000000054
:041498000000000050
:04149C00000000004C
:0414A0000000000048
:0414A400F3840100CC
:0414A8002D5D0100B5
:0414AC00ED6F0100DF
:0414B0007D61010059
:0414B4007B62010056
:0414B8004D5401008E
:0414BC0029120100F0
:0414C000D3810100D3
:0414C400493A0100A0
:0414C8000DC801103A
:0414CC001DC8011026
:0414D0000800000010
:0414D40024000000F0
:0414D80018000000F8
:0414DC0028000000E4
:0414E00020000000E8
:0414E4003C000000C8
:0414E8000C000000F4
:0414EC0034000000C8
:2014F00083482DE9F04F0C4601210170DFF80892DFF80882DFF808B2DFF808A27D494FF0EE
:20151000000C2027ADF1540D65461F4081F800C0C949119391F8FC62C849109205EA0200E5
:20153000139108BF00287AD110984FF0E047194662460F4002EA000008BF002843D1119EBB
:20155000109B4FF48601B9F8BA00DFF828C3CDF82C9012EA060701EA030108BF002919D186
:20157000C34912EA060701EA030108BF00296FD037464346109E1C8103F138015881002FA2
:2015900081E8C00004BF311CB1F1806F60D102285ED111E037464346109E1C8103F1380178
:2015B0005881002F81E8C00004BF311CB1F5803F4ED1B0F5505F4BD1186A6746436938686B
:2015D0002146984742E046465946B6F9087091F90000BC42A0F10100087017D1728906F1D5
:2015F000380003C8002904BFB0F5803FB2F5505F08D0002904BFB0F1806F022A02D012F0DE
:2016100047F803E013F098F816F090FA139890F90020521E02706FF00101318114E04346AF
:201630006FF0010003F1080108806EB1BD480078832802D08120514608704646316919B1FC
:20165000604688472146E8E7CDF82C90B9F8BA00109A119E02212F461140374008BF00293A
:2016700000F0CD83B14A43F201418142149200F09F83C91C814200F09B83594691F900103E
:201690005A464746491E1170B7F908108C4209D0139943F6040787420A9140F09A8316F00F
:2016B00065F896E3644890F8FCC207F1380090E800034FF482062F4617EA090706EA08005E
:2016D00008BF002820D113980C4F0A9007F1380003C84FF400322F460F4002EA000208BF91
:2016F000002A02D111F0D4FF73E313F025F870E33D1D0020741C00207015002058180020E1
:201710007B1C0020532E00202846BCF1010F51460E9002D00F78002F79D1834C8120149E0D
:20173000277808702B46A5816069A770427A017A337002F0070301EB032152098DB234BF98
:20175000291F891EDFF8EC81437A8DB233F07F0340F0198376490988A942C0F214830A301B
:20177000294610F00FF8216A04F118000522083116F030FAED1EADB20D960520E17E227F89
:20179000A37E2D4EA081C1F3011B227103EB012096F8FC326081002B08BFBBF1020F00F0CE
:2017B000F282BBF1020F00F3EE8263B110F0070F00F0E9825B490978862904D100F007015F
:2017D000022940F0E082011301F00201022953DA6378DFF8509100F00700022837D1464694
:2017F000D6F804A0002B32D1216A09A801220D3116F0F0F90620A081D047804699F80030C8
:201810000D48B56847680C96862B19D10FB916F005FE9DF9240016F058FE9DF9246078776A
:201830000020B8774046FE77A847608900F0100010F08CFF06E0C046080200207A1C00201F
:201850004046A84713980A9015F0F2FFA1E299F800000026862808BF01261398CDF83080D2
:201870000A9076B1002012F08DFFA77808E0C04600000C8CA81A0020CDF8308013980A90A8
:2018900063788FB183B9012F00F07A826089022F03D110F0070F40F07382032F05D100F0A4
:2018B0000701032901D06BE26089010909D310F4405F00F06582B84991F82074002F00F040
:2018D0005F82011301F00201022902DA810A80F05782B0490978C1F381098E11B9F1010F23
:2018F00000F04E82012E00F04B82C249BBF1020F09D08A5D11F809108918CFB206B3C109DD
:201910001ED3BF1E0BE072184944127909798918CFB2C10910D259EA060311D0BF1CFFB253
:201930000EE0C046572E0020882D0020552E0020941C0020D017002059EA060308BF022773
:20195000C0F300217A1A61719542C0F21982ED1B00090D44A9B2218124BF25200E900E984E
:201970004018743080B215F0BFFC65782061002800F006820021742210F008FB0020E07041
:20199000B4F80A801DB90D9908F0200008700D9B002094F805A01D780F90002D3CD0BAF1E4
:2019B000000F39D108F00708B8F1030F06D0B8F1010F22D1784890F86A04F0B17648B0F8FD
:2019D00054000023810809D3734991F8825095B94D681DB16D7E35F07F050CD15BB9800826
:2019F000984605D384498D68887805B1A84710B9B8F1000F01D00420E070674890F8FC02BF
:201A100010B1BBF1020F01DA15F058FAB4F80A80E07894F805A00F90216901F17400486010
:201A3000886525890D812089A1F85C005FEA18100ED3CAF1030082B2A1F85C20886DCF4969
:201A500016F0C8F82169B1F85C20886D801888655048CA4D00780F9BC0F301122878A1F8B7
:201A70000C8000F07800104318430874FF258D732079BAF1000F0E9018BF002081F8306023
:201A900081F83A9081F84900A089002FA0EB0A0085B2A58100F06A81B946216AE78068466D
:201AB0004A464919083116F095F83A487F19BDB2A5810078C0F30111129121690A7C6E4605
:201AD000801010F0030F00F0030702F0400B43D012980023022801D1D0090BD29DF80120D5
:201AF0009DF8000000EB0220A1F844000DF10206A1F84200C84AB1F84400B2F85A2082428F
:201B100003D04FF6FF72824223D1032F12D072783078C14B00EB022082B24A86B3F858109E
:201B3000B61C0120914213D04FF6FF71914218BF00200DE0C84800683146323016F07DFCB0
:201B5000C548B54900684F31323015F07FFE08360346002B00F00D810E480078831123D019
:201B700012982169022803D0087CC00903D309E05BEA070706D172783078B61C00EB02207D
:201B9000A1F84200032B09D07078327802EB00220A8509E0A32D002008020020AE480068C2
:201BB0003146283016F049FC08F00708B8F1030F07D0B8F1010F3BD1A94890F86A74002F17
:201BD00036D0A7482669876F4FF00008FFB17B7E33F07F0317D096F8300002280ED003280E
:201BF00011D107F1700006F1280115F02FFE50B11EE0C046A00B0000801C0020B7F87000AE
:201C1000318D884214D057F80C7C002FDFD1B8F1000F0DD1914F594B4046E070387842466A
:201C3000C0F3011118780F9200F07800084330748B4890F8FC7217B1129802280CDA0D9857
:201C500007784FB1BAF1000F06D10E980F9911F0D7F8A589B4F80690206981890909C0F081
:201C70008580806D69464A4615F0B4FF2169886D48448865276AB1F85C0001224844A1F895
:201C90005C000DF125007919083115F0A3FF6E1CB5B2A58121699DF82500896D08702169F0
:201CB0009DF825709DF82530886D401C8865B1F85C00401CA1F85C0007F0070081F82400D1
:201CD000C3F3C10781F8257091F8246020898046002E4ED05E497F183E78361D8642E6802B
:201CF00047DC216A324605A84919083115F072FF38789DF817209DF814109DF81630401987
:201D10003D78001D01EB026180B201EB0341A0819DF81530206901EB032181616DB14E4806
:201D300000686D1E06A92A461C3015F053FF397820696944C97D80F82610806D05A93246F0
:201D500015F048FF2169886D80198865B1F85C00A8EB06078019A1F85C00781E82B2228182
:201D7000B1F85C000A818018A1F85C0000F07EF80FE016F099FA11F08BFC0AE0A22D0020E7
:201D900016F080F805E016F07DF8CDF8308013980A90DDF83080D8F804008047216A0A687E
:201DB0000023137109682162D8F80810884710E04046807841465F46401C887097F9000043
:201DD0005946401E087011F063FC15F0CFFC13980A9023480B99104F00226FF0010690F88B
:201DF000FC02A1F8BA203E8110B11498007808B915F09CFE0A9991F90000401E08701948FA
:201E100090F9000010B9134800210170139A92F9000098B102E0C04658180020109B119F1F
:201E300002214FF0E0401940384008BF002908D092F90000002804DC16F0F0FA002003F0E1
:201E500037FC0949002015B00870BDE8F08FC0463C000000721C0020982D0020A32D0020A7
:201E7000080200207B1C00203D1D00202DE9F04FB64C20692589216AA689806DADF1440DD3
:201E90002A468919083115F0A5FE2169886D40198865216A7619B6B201220DF13E008919F7
:201EB000083115F097FE216A761CB5B2042204A8A5814919083115F08DFE9DF813109DF84B
:201ED000100000EB016023699DF812102D1D00EB01409DF81110A58100EB0120049015F05C
:201EF00081FFD863049815F009FCA3F84000EA2015F0D5FC0221B54827690170397CE07888
:201F1000084338749DF93E0016F0DFFA87F846009DF93E00398987F8480007F17400B8655C
:201F3000B7F85C00401A79684FF0000B401801467860B88987F847B0820A18D2020955D32A
:201F500010F0070F07D000F00700032812BF081C7868401C46E07968C87800F007024010A1
:201F700000F0380000EB42004018001D3AE00FB916F054FAB889800A2ED379684878C6110D
:201F90002AD13D89796658464B780A7803F07F035B0003EBE2137E2B0DD07F2B09D002F000
:201FB0007F0280188918801C891C80B28542EBDC08E0594600E00121801C87F8601080B210
:201FD000854201DA584605E07968091879603989091A3981A7F86800786E10B1B7F868008D
:201FF000B0B178687861B889000916D297F86000002800F0F980384612F0ACF82769F86CED
:20201000002800F0F180B7F85000002840F0EC8016F038F9584620610CE258465D4605904A
:2020300097F82460069005A906AA07AB0795384605F0D0FE002840F0CC80059A7D697868F1
:202050003B89291A581A1FFA80F80AB916F0E6F9B7F85C0000900195CDF808800698001D85
:2020700003900598B969BB6D324615300AF0BEFF002840F0AE80B64897F860303D89815D1B
:20209000681A388113B1384612F064F8BD8905F00705032D02D178680078F87397F80F901A
:2020B000732009A914F014FD832010A908F0ECFDDFF8A082DA4659460AE0C278012A03D19E
:2020D000002E08BFDC2027D0001D491C0990C9B29DF8400088427BDD09988278032D07D0D9
:2020F0000378AB420DD098F800300BB1022D08D0032DE9D10378032BE6D103465B784B4512
:20211000E2D1B310B3EBA20F05DA02F0030206F003039A42D1DD58468146059897F80FC02E
:2021300090F814E0594601E0491CC9B28E454BDD06694B00032D06EB030209D1F35C032B81
:20215000F2D152786245EFD10BE0C046882D00201278AA4205D098F80020002AE4D0022DAD
:20217000E2D10698067D002E08BFB9F1DC0F2FD0B869B0F1FF3F25D0712008A914F0A8FC13
:20219000089B5846BA6905998B4206D10699824601EB8A01C968914212D8401C2C330228D8
:2021B000F1DB0698521CB2F1FF3F00EB8A00C26002D107980121817087F801B0584609E083
:2021D000DB2007E0DB2004E0DC2002E0532E0020DD20787027697870B8697E7878651EB18F
:2021F000F22015F05CFB2769954D95F8FC02002800F09D80B989DFF84C8201F00702022A22
:202210005CD16678002E59D17E78002E56D121698DF83FB00DF13600283116F00EF92169DE
:202230000BA80A22283115F0D5FC464606F1100127690888D5F82033401C0880786E0DF1E4
:202250003F020421984704F1100928B9686818B19DF83F1080F86810276997F83000022854
:2022700011D1D9F8000005F57A71884602222830203114F07DFE30B908F116010DF136006F
:2022900016F0DBF8276970480078862807D1708A401C7082B88900F0100010F057FA95F8A8
:2022B000FC0220B1D5F8441309B12069884715F0E9FF5846206115F0BBFABDE0634A16786B
:2022D0005EB3C1F30131022927D17878002840F0B1809DF83E005E4946460870B38AE17847
:2022F00007F128021C37581C0029B0820CBF5846082058495B460B6000900197B5F80E3435
:20231000117A0D2005F05AFC10B914F0D7FD01E015F01EFA0F482769007840B1D5F8441397
:2023300029B1384688472846276990F8FC02BE890A9706F0070688B1B87BFF2876D0032EED
:202350000AD1384640680078042807DD6EE0C0464000000004050020012E67D1301C3AD06A
:20237000401E4ED0801E61D1B889C0F30130022803D17868007807282BD03889002855D04E
:20239000384641684A1C42600F788446C7739CF824606EB9002F49D00A2F47DA2E49008992
:2023B000C95D814209D0082F40D1082805D03DE0C07B00283AD00A2838DA60460189491E99
:2023D0000181C17B0B3101700A99C87B401CC87319E0322016E095F8F5030F280BD015F028
:2023F0001FFD40B90A988189091301F00201022901DA2969884795F82B040A9F387415204F
:2024100000E0162038700A9905F17C0013F07AFE124E7068804795F88410491C85F88410C8
:20243000B1688847202015F053FE42E70AA812F01BFD3EE711F02CF911B0BDE8F08FC046E3
:20245000080200208C1B0020572E0020552E00201A1D0020D01A002047000000D017002084
:202470002DE9FE4FDD4981460122A1F130000260D8480768002FFCD0D74AE34EC027D848D2
:20249000D84B17603268920808D2324652F8042C03F14104120C42F0F00222704FF0000A3C
:2024B0008346C1F800A0DFF88CC3DBF80810E04F0191880E43D2480E41D3802018744FF692
:2024D000D802A3F8512018703868C0F30464162CA8BF203C1E460F3E307800F01F00162818
:2024F000A8BF2038844223D0624602F1980EE44ACEF800A0251A022D05DC15F1020FB8BFA2
:202510006FF0010500E002254019156800F01F05844245F4F855A6F866504FF001051560FB
:20253000E8D110682E4616601068CEF80050106838460068C0F30420162808DB06E0A7F10E
:20255000D0000068C0F30460162800DB203800EB2170401C162805DA10F10A0FB8BF6FF0C6
:20257000090000E01520D54E00F01F0040F4F850A3F85900306880083ABFD148C0F800A001
:2025900041F040616246C80E8E0E80F0010000F00100106086F0010000F00100906001987C
:2025B00010F064FD0146182013F040FCA7F13806CD4C30683568A4F10408C0F3870105F0F7
:2025D000030041EA0021D8F80400C04D446840F2FF32534688B22C21009028464038A0472F
:2025F000F06AC0F30D011C2013F020FCB549706A014000F07C400143142013F017FC316A67
:2026100001F47C000904090C0143102013F00EFC7D4AB06A1268C0F30351C0F303445208E0
:2026300013D2DBF80020130511EB237103D41029A8BF0F2100E05146120414EB227403D46A
:20265000102CA8BF0F2400E0544644EA011400F47F4200F0FF01B9F1220F42EA044241EABA
:20267000020124BF00F0804001430C2013F0DEFB954CB9F1220F32BF01202068C0F30070EF
:20269000B9F1220F4FEA400040F0200085F8090126BF2068C0F3407001208D4EB9F1200F5A
:2026B00040F0100085F8090138BF514606D33168C80C00F44070C1F384510143282013F0B3
:2026D000B5FBB9F1200F26BF3068C0F301505046B9F1220F4FEA400040F0600085F80C01DC
:2026F00026BF2068C0F3C0605046B9F1220F4FEAC00040F0800085F8010126BF2068C0F3D1
:2027100045505046B9F1200F4FEA800040F47C40A5F89C0138BF6F490AD3306801038A15FB
:20273000920501F47C1100F00F00114341EA0031082013F07BFBCC3F4FF480002860664A1A
:20275000B86D40F21E216FF31F40814216D93868030E03F00F0113F00F0FC0F3034018BFBE
:20277000491E072805D006280EBF0720801C00F00F0041EA0011A2F108000170DDF804C040
:20279000CCF381477F1E02D07F1E31D02CE02068810C29D24FF480412960D2F80210430AC3
:2027B000C0F3033703F0800321F08F010B4347EA0301C2F80210D2F80130060A66F303034C
:2027D000C2F80130116800F0E70721F0E70147EA01000CE09402224300600C404010094050
:2027F000AC3F0050156208404FF000402A46106005480068C0F3C0070FB94020A8624FF4CC
:202810000070286402E0C046B03F005020684027C0F3C14040F0300085F8C800CCF38150AD
:2028300080B3401E08D0FFE7401E23D0022122E08813005000002043012013F083FF064683
:202850000420314610F0D4FD042013F07BFF8642FAD12248066826F07F4013F0DFFDD8F86C
:202870001400036807214FF06022300E98474FF4806028600321042010F0BAFD09E0C0462A
:202890002C2009400420012110F0B2FD144813F0C5FD203C206800F03F0085F8CB0FD8F843
:2028B0000030124ED96830680220884710480D4C076001212160BDE8FE8FC0460000094072
:2028D00094042A43FCFCFC008C13005040A00C409813005000803F400A600840A83F0050F1
:2028F000BD37860094046042A40100102C20094000600C402DE9F04F0D46C84C0168616236
:20291000416880686160ADF14C0DA060284613F05DF94FF008094FF0010B06A8ADF8189001
:20293000616AADF81AB08847BD4E9DF81C1071700899716108B114F01DFE28688047A04649
:20295000D8F80400804712904FF40057ADF800901E200197D8F82410ADF80200684688475D
:2029700013F000F8C94C206C40688047206CC16810A88847206C836810AA00200146984789
:20299000E06308B914F0F6FD14F0D4FFC14FC4F8D470C24AC4F8DC20C149C4F8E010BC48C7
:2029B00030610025A4F85450BB4BC4F8D830BD4FC4F8E47004F5C472C4F8642104F1C00105
:2029D000C4F8681104F1D400C4F86C01B64BC4F8E83013F093FF04F1980704F51C70C4F881
:2029F0007471B34AC4F87001B04BC4F80821B14FC4F8B03003F16E00A765B04AC4F8B40064
:202A1000AD4B2266AF4FE365B4F85410C4F8107241F00100A4F85400AC4AC4F83022A8497B
:202A30006166A94BC4F8203204F15807C4F88471AB486062A6492161A74AE261A54BA3616A
:202A5000A649216214F016FAA64FC4F80073A849C4F80C13A44BC4F80433A44AC4F8082339
:202A7000A44FC4F81073A649C4F81C13A24BC4F81433A24AC4F81823A24FC4F82073A4493A
:202A9000C4F82C13A04BC4F82433A04AC4F8282384F8FC52B4F85400B56040F01000A4F881
:202AB00054009C4FC4F830739D49C4F83C139A4BC4F83433994AC4F838239A4FC4F840731D
:202AD0009B49C4F84C13984BC4F84433974AC4F84823984FC4F850739949C4F85C13964B75
:202AF000C4F85433954AC4F85823964FC4F86073974981F800B0944BC4F86433934A15606C
:202B100002204D8014F0E8F8FF210222F06215F0E2FCF01CFF21022215F0DDFC022014F005
:202B3000DBF88C4F386008B914F024FD38682946022215F0D0FC11A80FA912F02FFFF06A5A
:202B50009DF84410421C01709DF84400107025709DF84400B07014F0C7FAB061D8F82410EC
:202B7000ADF808901420ADF80A0002A888471527ADF810900398ADF81270D8F82410F06114
:202B900004A88847754F0598DFF8DCA1744B3D70801E3062704E1D700AF1080235701088CC
:202BB00075700E30356180B214F09EFB074677610FB915F033FC09978DF828509DF8290001
:202BD000684965F301008DF829009DF82900534665F383008DF8290018899DF82920088046
:202BF00065F307128DF82920ADF82A00706909A94A4614F0EFFF3762756212F0F1F85B4EA6
:202C10003078012802D0284602F052FD58480570584F3D703078012807D003E0D017002057
:202C30006C1A0020284602F043FDD8F808101298884700F0DBFE14F077FB94F82B0411F0E2
:202C500033FF584602F034FD12F058FB4A4805703078012802D0284602F02AFD10F032FBBE
:202C70001820ADF83090454FADF83200444E0D97D8F824100E960CA8884708B115F0CEFB54
:202C900002F0D2FF13B0BDE8F08FC046080200202D480100518F000001370100F374010053
:202CB000C9D20000DDE40000A51D010080010000DDD100008DBC000059B40000714A0100A4
:202CD0004560010011410100F121010039840100D592000039DE0000216C010011200100DC
:202CF0009D57010089070100DD6B00002D2501003D590100F1850000E5EF0000015400006D
:202D1000952D0000E9140100858D0000B5D30000417D0100ED970000CD450100F56D010090
:202D30009DD4000041AB0000BD7000002F750100A5F00000593B0100D16D01008D4B010012
:202D5000597001002D790100EB830100382E00201C1D0020482E0020882D0020532E002098
:202D7000552E0020401600208C1C00203D1D0020572E00204E2E0020542E0020731501007C
:202D9000C41B00202DE9F04FADF18C0D1C9104461D920DF15700D1491E93082214F01AFF8B
:202DB0002046694612F0F2FF1F90002804BF0020229000F0098202200027A41CDFF824B35D
:202DD0002090C74E2297204602A911F040FA5FEA000900F0F68122990DF13900162215F031
:202DF0007AFB9DF809707F1E00F088807F1E40F0E081B9F10A0F40F3E781A41C04A804228D
:202E1000214614F0E7FE241D05A80222214614F0E1FE42F20B000DF1160111F0CFFBBDF822
:202E30001600BDF81410884200F3CE81A41C14F8010B14F8017B14F8015B8DF8390014F8F5
:202E5000011B8DF83A700DF139028DF83B50204606F0EEFBC34909780028044400F0B48167
:202E70001F9D012905F1020500F09C814FF400500DF14F0111F0A2FB0DF14F000DF1570130
:202E9000082214F075F840B11C990DF14F00082214F06EF8002840F0858142F2010004A9C0
:202EB00006F09CFC42F20B0005A906F097FC42F205000DF1390106F091FC0DF13A0142F29D
:202ED000060006F08BFC0DF13B0142F2070006F085FC0FA942F2090006F080FC9DF83C003B
:202EF00028B1022840F05E8142F2030001E042F20D000DF13D0106F071FC53E1B9F1040FC7
:202F100040F36281A41C14F8010B14F8017B14F8015B8DF8390014F8011B8DF83A700DF1B0
:202F300039028DF83B50204606F082FB0028044400F04A811C9806A906F01EFD9DF83600F3
:202F5000002840F011819DF83C0000287DD1B6F84E70002F00F00481B6F85200874207D080
:202F7000308B718B884201D109F074FBB06D21E0B76D4FF400500DF15F0111F01FFB14F034
:202F900013F94FF6FF78229D2190AA46B6F84E00A84243DCB06D4FF6FF7141450AD04FEA89
:202FB000480707EB88073818808812F027F8B06D3F1823D1B6F84E300746002B08BF229D26
:202FD00019D05846229D40681946D846BF1FBF1DFA782AB1491E05F10105F8D1BF1D0AE07D
:202FF0008047B6F85210491CA6F85210D8F808108847B6F84E30AB4200F099801C980AF0FE
:20301000B7FAB8800120F870FD788DF83650B888ADF83700229B8DF82330A5E0B88811F037
:203030008FF9014608220DF15F0013F0A1FF40B138880104219815F018FA82453CBF824677
:20305000A8466D1CBF1DADB2A0E7B6F84C70002F00F08680B6F85000874207D0308B718B43
:20307000884201D109F0F6FA706D20E0776D4FF400500DF1670111F0A1FA14F095F84FF68F
:20309000FF78229D2190AA46B6F84C00A84250DC706D4FF6FF71414509D008EB48173818A6
:2030B000B0F81F0011F0AAFF706D3F1829D1B6F84C300746002B08BF229D20D0DBF8040072
:2030D000229D1946D846213F2137BA7F62B1491E05F10105F8D1213711E0C0464C040000D5
:2030F000BC0F0020D01700208047B6F85010491CA6F85010D8F808108847B6F84C30AB42C8
:2031100015D022993846212215F0E5F91C980AF02FFAA7F81F000123FF2039462122BB778F
:203130000546787206A8FD7214F054FD1CE0612057E0B7F81F0011F003F9014608220DF1EA
:20315000670013F015FF38B17968219815F08DF982453CBF8246A8466D1C2137ADB293E7A1
:2031700064203EE00A0200209DF836000DF13901162240F004008DF8360008A814F02AFD6C
:203190001F9D9DF83C00AD1C48B19DF84E700DF13D00394610F004FD3F1A8DF8357006A891
:2031B0000FF07CFB209809EB0007BF1CB8B2209003E01F9D4C44A41CAD1C209885423FF774
:2031D00002AE2098022803DC229A6720114604E01F9A911C121A2298921C1D9B19801E99EE
:2031F0000A8023B0BDE8F08F2DE9F04F0320ADF1540D13F02BF9C74C0025022004F11C0134
:2032100041F80C5F401E8D60FAD104F14000A846062701467F1E21F80C8BFBD14FF00809E4
:20323000C84BC749C84EA0F800901B1D816004F11C07AA4623F003031A46F11A216210469F
:20325000A3611E46E3615B18834200F2BB81881021F00301E82302EB800040F804ACEC391A
:2032700033604046C2F8E810E83222611BF0FAFF6061B6493868DFF8D8B220610A680BF122
:203290000C06326049687160CC48CD494A4613F06FFE28B9C948D0490A680260496841609D
:2032B000CE48CF4FC0F8B470C0F8BC50C0F8CC50CC4EC0F8D050CC4BC0F8B860CB4AC0F8B0
:2032D000C030CB4FD0F8B410C0F8C420C0F8C87009B1404688471CF03DF8C64ECDF838A0BB
:2032F00041460C2206F128000EF050FEC24F0222ADF8209041F27073F762708DADF82220C1
:20331000616A33631027099740F01900708508A8884700280CBF0A9F47460120ADF82C90FD
:20333000616AADF82E000BA888479DF830005C4620700D99616077B1D021397087F801803D
:20335000B87087F8038087F804803946BD600220FD6012F00DF9A949182001221BF038FF7E
:203370009649E22014F034FE18201CF019FA60706068B346CBF808000BF06AFDA94F0BF11D
:203390008400A060DBF808509D4C41466762F520A56014F0B7FA9B4D0D200E26687005F14F
:2033B0000C01AE7005F118000DF002FCA860687814F0E6FC00B1C146A87814F0E1FC08B981
:2033D00049F010099049A86814F026FF8F49C82205F1240011F0FCFA8D48B9F1100F686040
:2033F00010D1606A70B1C26862B1FF208DF810004FF6FF77ADF8127004AEADF8147096E8C5
:2034100003009047834D05F1140005F108010DF0CFFB6860404614F029FF4746AE1E814688
:2034300006F8028F02207070384614F08BFF014668684A46C9B212F005FB7F1C022FEFDB25
:20345000754905F120004FF4FA7211F0C1FA734D05F11000291D0DF0ABFB2860606A0028F4
:2034700045D00769DFF8B8916FB10094494612A80A688988026012AE818096E8030001234F
:203490004246B847606A002831D0C26852B1494612A80B688988036012AF818097E8030001
:2034B0009047606A18B307690FB306208DF80800ADF80A0010AEADF80C8002AD009695E84B
:2034D000030042460223ADF84020B847666ABDF840007769A08057B1BDF8400002AE401C5A
:2034F000ADF8400096E80300022210ABB84737A014F0FAFCE820032114F004FAE720092148
:2035100014F000FA606A0626002833D00769002F30D001E0D01700208DF818600425ADF82A
:203530001A500EA8ADF81C8006AB009093E8030042462B46B84768B90E981930824619E092
:2035500045F90100582E0020004B0020C8FF01005C1C0020606A8DF8186006AFADF81A5020
:203570004469ADF81C8097E80300CDF83CA02A460FABA047CDF838A050460EF013FBE020DA
:203590000C2114F0BFF94F20032114F0BBF95720052114F0B7F94E20042114F0B3F95920DA
:2035B000032114F0AFF914F047F80BF10200012114F06CF800F0B4FDFCE7C046681C002032
:2035D000A80B000040F804AB3EE6C04654492053656E736F7200C046F01200502007002041
:2035F000CD51010071560100290B01001D5A010019E800005816002020BF0200DD66000074
:203610006C14002060190020FD5A01004D7A0100FD7B0100F019002051F90000101C002009
:20363000C00B0000D40700202DE9FC47DFF848930F460646F80B80F0A181DFF83883B80F1A
:2036500080F04281B80880F03581F80A80F00F81B80B80F0FB80780B80F0BA80380C80F0B0
:20367000A9803809C0F0AB81082014F029FE002840F09B80802014F023FE002840F09580FC
:2036900068460DF039FD012803D10098002800F08C8000240125E0B214F0B4FA48B1867AF9
:2036B0003EB1857290F9090005FA00F0C0B212F019FB641C032CEED344460320A070A068D6
:2036D000783014F0CCFEC248002601680660C14950F8082CB046324640F8088C04F14C0064
:2036F00014F0CDFE304613F09FFD14F03FFBE6786EB126795EB9E1686669A369401A06EBF6
:203710001030B0EBC32F9CBF6061454623D913F06BFE414600B12946081C18D0AE4840F6DE
:203730000901018000F10D03414641801A7800F10C0665F303021A70327861F30302327084
:20375000416014F0CDFC418811F4406FFBD0E57045466561257111F065FF26789F48056018
:203770001EB9A068403014F09AFE022012F0ACFB11200BF04BFDA068007C10B90E200BF099
:2037900045FD607818B16570052012F09DFB944814F024FDB4F94800B4F94A10A5708842C6
:2037B00014BF022007200DF035F827F008070FF0AFFE04E14446A06B80684688002EFAD0B9
:2037D000A06B806840880128F5D027F40047EEE712F054F938B1B56930466FF480710022B7
:2037F0004FF00073A84780494446002204F14C0014F045FE0220A070B0680188A1F60205AA
:203810002DB141F21E016D1A18BF183000D11030018821F47C7141F43471018000257574BD
:20383000266914F0A3FAD4F81011A26804F58873914214BF0121291C26B1801B03EB810669
:20385000020BB260256127F48057B0E7484614F022FE061C08D0706830B17468F068B6F9E2
:203870002C1000222023A04727F40057A7E014F000FE4446054604F1340014F00CFE061C87
:2038900012D0A06810B1783014F0E9FDF068A06014F06CFA2061534814F0A0FC4FF40061B9
:2038B00004F1A80014F003FE284614F0D7FE27F4806784E007F086FC4046443014F0EBFD4A
:2038D00008B927F002077AE014F0D3FD8246B0680188A1F602052DB141F21E016D1A18BF34
:2038F000183000D110300188444621F47C7141F434710180E068D0B1042012F023FFB0B17D
:20391000E56814F033FAF168401B738AF060020BF26098188842F06002D240184008F0602B
:2039300040F6C41181422CBFB0F5FA7FF160504614F094FE12F0A2F890B1B56930466FF44F
:20395000807100224FF00073A84704F1340014F0A2FD002808BF47F0020701D00FF0D8FD03
:203970007469002130464FF080630A46A04727F0005724E0F82300203424002014F079FDCB
:203990000146484614F087FD061C13D0356AA80810D225EA05003062084614F05FFE706857
:2039B00058B155B17468F068B6F92C102A460023A04702E0084614F051FE27F4804727B112
:2039D000484639466C3014F072FDBDE8FC87C0461410044035390100082E002000000460FC
:2039F0000DD90000BDB60000BDA500002DE9F04FD64F4FF00008ADF1140DD24DCDF8088010
:203A1000F8688DF80C8000288DF80D8037D1CE48CF4984380068814217D0CE49814214D029
:203A3000CD49814211D0CD4981420ED0CC4981420BD0CC49814208D0CB49814205D0CB49E2
:203A5000814202D0CA4981420CD112F0CFFC012814BF40460120787005F12000006800F147
:203A7000200408B914F0DAFC216807F1140088474FF4FA70F884BF4EBE620624FC62DFF85E
:203A9000F892EB6999F83B244FF0010A41468801A0EBC100C01890F8266036B990F82540E0
:203AB000491CA242C9B2F2D103E090F82510914204D1834202D012F089F8EB69DFF8BCB274
:203AD000686A17C88BE817007878012814BF40460520AB4C8BF8000099F8696426B998694C
:203AF0000068C4F8AC0005E0D8690068C4F8AC0013F020FE632004A911F062F899F83B0474
:203B100012F07EFA064604F19E0108786AF30200087099F83B24812A03DB842A23DB862A0F
:203B300011DB94F8A00004F1A70140F00F0084F8A000087868F303000870B07B052814BFE4
:203B50002420292016E094F8A000292340F00F0084F8A00004F1A70184F8A430087868F337
:203B70000300087008E094F8A00040F00F0084F8A000212084F8A40004F1A5010878812A24
:203B900068F38710087001DB842A1ADBB37A83B904F1A5029DF810001178401E60F3050142
:203BB00004F1A6001170017821F03F0141F0180116E004F1A5019DF81020087862F3050095
:203BD00006E004F1A501087820F03F0040F00200087004F1A600017821F03F0141F0200124
:203BF0000170B07BB1890A2304F19E02401D484390FBF3F1138861F3CF031380B0891921FF
:203C100004F1A003800390FBF1F2196862F31C2104F1A8021960E869117890F8243063F3D4
:203C30000201117004F1A80290F824001378C11061F3C303137099F92A040FF0C9FC4FF6E3
:203C5000FF71814218BFA4F8AA007168308933684FF47A72401E414303EB5100B0FBF2F0FA
:203C7000EB69A4F8B000186A0078A4F89280C4F8948004F19D0384F8B40018786AF3030067
:203C9000187014F005FBC8B9B0893E49B2FBF0F0C0B20870B2FBF0F03B4A507099F83B042E
:203CB000022806D0842809DB862807DA05215C2001E00221A820354B19701070FB682E6AE3
:203CD0005BB3404611F0AEF8B87899F83B14884212D1F97899F869242E6AF86891420DD1A4
:203CF000022142468DE80600366D9034434602AA2146B047EC601BE02E6AF86871688847AD
:203D100023482B6A80F800A01E68224890345946224607F11403B04707E0903422461D4842
:203D3000346807F114035946A047F860686AA86299F83B0499F86964B87005B0FE70BDE8F0
:203D5000F08FC04658180020181300509C1A002000F0022000F0012000F000200080022018
:203D70000080012000F0820000F082200080822000800020A96E0100080200201C2E002020
:203D900070150020B01B0020181D00208C1B00203E1D0020382B00202DE9F04F064692F83E
:203DB00008B0307D09AF8946ADF1240D04933528039205D0114606F170000A2213F00AFFE4
:203DD000DFF8C4C239F07F0506BF604600884FF6FF700590F08A800934BF002008203076A9
:203DF000F08AC00834BF102080207076F08A400903D260460E30007800E00020B076F08A34
:203E100041082CBF20240024000928BF44F010047568002109F07F09307D06916D1E022846
:203E30000EDB0C2808DC0C2803D1022044F40854069044F0030404E00D280CBF02200120BB
:203E5000044396F88C0008B144F00804210900D328B1DFF8C88298F8203413B908B1DF2099
:203E70004BE121096ED306F12401DFF8A4A296F88D50079100EB0A011AF805300A799918EE
:203E90003389491DCAB29918A24B1A8808908A42C0F2358100284CD0049A039906F184006F
:203EB0000AF018FD0799002808603FD0806AB0F1FF3F39D070680023401E8DB196F88E100F
:203ED000524600F80119515D491EC9B241B18A1992F88320491EC9B2002900F80129F6D1E2
:203EF000079970660968896AB162090E00F8011996F82A1000F8011996F82910089A00F861
:203F1000011996F8281005F0030500F8011902F0070141EAC501017071683589091ACAB210
:203F30007060A918318105E0DB2700E0F3277770E6E00023F08A7370C00828BF44F0100429
:203F500075686D1E336DA3B9B36D93B998F83914012903D13089B0F5EE7F06DA200904D2FC
:203F700002290AD144F4005401E044F48054012002E044F408540220069098F802000128A8
:203F90000CD098F8FC0248B196F86B00042805D1022024F48054069044F4005444EA893498
:203FB000B9F1020FA4B20AD0B9F1030F10D1ED1F08F22C41284614F040FA6D1E08E0B8F827
:203FD0001204001205F8010998F8120405F80109069802280CD0B9F1000F15D0BBF1000FF8
:203FF0000CD004990598814208D144F040040BE0BBF1000F08D1B9F1000F05D005990812C2
:2040100005F8010905F8011944EA8B24BBF1020FA4B209D0BBF1030F0ED10399ED1F2846F6
:2040300014F00BFA6D1E07E003990888001205F80109087805F80109BBF1000F05D00498FD
:20405000011205F8011905F801093878F0B932480178307D0D2814D068B9306D28B998F8DE
:20407000FC03411C88F8FC130AE098F82104411C88F8211404E098F80A04411C88F80A1417
:20409000014605F8011903E01606002044F48074201205F801092C7070683789401BC1B22C
:2040B000756078183081200926D3B06D00B1306298F8FC0210B1307D0D281DD1746A14F156
:2040D000150001D114F0AAF9A16A481CA0623289306AB162471B0092D21B019090B2029023
:2040F000706A96F88C202B46153008F08FF800281CBF7070071C07D10020707005E0E52798
:204110007770F32013F0CBFBF8B209B0BDE8F08F3C000000941C00208C2D00200802002036
:204130002DE9F041C84CC94DDFF824836088ADF1600D4108C0F083800CA808A90EF0C4FD6D
:2041500001286DD1404624300068D8B10769CFB1062002268DF808000022ADF80A600FAB67
:20417000ADF80C2002AE009396E803000C23B84740B9BDF83C006085109FE7621198206379
:2041900013F0E0FD0226BDF82210BDF8200084F8246009AAA1830FF03BFB011C02D0B6A0FA
:2041B00014F030F930460EF0FBFEBDF830009DF82C70A5F840000DA985F8427005F1500037
:2041D00014F0BBF8BDF8320005F1460609A9A5F84E00304614F0B1F8BDF82200B5F840105B
:2041F000A5F84400502013F081FBB5F84E10532013F07CFB4A20314613F0EAFE95F842103C
:20421000E12013F07FFBB5F844104B2013F06EFB05F10A00102113F039FA0120207008E038
:2042300012F072FFE06001200EF0BAFE002013F047FEA01C012113F01BFA204640888008D0
:204250000DD3E06A12F032F912F056FC00B2A082E08202F0F7FDA01C022113F009FA6F89AA
:20427000780805D305F10A00012113F001FA6F89B80805D305F10A00022113F0F9F96F8916
:20429000780917D383491820422217AB1AF0A0FF95F85A0005F10A06032818BF042802D1E2
:2042B000286E12F0EBF811F0A9F83046102113F0DFF96F89B80907D30DF0E8FD05F10A00DA
:2042D000202113F0D5F96F89F80907D30BF0E8FC05F10A00402113F0CBF96F89780A0AD38B
:2042F00095F85D0013F0ECFD05F10A004FF4807113F0BEF96F89380951D395F85C0005F1AE
:204310000A0600283FD0401E37D0401E02D0401E31D03FE095F85810472013F0F3FA95F85A
:204330005910542013F0EEFAB5F844104B2013F0DDFAB5F84010502013F0D8FA09270323C7
:2043500095F842008DF8597016AA8DF85A3052498DF8580001278DF85B7018201AF038FFF8
:2043700095F85A00012815D1E87898B13046202113F08CF90EE003200AE05220012113F0BD
:20439000A9FA022004E05220012113F0A3FA01200EF09EFD3046082113F06AF96F894546EE
:2043B00017B1A86814F056F9E988687849081CD3A97802094FF0000601D301290ED040099B
:2043D0000ED301290CD030A013F08EFDA01C012113F05CF9A86814F03DF901E010F08CFAA1
:2043F0006E70A81D012113F043F9608800283FD10A200825294CADF812004FF0FF37ADF8EC
:204410001050616A059704A88847002830D10720ADF84850616AADF84A0012A88847149EC8
:20443000159628BB1E499DF84E200878904214D19DF84C004A7882420CD089684B6C63B13E
:2044500000213246984708E058160020241700206C140020304600F025F8159840B1ADF89D
:2044700018500320ADF81A00616A079606A8884718B0BDE8F081C04641757468204572723E
:204490006F723A20307800C05374617274696E672E2E2E00D14B010079830100D017002072
:2044B0005C1C0020B0B50446BA480768ADF1480D002F00F0A8812078401E112800F2A381B4
:2044D000DFE810F06A015201380123011B010401F100E300C300B2008D005D005300420001
:2044F000A1012A001C001200F86B002800F08B81684621460CF01EFFF96B82E1386C00286A
:2045100000F081816846002101220DF03FFD60788DF80000396C74E1F86A002800F07381A9
:20453000684600210E220DF031FDA11C684613F091FAA57BA1890022ADF80A1005B1012244
:204550008DF80C20F96A5DE1B86B002800F05B816846002102220DF019FDA5788DF80150E9
:2045700060788DF80000B96B4BE1786B002800F04A81684621460CF0DDFE796B41E1386B23
:2045900008B36846002114220DF000FDA5788DF80150A3680193A289ADF80820A17B8DF826
:2045B0000A1060788DF80000E57B8DF80B50237C8DF80C3094F911208DF80D206169049105
:2045D000396B684688476068002800F01C810146F22008700020487010F0CAFF13E1B86AA5
:2045F000002800F010816846002124220DF0CEFC6078A11C8DF800000DF1020013F02AFAE5
:2046100004F10C0103A813F025FA257EE08A04F119018DF818500B22ADF816000DF11900B3
:204630000CF094F9B96AECE0786A002800F0EB806846002102220DF0A9FCA5788DF8015005
:2046500060788DF80000796ADBE0386A002800F0DA806846002112220DF098FC65886279DF
:204670006078ADF8025023798DF80520E11D8DF80000A5798DF804300B220DF107008DF804
:2046900006500CF063F9396ABBE0F869002800F0BA806846002101220DF078FC60788DF8AB
:2046B0000000F969ADE0B86910B120460FF07CFDA07820B9A069002800F0A58003E0A06918
:2046D000002800F0A08012F0FFFC9CE07869002800F099806846002113220DF057FC6D4600
:2046F000A01C0168406829600B22686004F10A0102A80CF02BF9796983E03869002800F097
:20471000828020460BF076FA7DE0F86800287AD0684600210E220DF039FC6078A11C8DF83C
:2047300000000DF1020013F095F9A089ADF80C00F96866E0B868002865D0684600211422D5
:204750000DF024FCA01C01686D46296040686860A07A0B2204F10B018DF808000DF109007F
:204770000CF0F4F8B9684CE0786800284BD06846002110220DF00AFC60786588211D8DF845
:2047900000000B22ADF8025001A80CF0DFF8796837E0C046641C00203868A0B36846002109
:2047B00019220DF0F3FBA01C01686D46296040686860A07A410824BF01218DF80810810864
:2047D00024BF01218DF80910C10824BF01218DF80A10010924BF01218DF80B10C10924BF5D
:2047F00001218DF80C1030F07F001CBF01208DF80D000B220DF10E0004F10B010CF0A6F8E5
:2048100039686846884712B0B0BD70472DE9F04F09AFADF13C0D08900A92388809911E469E
:20483000ADF81800101C08BF002000F08481002700F101094FF0FF3A4FF0010BB8466CE173
:20485000252940F063811078521C0A922D2818BFADF8068005D15846551CADF806001078E5
:204870000A9530281CBF4246434605D10A9908785A465B46491C0A912A28CDF800805546D9
:2048900016D1306804930A99CDF808A0C01C4B1C20F00300001D306050F8044C0A93002C7E
:2048B0000878009418D5ADF806B06442009413E044460AE0610001EBC4010918A1F13004F2
:2048D0000A9908780094491C0A91302801DB3A28F0DBCDF808A004932E282BD10A99087837
:2048F0002A2801F101010A9111D13068CDF80880C01C20F00300001D306050F8045C002D8F
:2049100048BF454608782B46491C0A9111E0454643460AE0690001EBC5010918A1F1300512
:204930000A9908782B46491C0A91302801DB3A28F0DB02930AB1224604926C2804D04C2848
:2049500018BFADF8048005D10A990878ADF804B0491C0A910BA9CDF80C800FAB0791642812
:20497000059300F08B80692800F08880BDF818C0752872D078286ED06F286AD0702850D038
:2049900063283DD073281ED009980A990128A1F101010A9115D96B490C68B5F1FF3F03D07D
:2049B000A84288BF6D1C00D8099D029508A80AA932466B46A0473F180A99039801F1010914
:2049D00074E040462AE030680A99C01C20F00300001D306050F8040CBCF1000F01F10109FC
:2049F000014608B955A00146079113F041FA0390B5F1FF3F5BD0A842C4BF281C039056E071
:204A10003068C01C20F00300001D306010F8040C5D468DF82C000A990395584601F1010911
:204A300045E0082035680490E81C20F00300001D306050F8041C082210230FA80DF0F6FEB7
:204A5000401E0790402101700A99079801F1010929E0082302E0102300E00A230A993068B0
:204A700001F10109C01C20F00300001D306050F8041CAA42BCBF2A1C049210E00A993068B8
:204A900001F10109C01C20F00300001D306050F8041CAA42BCBF2A1C04926FF009030FA8A1
:204AB0000DF0C4FE0790059D281A0390009C241ABDF8065000945DB906E008A8202109AA00
:204AD00011F0B5FF009C7F1C641E0094F5D503980546401E039075B9BDF80600E8B1009809
:204AF000401E009019D408A8202109AA11F09FFF00987F1CF4E70798411C0791017809AABA
:204B100008A811F094FF03987F1CE1E708A809AA11F08DFF7F1C09F101094A460A9812F878
:204B3000011C401C00290A907FF48AAE089808B14146017038460FB0BDE8F08F286E756C55
:204B50006C2900C0F80B0000BA482DE9F84F0025B94CB749056094F8E200002800F0638195
:204B7000012800F02F81B54E02283CD0032840F05A8151F8250CD4F8B8100029A0F5C06001
:204B9000C4F8D400B8BF49420028B8BF4042814226DA4FF08057D7F8A4014568B4F8BC00F0
:204BB00030214FF47F42082300903046A847D7F8A4014568B4F8C00004214FF4F80212234C
:204BD00000903046A847D7F8A401B4F8D070456820214FF440620A2330460097A84701254E
:204BF00084F8D8501AE151F8258C13F003FB2F4600B901273946924F38680028FCD0B146CA
:204C1000012609F10409D9F82CA03E6009B113F0F7FACAF30720C4F8BC0013F0EBFAAA4639
:204C300000B9B2463B68002BFCD0D9F800B0BAF1000F3E6001D013F0E3FACBF38440C4F851
:204C5000C00013F0D7FAAA4600B9B2463B68002BFCD0D9F81C90BAF1000F3E6001D013F0CC
:204C7000CFFAC9F38120C4F8D000B8F5C061C4F8B81000F09C8094F8D80068B9C4F8D410EF
:204C9000D4F8C000C4F8C800D4F8BC70C4F8C470D4F8D030C4F8CC30D4F8D400D4F8BC3030
:204CB000002854BF02226FF0010204F1C8010F6800EB40008018421000EB927207EBA20056
:204CD0000860D4F8C810C4F8C43000291CDD1E293CDDD4F8CC0030B93429B4BF15391E21A8
:204CF000C4F8C81025E02A29BABFD4F8C8000B381E20C4F8C800D4F8C4003F28B4BF401CE0
:204D10003F20C4F8C4001FE0D4F8CC00032812D011F10B0FC6BFD4F8C8000B30301CC4F888
:204D3000C800D4F8C4000028C4BF401E051CC4F8C450032508E011F1150FC6BFD4F8C800C2
:204D50001530301CC4F8C800C4F8CC504FF08057D7F8A401B4F8C43030214FF47F4245682A
:204D7000364800930823A847D7F8A40104214FF400321123456831480096A847B4F8C86037
:204D9000D7F8A40104214FF4F802122345682B480096A847D7F8A40120214FF440620A238C
:204DB000B4F8CC60456825480096A84701E084F8D85040F2FF50404502D8801C40452DD2E7
:204DD00008202EE051F8251C1E4F4BF2F5204843060A3868C0F3814001280AD111F08CFE06
:204DF00010F002FC13F012FA3111C010484306EBE03694F8E50030B91348006820F07F4006
:204E10003618760801E084F8E5501048310C0660012741600E4D8760287808B90B2000E0B2
:204E3000052084F8E40004F073FEBDE8F88FC0462D400C402C500C405813002000A00C404E
:204E500000800C40B43F0050102009403C600C40010B00002DE9F04FB34C8146201D0768FF
:204E7000ADF12C0D002F00F03C814FF00008388979689E4ECDF81C80C50009783078103506
:204E9000890906D340F6485191FBF0F16D1805F5AF753E7D68438500352E0CBF46464FF4D0
:204EB000FA560DF12601E8200FF08AFE9DF82600032808BF44F620666068007DAD19352809
:204ED00003D1D4F86003804745430220DFF82CA28DF820000AF10C000068069506A908F053
:204EF000CBFE0120844E8349814F0870317887F80080012901D000F0DBFB60680589466865
:204F100012F022FA3088000942D394F8FC0200283ED061684B6A4F6E986AB0F1FF3F26D0BB
:204F30002FB3421C9A628862030E07F80139606890F82A0007F80109606890F8290007F8F6
:204F50000109606890F8280038706268106A00950190801B281A80B20290916A506A92F8CD
:204F70008C203346153007F051F9074600E0DB27D4F8401367B119B9E4200CF0D3FD04E08A
:204F90005F4880F80080E4208847002F40F0AB80294630460CF0F6FB642009A90FF010FEF0
:204FB000584894F8FC12007831B994F82B0409F0B1FF012805D090E009F0ACFF012840F076
:204FD0008C80DFF844A1A81C87B20DF125010AF180000780E9200FF0F3FD9DF825000128FB
:204FF00005D13D46C5F3022040F0180005E02D1DADB2C5F3022040F0080006F8010D06F87C
:20501000015D55469DF82400A5F872800028C5F88C600CBF3D483E48CDF8108002238DF899
:20503000158005F138068DF8143005F1700AA6F8028005F14501C5F8C800364FCAF818001E
:20505000087820F00F0040F00300087078688047DFF8C4B00A90B9F1010F1DD0B9F1040F06
:205070001AD0B9F1000F14D0B9F1050F0ED0B9F1030F08D194F83B0410F0C2FFC07B022877
:2050900018BF56460AE005F1700607E0DFF88CB004E005F1540601E005F138061448006A2E
:2050B000164B046D02278DE88001D868314604AA5B46A0471A49174F0880B96800280AD48A
:2050D000184A92F900000A4F7035401C10700A98FD60884707E00A9888471A200CF022FD7E
:2050F00001E013F09BF90BB0BDE8F08FB01B002058180020731C00203D1D00209C1A0020CF
:20511000572E00201B1D0020701500204E9055550E7A5555D0170020F1AD000069E2000033
:20513000CC1A00207A1C0020080200202DE9F04FAC4C07460020ADF13C0DDFF8A482ADF836
:205150000C00201D00688946017D252900F00281703005A904F010FC002818BFC0B240F091
:205170003B8101A804A90DF02BF912F08BFC00280CBF41F2081543F2C82504A901A80DF0AB
:205190001FF998F82B2201993B684FF47A7A504650430AFB1100C01A8542C0F2D880D8F8DC
:2051B0000422521A0AFB02F1C91A8D4200F3CF808542A34609DD002807DD95FBFAF04FF402
:2051D000916100B201FB003038609DF81F00002857D042F204000DF136010FF0EFF911F0FF
:2051F000C3FF0699441A42F206000DF135010FF0E5F99DF835009DF81D10FF2804BF0A20F5
:205210008DF83500FF2908BF0A219DF835609DF81C507548B4FBF0F2701884B25646A8101F
:2052300054437043A04298BF041C41F20810241805A811F08CFD9DF81C103D68B0FBF1F209
:205250004A43821A714392B272438B1A891A5B1B491B8C4201D9002908D56142994212D236
:20527000002B10D5B4FBF6F109B203E06100B1FBF6F189B23A684FF4916303FB01253D6011
:2052900001E03D68002006460DF1120102A80DF097F80298D8F804120024B5FBFAF28018ED
:2052B0000290814203D998F82B32834202D998F898712FBB9DF81C00B6180004B04298BFD1
:2052D000361A9DF81F00002808BF9DF8200024D09DF81C00B6FBF0F085B2BDF833000FF0C2
:2052F0002FF89DF83120014628460FF001FC054611F01AFD024608A928460FF011F90CE021
:20531000814204D8BDF81200401CADF81200BDF8120098F89B110DF039F989F8000088F8D1
:20533000F501DBF80400007D052811D19BF8110470B999F8000003A9ADF80C0042F20C0005
:2053500004F04CFABDF80C00A8F8F00100E06524204641E012F096FB00280CBF41F20815EB
:2053700043F2C825214800784FF47A7404FB00F13868491BA1F5FA62824206D2A1F57A61F6
:20539000B0FBF1F24A43801A386068460DF10E010DF016F83868009998F82B2204FB0101D3
:2053B00054430091611A8D4211DCA4F5FA648C42BCBF00F5FA60386098F89B11B8F87801F2
:2053D0000DF0E4F80146002089F8001002E099F80010652088F8F5110FB0BDE8F08FC04675
:2053F000BC0F002008020020A0860100E71100202DE9F04F002898461446ADF12C0D00F0CD
:20541000F38011F47C1F40F0EC8011F00F0F00F0EB8007460591002006900A904FF0000AD7
:205430000990554608954FF0010BCDF810B0054650460790059805990BEA000021EA0B01FC
:205450004FEA4B0B401E059100F0AB80401E70D0801E5DD0001F40F0BE8042F205000DF171
:205470000E010FF0ABF89DF80E00002800F0B3801CB1276694F86B0006900720152607F835
:20549000010B022301A907F8016B42F2010007F8013B0FF093F8684603A90CF091FF069838
:2054B0000FF066F80146019A00983E4640180090824206D8801ABDF80C300090581CADF8C3
:2054D0000C00009B50085146814609041804030C19430004534610EB090041EB0A0102F001
:2054F00085FF0090BDF80C309DF80C009DF800209DF8011006F8010B181206F8010B9DF8C8
:20551000023006F8012B9DF803200935BF1D42E00220152607F8010B042307F8016BB8F188
:20553000000F07F8013B0CBF099898F800002D1D4EE01CB1E76594F86B0006900520152697
:20555000049B07F8010B0DF10F0107F8016B42F2040007F8013B0FF031F802A80FF06EFD69
:2055700006980FF005F802999DF80F609DF80F30069AED1D4018000200EB6600B0FBF3F02B
:205590003E4602903F1D06F8012B9DF808109DF809309DF80A2006F8011B06F8013B32702F
:2055B00018E00320152607F8010BB8F1000F07F8016B034607F8013B04BF0A9807F8010B63
:2055D00005D098F8000007F8010B98F801006D1D07F8010BADB2059800287FF42BAF2E4640
:2055F00061E011F00F0F01D000205DE080468A4602264FF4803908F1020509EA0A002AEA42
:20561000090A4FEA4909B0F580301AD0B0F5803014D0B0F500300ED0B0F5802009D0B0F5EE
:20563000002004D0B0F580102AD1072404E0062402E0052400E00424002704E00224012791
:2056500001E001242746A81C214600F04BFC47B104F00F04C0F30A0141EAC42141F4004122
:2056700005E004F07F0400F0FF0141EA042105F8011B0912871929702D18B81C6D1C86B237
:20569000BAF1000FB9D1022ED8BF00260BDDB01E4FF6FE7708F8010BF019C0F3022040F03F
:2056B000A00088F8000030460BB0BDE8F08F70472DE9F047AC4C06466068ADF1280D8047BB
:2056D000994DDFF88882A24F934C8246012E00F0BF802078DFF854920F284FD08F4890F9F2
:2056F000000010F1020F05D18D4890F9000010F1020F43D08B4C20782E68079006F13C0060
:2057100000688047079D6168E668401A0896A900B0FBF1F2089DA068002304F1180686E80F
:205730000C00AA421E463146B14102DA2946884205D805463146AA42B1411FDA08900898D1
:20575000194604F11805801A994185E80300079B04F1180696E803001A46DB1712F06AFAF6
:2057700004F1180540F6B832D317801A9941002985E8030002DA01214846017012F0EEF90A
:20579000002860D06A48007800285CD169480078002858D168480078002854D1674800780C
:2057B000002850D14846007800284CD164480078002848D163480078002844D1624800785E
:2057D000002840D100200CF047FD00283BD144462078002837D15F4D286A436CF86802212A
:2057F00004AA98479DF8100068B3DFF830812A6AF86898F90010002611F1020F18BF0126F8
:205810004FF001092EB1926B98F9001090472A6AF868434E96F9001011F1020F03D0926BD4
:2058300096F9001090476FF00100307088F8000084F80090002012F033FC286AC169F868E9
:2058500088470020687048498968504688475FE001200CF001FD44498968504688472078B5
:205870000F280DD008F0B8FB28680C37436C3868022105AA98479DF81400002846D047E078
:2058900044462078012841D1012012F009FC324E96F8C2000028FBD12E4D286A436CF86893
:2058B000022106AA98479DF8180050B196F8C20038B92078012829D10020207012F05AF977
:2058D00024E02948406880470021029180468DF80D1002202070214E71802A6A8DF80C0081
:2058F0001F4B146D8DE80300F86802AA3146A0471D498C68002801D512F090FD194991F9F8
:205910000000EE60401C08704046A04711F00CF80AB0BDE8F087C046FD050020701C002039
:20593000711C0020B01B002078180020562E0020532E0020552E0020572E0020542E0020E0
:20595000721C0020731C0020741C00203E1D00209C1A002058180020382B00208015002011
:20597000FD4601007A1C0020D01700202DE9F04FAA4C07466068ADF1340D80470B900AA9C2
:20599000822005F081F9A64EBDF8280038BB00244FF6FF75ADF8284017E0ADF80450BDF893
:2059B0002800ADF80650FF210822ADF8000002A812F091FD8DF81840D420694602F008FF12
:2059D000BDF82800401CADF82800301DBDF8281000888842E1DC82200AA902F0F9FEDFF853
:2059F00044920020B246ADF828009DF8280000268DF8000069468DF80160D02005F044F9BD
:205A10004FF000080126F0B99DF80B30012B07D19DF80A0020B90DF1020012F0CFF890B901
:205A30007D7B002D0CBF0522092246469D420AD10DF1020007F10E0111F0A6FC002818BF25
:205A50004FF0010809D1002E40F0D780B8F1000F03D1787F002800F0D080564600240CE0C8
:205A70006E490B98896888471A20D4E0BAF804006D1CADB24BE0641CA4B2B088A04242DD36
:205A90009DF82800ADF8224008A98DF82000D12005F0FAF80028EED19DF82400FF28EAD083
:205AB000ADF800006946D42005F0EEF8002837D102A8391D082211F067FC0028DBD0388862
:205AD0007D88ADF80400B8F1000FADF8065008D0387BBDF82810BD698DF818000DEB8101A0
:205AF0000D61D420694602F073FEB8F1000F0AD0387F9DF82510884205D08DF8250008A915
:205B1000D12002F065FEB088A04276D10025A84270DDADF80050D420694605F0B5F828B15F
:205B30003E490B9889688847192074E00DF1080B584612F043F8002300B101233C1D181C6D
:205B500006D158462146082211F01EFC00288DD07B8838883A7BADF80630B8F1000FADF8DF
:205B70000400BDF828308DF818200DEB830101F110010CBF0020B86908220860214602A819
:205B900012F028F899F8FC0230B1D9F84C231AB1BDF8001020469047002401E0641CA4B27B
:205BB000B088A0427FF762AF9DF82800ADF8224008A98DF82000D12005F066F8E82803D0F3
:205BD0009DF82400FF28E9D19DF8000000228DF824003B7F8DF8262069468DF82530D420B9
:205BF00002F0F6FD08A9D12002F0F2FDB088A0427FF73CAFA8423FF433AFBDF82800401C7A
:205C100080B20228ADF82800FFF6EFAE03490B988968884700200DB0BDE8F08FD017002002
:205C30008C1C0020080200202DE9F04FAB4C04F128000068ADF1240D0FF040FA08B111F0CF
:205C50008BFCA148DFF898A2DFF884B20068A14E089011F055F811F047FAE569A769B5F51F
:205C70007A7F13D0C01B4FF47A720023A5FB000102F0BCFB80464FF47A72002311F0DAFFCF
:205C90002A46002302F0B2FB381801E0A0EB0708A0618C488B49006820F002000860706894
:205CB0008047DBF80010DBF8042045464919B1F57A7F0DD34FF47A73B1FBF3F3D218CBF858
:205CD00004204FF47A731F46B1FBF7F25A43891ACBF80010B168884770688047DAF80410E6
:205CF0004919CAF80410B1688847DAF8000000285FD007464FF00009706880474FF00008D0
:205D10001FFAA5F3079083B95FFA95F36BB93979E8B2884204DD79682846884209D20AE015
:205D30003879E9B2401A387108E079682846884201D3414601E07968091A7960B88878B979
:205D5000FB8853B9FB6843B13B8933B1B87A19460AF0EEF9F8687860B88808B9FB880BB1BB
:205D70003B896BB9B9F1000F04BF3868CAF8000003D03868C9F800003868B846074601E04D
:205D9000B9463F68B16807988847B8F1000F0ED0B8F8043043B9B8F806302BB998F80A00EC
:205DB000B8F808100AF0C4F9404611F07DF9002FA2D144484349006840F002000860E06853
:205DD00028B3804723E015F8060C2169A5F10C07032819D0E16A9DF816000978884210D186
:205DF00015F8080C10F0DAFBB979012903D0022908BFA87000E02870002029460DF0A8FCBC
:205E100005E011F0A9FB02E009B12846884708200727ADF81000716AADF8127004A8884787
:205E3000069D0028CFD0294800680088C8B1706880472649096800220D880A80B168884766
:205E5000089A00202946207090470546FF202070706880471D4909680A8815430D80B1689A
:205E7000884710F04DFF0746B7F1FF3F1CD0706807B9194F216AB94238BF0F1C80471C232A
:205E90000546626AADF802300820ADF80000716A019268468847A16A3846491CA1620FF05C
:205EB00085FBB1682846884708200A27ADF808004FF0FF35ADF80A70716A039502A8884778
:205ED000C7E6C04610E000E0D40B0000482E0020981C0020D01700208EC2F5286C1A0020CC
:205EF000342E0020F0B504460846ADF16C0D401E70D0401E0DD0801E00F00981401E00F07D
:205F1000EF80401E00F0E180401E00F0AD80002042E142F2010007A90EF050FB42F20B0028
:205F300008A90EF04BFB42F206000DF165010EF045FB42F207000DF166010EF03FFB42F274
:205F5000050019A90EF03AFB04A80AF095F906460DF1670142F209000EF030FB9DF86700EF
:205F7000002808BF002503D0022010F0D4FB0546204607A9042211F02DFE241D08A9022270
:205F9000204611F027FEA71C9DF864009DF865309DF866109DF8674007F8010B9DF8672011
:205FB00007F8013B2B4607F8011B610706F0070444EA916005F0030404AD40EA84103146A0
:205FD00007F8010B012400953846019406F040FC0A309AE042F206000DF165010EF0EEFA6F
:205FF00042F207000DF166010EF0E8FA42F2040019A90EF0E3FA04A80AF03EF905460DF116
:20601000670142F208000EF0D9FA9DF86700002808BF002303D0012010F07DFB03469DF8A3
:2060300064009DF8657004F8010B9DF8666004F8017B9DF867209DF86770790704F8016B37
:2060500003F0030705F0070646EA916004AE40EA8710294604F8010B00270096204601976B
:2060700006F0F6FB001D50E042F2150011A90EF0A5FA13AF42F2160039460EF09FFA15AD58
:2060900042F2170029460EF099FA17AE42F2180031460EF093FA204611A9082211F09AFDB0
:2060B000083408222046394611F094FD04F1080708223846294611F08DFD082207F1080023
:2060D000314611F087FD202066E042F214000DF122010EF073FABDF8221002200A1258E0FD
:2060F00009A80021202212F0F6F942F2130009A90EF064FA09A812F0F0F9024609A920463A
:2061100011F068FD09A812F0E8F980B244E042F20E0002A90EF052FA0DF10A0142F20F009C
:206130000EF04CFA0DF10B0142F20A000EF046FA03A942F210000EF041FA0DF10D0142F21C
:2061500011000EF03BFA0DF10E0142F212000EF035FABDF808009DF80B209DF80C709DF848
:206170000D609DF80E509DF80A1004F8010B02F00102001204F8010B07F0010042EA400283
:2061900006F0010042EA800205F0070042EA4012042004F8011B22701BB0F0BD2DE9F04F35
:2061B00009AF8B46ADF1140D03938046029212F060F9A549019035390868404508BF4868E3
:2061D0009F4C04904FF0000984F8459110F02EFE061C00F01C81D4F83851B4F94800A84584
:2061F00000F101006FF31F30B08507D194F84401410824BF00F0FE0084F844010298006831
:2062100000B94846B0629BF80C0000F00F00022814BF4846DBF8080070620498002867D044
:206230009C3011F0E5FE002840F0EE8040460FF065FE051C0DD1636B5BB1A16B626B3046C8
:2062500009F0D6FB28B1012384F84531606B3060666394F845A1BAF1000F49D10DB9656B75
:206270008DB12A683046294609F0C2FB18B92D68002DF6D107E0022384F84531286830602B
:2062900094F845A12E60BAF1000F31D102980179049807F05DFD0146012926D094F84501F8
:2062B000002825D1012923D0616B09B10D68D5B99BF80C0000F00F00022819D19BF80C00B9
:2062D000C011400814D241B9A56B8DB1A16B30464A4609F08DFB58B996E030464A4609F04E
:2062F00087FB28B990E00968E0E7042084F84501002E00F08E8008F1780012F0B0F8C6F898
:2063100008B0B08D029DA4F84800287986F82E00039B73604B48C6F80C8097E80C0020218E
:2063300006F110071940104006F1180387E80300484686F82F90494683E803006879012840
:2063500005D196F82F0040F0100086F82F00019812F084F994F84501042807D1D4F83C01B6
:20637000B4F9401194F8422112F002F812F081F8054694F8450102280DD196F82F0040F097
:20639000800086F82F0088F8C290284612F066F9B6F92C0050E0012813D104F1840012F08C
:2063B0005EF896F82F0040F0800086F82F0088F8C290A06B0028E8D1284612F04FF922487D
:2063D000007830F004001CD104F1340031466A460EF018FC18B9284612F040F92AE0B08D01
:2063F000A8F8C0009DF8007096F82F0040F0800086F82F00012F88F8C290C6D1284612F005
:206410002DF911F053FCC3E74FF0020901E04FF0010994F8440140F0040084F84401019879
:20643000C4F8388112F01AF9B9F1020F08BF6FF0020001D06FF0010005B0BDE8F08FC046CF
:20645000F8230020FDEFFF9F3D2500202DE9FE4F0546287D012808D195F917000DF0B8F83E
:206470004FF6FF71814200F016819548EF7B017894481FB990F883208A4208DB012F03D1BB
:2064900090F882208A4202DBF120BDE8FE8F80462E6A95F83500B5F8289095F83470AC8BE9
:2064B0004FF0000A5FEA060B029017D098F8FC32002B2FD0D8F8141300292BD006F0FF00B8
:2064D0008847D8F8141306B20BF47F008847361830B2001D00B2C83086B200E0C8260CB127
:2064F000241DA4B298F82004012809D147B1764802993F1897F804A0405C8019401D86B299
:2065100009EB040080195044801C80B210F01EFD071C02D11A20BDE8FE8F09EB0A003319B1
:206530003881002C03EB070078600EBF0020B819801C00217822C7F8A40007F10C0011F01C
:20655000CAFF09EB0600FF2110220019A7F84C0007F13C0011F0BFFF07F12C000F21102299
:2065700011F0B9FF00243C707C707868696A2A8D11F030FB07F1840005F12C010B2211F033
:2065900029FB07F19000294611F07CF96889A7F89A00287B87F89C00687B05F10E0687F806
:2065B0009D00326869460A60706848609DF800102046012908BF01209DF80110012908BF47
:2065D00040F004009DF80210012908BF40F008009DF80310012908BF40F010009DF8041025
:2065F000012908BF40F020009DF80510012908BF40F040009DF80610012908BF40F08000F3
:206610009DF80710012908BF40F48070A7F89E00A87D87F8A000E87D87F8A10095F83800DE
:2066300087F86C00AA8BA7F8A82022B1D7F8A400A96911F0CFFAA87F87F8AA00286AC7F800
:20665000AC00B7F8A800C0B1D7F8A400A8B17868401E7860F82101707868401E78600470C0
:20667000B7F8A810B7F8A8607868401A786038898019801C38817868B865B7F89E00410A96
:2066900016D395F83710052905DB00F0040100F00100084302D0E820BDE8FE8F08F188065B
:2066B00030460BF0BFF995F83710304611F07AF898F8000039460DF04BF82046BDE8FE8FFD
:2066D0008C1C0020080200203C0000002DE9FE4FDFF82892074609F1040000688047DFF837
:2066F000148200248346002F88F8034064D010F005F908F26C402146AC22054611F0EBFED3
:20671000DFF8F4A10AF104000188C80000EB011080B210F0E1FAC8F80C0560B105F18C0739
:206730000226BAF8040000EB400080B210F0D4FA47F8040F08B911F071FE761EF1D1E81D62
:20675000FF21082211F0C7FEFF2105F11000082288F87B1411F0BFFE022703234FF6FF7CED
:20677000012288F88C3405F19400A8F88EC4042100F8042F417083707F1EC170F8D105F1A9
:20679000A0000526022700F8042F417086707F1EC270F8D1BAF8047085F8A8304FB12146A9
:2067B000D8F80C057F1E084401F11801A0F802C0F6D1022088F8700498F8FC024D4618B1D3
:2067D000D8F8000300B180470CF07CFD98F92A0411F01CFB10F0BEF811F00EFB11F09AF9BE
:2067F00011F08CF9464F072657F8040B00B18047761EF9D111F0CAF9464606F14C00016811
:2068100009B10EF031FB3F48006886F85640C0B112E038460FF02EFA029002A80EF024FB20
:206830001EE038460FF026FA019001A80EF01CFB12E068460EF018FB0AF0E8FF0028009014
:20685000F7D131480078012802D02046FEF730FF2E4806F178070470B06F0028E1D13F1D35
:20687000F06F0028D5D1B467F4672948C6F8880186F88240274FC6F88C71274BC6F890314B
:2068900086F88340254AC6F89421B4702449C6F8981186F88440234FC6F89C71224BC6F823
:2068B000A031254B214AC6F8C0302149C6F8A421224A204FC6F8C420234BC6F8A8112049B6
:2068D000C6F8AC711F4FC6F8C8105846C6F8CC70A968C6F8D030884706F21141522000F0E7
:2068F00035F896F82B040DF0CBFD0CF0EBFC2046BDE8FE8F080200208C1C0020D017002065
:2069100010030020482E00203D1D0020522E00208707010033840100F96B010091940000B3
:2069300011DF000019730100DD5F010069BB000029A70000A55B010007FE000049AF00009B
:206950005D2A0100F10C0100713201002DE9FE43994E80460F46B8F1450F08D106F50F7450
:206970003422204611F036F9C6F8F04321E110F0A9FDFF2808BFF42000F01C818F4C04EB29
:206990008004A07810B9E178002937D0E178814208BFFB2000F00E81B8F1580F24D0B8F1CF
:2069B000600F1AD0B8F1E00F0ED0B8F1E80F05D03A7890421FDC91421DDB1FE080493878C1
:2069D000097888421AD1F4E097F900000CF000FE4FF6FF7181420ED010E038880A280ADBF6
:2069F000B0F5804F07DA09E038888F2803DB47F60251814202DCE820BDE8FE83724D686806
:206A100080478146207862783946301800F57A7011F0E0F8A968484688474046503800F07B
:206A3000C680801E00F0AD80401E00F0BD808D3800F0B580401E00F09B80401E00F0AC80ED
:206A5000801F1ED00D3840F0B4800E2096F869748DF8020017B11B208DF8020096F92A1479
:206A70009DF90200884204D0E0200DF10201FFF76DFF10F05FFE96F86904002800F09980E4
:206A900073E0012103208DF8051030278DF8030000248DF808704FF4FA558DF8064096F8C9
:206AB0003B14ADF80050052081298DF8040009DB842907DA8DF8030014278DF808700820D0
:206AD0008DF804009DF8030096F80D14884204D04F200DF10301FFF739FF9DF8040096F872
:206AF0001914884203D0572001A9FFF72FFF96F83B04842808DB862806DAC0208DF8080020
:206B10004FF4FA47ADF800709DF8080096F81D14884203D05A2002A9FFF718FFBDF80000EC
:206B3000B6F81A14884203D058206946FFF70EFF96F83B0478B902208DF805000B278DF841
:206B5000074020498DF806707D260E80E7200DF10701FFF7FBFEF7200DF10501FFF7F6FE48
:206B7000E1200DF10601FFF7F1FE0DF045F820E096F82B040DF084FC01281AD01A20BDE8B4
:206B9000FE8396F8110418B902200EF01DFE10E0022011F08DFA0CE010F0B0FF09E096F908
:206BB0002A0411F033F904E010F0B4FF01E011F023F90020BDE8FE83080200205003000012
:206BD00043060020941C0020D01700202DE9F04142F20400ADF1280D0DF123010DF0EEFC0A
:206BF00042F205000DF122010DF0E8FC42F2010069460DF0E3FC8B4C8B489DF82310C4F85C
:206C1000A80164204143C4F8A0118849C4F8C4119DF822104843C4F8BC018548854EC4F8BD
:206C3000E001B07888B342F203000DF106010DF0C5FC10F079F805460DF1060029460CF0DB
:206C5000AFFF2D1A9DF8220084F89B5170B1009860B104F5DC700DF023FB04F5BA7009F0CA
:206C70000FFF012084F8940184F8980142F202000DF106010DF0A2FC0DF1060010F0F4F9E8
:206C900004F5CE700DF00CFB11E042F202000DF106010DF093FC0DF1060010F0E5F904F516
:206CB000CE700DF0FDFA04F5BA700CF081FD96F83B040FF0A5F9C07B022804BF012084F8C6
:206CD000F40194F8F801002840F0A88004F128000021382211F0FFFB0026A681E08900EB76
:206CF000800080B280460FF0F7FF04F12805074627610FB911F0B7FB38463146424611F027
:206D1000EAFB4D484D4FE06305F1080067630DF0C7FA42F21B0001A90DF050FCBDF8040089
:206D300001A9A4F84C0042F21C000DF047FCBDF8040001A9A4F84E0042F21D000DF03EFC4C
:206D5000BDF8040009A920835D200DF039FF9DF8240000280CBF301C012084F85C00B4F8C6
:206D70004C0038B100EB401080B20FF0B5FF0028606551D0B4F84E0040B1410001EB800107
:206D900088B20FF0A9FF0028A06543D0208B38B1C00080B20FF0A0FF606108B911F063FBBD
:206DB00027490DF11A00082210F014FF01273546208BA84223DCB4F84C50668355B1606DC3
:206DD0004FF6FF720146A0F81F206D1E8E7701F12100F7D1B4F84E504DB1A06D4FF6FF715A
:206DF000024681806D1ED67002F10600F8D1201D3146062211F06FFB84F8F8710EE06069C4
:206E10000DF11A01082200EBC50010F0E3FE6D1CADB2CDE711F027FB11F025FB0AB0BDE84F
:206E3000F081C046BC0F0020014301003DCC0000D98301000802002019B90000002A751585
:206E50004C040000F0B500215022ADF15C0D02A80BF09CF8F22016A911F0B2F88F4DBDF84D
:206E7000580016A9A5F87000F32011F0A9F8BDF858000DF10901A5F87200E22011F090F87A
:206E9000688DADF81200410806D305F11401096805A80160BDF81200810805D3291D09888B
:206EB00006A80180BDF81200C10807D305F1180109680DF11A000160BDF81200010908D384
:206ED0000DF11E0005F15401302209F03FFDBDF81200400903D3286B1590EF6A14977048DA
:206EF000007800280CBF0121002101200AF03AFBBDF8120041082CBF0F240B24810824BFBB
:206F1000A41CA4B2C10824BF241DA4B2010924BF3034A4B2400924BF0834A4B220460FF03E
:206F3000C3FD071C00F0B78005260DF1090100F8016B0A68026049684160BDF8121008306B
:206F500011F088F9BDF81210844648080BD3BDF81410604611F07EF9BDF8161011F07AF98A
:206F7000BDF812108446880807D3BDF81810604611F070F9BDF812108446C8080BD3BDF805
:206F90001A10604611F066F9BDF81C1011F062F98446BDF81210434A9388080961D3BDF831
:206FB0001E10604611F056F9BDF8201011F052F9BDF8221011F04EF9BDF8241011F04AF910
:206FD000BDF8261011F046F9BDF8281011F042F9BDF82A1011F03EF9BDF82C1011F03AF901
:206FF000BDF82E1011F036F9BDF8301011F032F9BDF8321011F02EF9BDF8341011F02AF901
:20701000BDF8361011F026F9BDF8381011F022F9BDF83A1011F01EF9BDF83C1011F01AF900
:20703000194611F017F9117811F014F9BDF8421011F010F9BDF8441011F00CF9BDF846100E
:2070500011F008F9BDF8481011F004F9BDF84A1011F000F9BDF84C1011F0FCF8BDF812102D
:207070008446480906D3149960460EF042FC15990EF03FFC05F11C01224630463B4604F030
:207090007DFA0820ADF80260074D01972968ADF800006846884717B0F0BDC0465816002093
:2070B000F21900206C140020F41700208F492DE9F04F06460822ADF16C0D15A810F08AFDCC
:2070D0008B4C94F8F30106F1280A06F12807002800F008817078002840F00481FF20854BA5
:2070F0008DF818001D78F06C012105AA01F042FEDFF80492DFF8048228B99DF8180008B9D7
:207110009DF81C5070BBB08900F00700022814BF04200520B073B08900F00700032807D167
:2071300073684046001D01681878042800F09C8096F83000022815D149468878012811D029
:2071500001F57A710D4606F12800022220310FF00FFF38B905F116010DF13E0011F06DF9A9
:207170000DF13E07706E002800F0BC80012102AA0AF0B2F9002840F0B5809DF80800B073CA
:20719000F06C40B1394612AA0DF14A03FBF7FAFD002840F0A7800DF14A000090706E39466F
:2071B00012AB06F0FFF8002840F09C804946891C0878012854D04FF4005013A90DF0FEF95D
:2071D00013A815A908220FF0D3FE30B113A8394608220FF0CDFE002842D194F89901002894
:2071F0003ED0D4F88851B4F8846142F2010004A90DF0E4F9049A4FF000410020E2FB05104F
:20721000051CD4F8900110F082FE2D180498A84202D8761C2D1AB6B24746786880475FFAED
:2072300080F8D4F88001A84205D1B4F87801B04208BF00260BD0C4F88051A4F878610020B8
:2072500084F875010FF090FF0126C4F88C01B968404688470EB10BF061F9012084F898016E
:20727000002084F899013DE0CDF85CA08847AB46234D0A274FF00008CDF864A096F830902B
:20729000189014F809A0287A484505D11999524628460FF06DFE20B17F1E05F10C05F2D122
:2072B00000E0A8465FEA08070FD194F870011449451C870084F8705107EBC0077F18E8B24F
:2072D0000A2804BF002084F87001179938460A2210F080FC09491898896887F80AB08847CB
:2072F0000420B0731BB0BDE8F08FC0464C040000BC0F00201B1D002008020020D01700207E
:20731000B41000202DE9F043071CADF1240D00F01381F86B002800F00F81B7F84020002A76
:2073300000F00A81007817F130014FF0000603D097F83810052902D0002E00F0FD80DFF8B0
:207350000482401E69D0801E55D07F4CC01E3DD0001F40F0F1807A4DA878002800F0EC805C
:2073700003A8314604220AF011FEB7F840002A78032840F0E180F86B401C10F071FF4346A7
:2073900003F17C073988012A01F10101398009D0D988421A022A05DBB3F87E108918491EEA
:2073B000A3F87E10D880E7782E70400808D2012F00F0C2800121E17030460AF0D3F8BBE072
:2073D000002F00F0B980E6703146F5E7012A40F0B3800725E0788DF8205000280CBF012180
:2073F000311C3046E1700AF0BDF8E07802228DF8210028460CE0012A40F09E804346B3F891
:207410005C000122401CA3F85C0004208DF82000394608AB04F0B2F88EE0684631460C2230
:207430000AF0B4FDB7F840000B285ED1FC6B14F8010BC14689F82800204610F011FFA41CDB
:207450000346204610F049FC0546201D10F045FC8046387A4C4689F82400022806D039680F
:2074700004F11C0001607A68426001E03888A08303F00100190928BF40F00800590928BFC4
:2074900040F010006085834218BF0226B5F57A7FADF8020016D32D48A84213D3E56210F034
:2074B0003DFC814610F03AFC00EB092910F036FC00EB0920B0FBF5F16943401A0A300EF054
:2074D000F5FF00E00226E06AB8F57A7F019008D342F21070404504D3C4F8308010F032FC9A
:2074F00000E00226206B029001E04446012602258DF8016068468DF800500DF045FA0DF1FB
:2075100011009DF801108DF8105010F0A3FEBDF8021010F09FFE01990EF0EBF902990EF0A5
:20753000E8F939460D2204AB284604F027F8B4F86200401CA4F8620009B0BDE8F083C0463D
:2075500024170020581600206C140020407E05002DE9F047DFF80CA20746AAF13500DFF809
:20757000F8810068800880F0E7800FF0C5FA814908310B6800261C17641C990D0AD2C0F17B
:207590003E0110F10A0F4FEAE101D8BF08218C42B8BF0C1CDFF8C4C1990E0FD2590E0DD30F
:2075B0006246143A1168C1F304211629A8BF20391268C2F30462162A0EDB0CE0634AD2F853
:2075D0007C11C1F304611629A8BF20391268C2F30442162A00DB203A09199146162905DAF5
:2075F00011F10A0FB8BF6FF0090100E01521584C584D01F01F0242F4F85222802A6812F059
:20761000030F18BF0126D20828BF46F002060FB146F00406424692F90740041B052C04DAC3
:207630009479B44208BF918866D00F28A0F10F0827DB08EB0014A4F1F0084FEA282EBEF16E
:20765000070F88BF4FF0070E7546062D88BF06255CF82570042404EB850465462C59E41B51
:2076700004F0FF05F70824BFC4F307273D44B70824BFC4F307473D44770828BF05EB1465C3
:2076900001E00025AE465CF82EC0F7080CF0FF0424BFCCF307273C44B70824BFCCF30747A1
:2076B0003C44770828BF04EB1C64ADB2A9EB0101A8EB0E277D43002905F1800504EB15241C
:2076D000D8BF012103F0FF0334254D43A9B259434FF6FF73B1FBF4F18B4238BF191C802823
:2076F00089B2918005DA10F1800FB8BF6FF07F0000E07F20D0719671194800681F29106022
:207710004FF0000008D340F2FF128A4206D24908401C8A42FBD301E01F219180124F0F3936
:20773000090940EAC10047EA0001CAF8FB1F0026CAF8FF6FBDE8F0870C490D4F424608205B
:207750000F60921D1070BDE8F087C0463C1100506E620840242208403C2E00209C1300508D
:20777000082009403500094000E7A48030100940FDFDA400AC3F005001282DE9FE4F40F0E1
:20779000EE80DFF810B2DBF8DC00012840F0E4800220CBF8DC000FF057FD01200DF086FBB3
:2077B0005FEA000805D00120CBF8DC000FF05CFDD7E010F078FE6C4902900020086001205E
:2077D0000EF0C0FF012818BF002003D100200BF0B1FC0120654900900020654F08603868E5
:2077F000112010F025FD00280CBF00240124102010F01EFD08B144F002040F2010F018FD68
:2078100008B144F004040B2010F012FD30B1624814300068574E016B308888470A2010F030
:2078300007FD002600B101264FF0805A0AF5DC75301C04D02868504E016B308888474F48F5
:20785000012606602868816944F0200088474C48066010F0E7FC00F001010191400814D25F
:20787000484810F092FC8146B9F1040FF8D0B9F1010F05D1DAF8D801426842480321904724
:207890004149086820F0030008600020FFF760FE2B683868986B8047019801280DD0B9F1A9
:2078B000010F05D1DAF8D80142683648314690473549086840F0030008602C4806602868BE
:2078D0004169204688470B2010F0B2FC20B12868284BC16A188888470A2010F0A9FC20B1D2
:2078F0002868254BC16A188888472448032206602349CBF8DC2000230B602868416B20468C
:2079100088470128F9D1386804200DF0CFFA044615481E490660386808688009FCD3009897
:20793000012802D130460BF005FC10F069FC08200DF0BCFA07460298CBF8DC6010F086FE1F
:20795000134800880BF058F90FF08EFC57EA040018BF4FF0FF3804E06FF0040801E06FF03E
:2079700001084046BDE8FE8F0C400940000222432C2009405E0900005A090000282008602B
:2079900080010443004003402422084014100940FC0A000058130020A40100102DE9F04302
:2079B000002B08BF002A10D10029BCBF00204FF0004106DB50EA01071CBF6FF000006FF0BA
:2079D00000410AF0FCFCBDE8F0835FEA530898EA610803D50026404266EB01015FF0000992
:2079F00013F0004E03D00026524266EB03031C461546002C08BF8D429CBF2C1C0025070CE8
:207A100047EA01470E0CB44208BFBD429EBF240444EA15442D04070A47EA01670E0AB44212
:207A300008BFBD429EBF240244EA15642D02470847EAC1774E08B44208BFBD4200F2928049
:207A5000870847EA81778E08B44208BFBD427BD8C70847EA4177CE08B44208BFBD4265D832
:207A7000070947EA01770E09B44208BFBD424FD8470947EAC1674E09B44208BFBD4239D876
:207A9000870947EA81678E09B44208BFBD4223D8C70947EA4167CE09B44208BFBD420DD8BE
:207AB000E60146EA5566EF01B14208BFB84201D3C01BB14159EB09094EEB0E0EA60146EA1D
:207AD0009566AF01B14208BFB84201D3C01BB14159EB09094EEB0E0E660146EAD5666F01A9
:207AF000B14208BFB84201D3C01BB14159EB09094EEB0E0E260146EA15762F01B14208BFAA
:207B1000B84201D3C01BB14159EB09094EEB0E0EE60046EA5576EF00B14208BFB84201D3B7
:207B3000C01BB14159EB09094EEB0E0EA60046EA9576AF00B14208BFB84201D3C01BB141D8
:207B500059EB09094EEB0E0E660046EAD5766F00B14208BFB84201D3C01BB14159EB09096F
:207B70004EEB0E0EA14208BFA84201D3401BA14159EB09094EEB0E0EA34208BFAA423EBFBB
:207B90002D0A45EA0465240A8AD373464A465FEA080803D50026404266EB01015FEA48086D
:207BB00003D50026524266EB03031E4617460B46024631463846BDE8F08370472DE9FE4F4B
:207BD0000CAF9946934604467D680291294604F08FFA061C00F0EE803888F082774F347553
:207BF00097F8FC0218B1012C04BF1520307506F1840029460B220FF0EDFF012C04D00D2C19
:207C10001CBF7068401C00D170683062002597F8FC0235650028B5654ED0052C18BF012C29
:207C300045D14FF0040A86F86BA0F08A86F86950C00934BF97F80D0497F8360459460A22A7
:207C500086F86A0006F170000FF0C4FF9BF8080003282CD1032097F8113402903BB3DFF8F2
:207C7000608108EB8408D8F8000010F47F0F0ED086F82CA0D8F8000006F12C01012200F4FF
:207C90007F003063304602F097F9D8F8000010F0FF0F0CD02A2086F83C00D8F8000006F145
:207CB0003C0100F0FF003064304606F043FF97F8FC0208B10D2C13D0009502994B463046AD
:207CD0005A46FCF769F8071C75D1E41F012C03D8707E40F020007076304606F08FFF6AE0C4
:207CF0000520374C86F86B0004F13400016811F0F70F18D02A2186F83C10BA78006806F1BC
:207D10003C01012A00F0FF0030641CBF20F00800306497F8110418B9306C20F0020030642A
:207D3000304606F007FF009502994B4630465A46FCF732F85FEA00083AD1224806603489E4
:207D5000756801A964200CF03BFF1F4EA01C0DF1050187B206F180000780E9200CF030FF3A
:207D70009DF80500012806D13C46C4F30220022140F0180006E0241D0421A4B2C4F3022018
:207D900040F0080005F8010D671A05F8014DB9B2C6F88C50AD1C284609F0F4FC9DF8040006
:207DB00000280CBF09480A48C6F8C800C6F88800474600E01A27F8B2BDE8FE8F080200209D
:207DD00008010000D01A0020701500204E9055550E7A55552DE9F043044694F830900F46ED
:207DF000984615468B20ADF1340D0DF10A0102F04BFF8A20694602F047FF94F82500002801
:207E10003ED1B9F1000F19D1BDF80A104FF6FE70884205DCBDF80A1088422FD1694615E036
:207E3000B4F844009DF80A608DF80C0000128DF80D00BDF80A008DF80E601BE0B9F1020FA6
:207E500009D0B9F1030F19D104F1280103A810F0F4FA092612E0207CC00934BFB4F8420075
:207E7000B4F844008DF80C0000128DF80D00208D8DF80E00001205268DF80F00002013E0A9
:207E900002280CBF05260926012818BF04F11C0104D1892006A902F0F7FE06A9324603A88B
:207EB0000FF098FE94F826000DEB0601C8723A4603A831460AF048FA002840F08F80B9F143
:207ED000000F19D1BDF80A104FF6FE70884205DCBDF80A1088422FD1694615E0B4F844003F
:207EF0009DF80A608DF8200000128DF82100BDF80A008DF822601BE0B9F1020F09D0B9F117
:207F1000030F19D104F1280108A810F096FA082012E0207CC00934BFB4F84200B4F84400A7
:207F30008DF8200000128DF82100208D8DF8220000128DF8230004203E6881460BA98220DF
:207F500002F0A2FE9DF82C10307B8142D8BF9DF82C00002842D007460024722029460EF03E
:207F7000B7FDB0689DF82C100019C8F80000007881422FDD2B68C10001EB001158182860EB
:207F90000146D8F800004278012A1FD0807828BBB9F1040F06D0091D08A80FF057FC012827
:207FB00016D017E008884B888DF82800042208A98DF82A3000128DF8290018128DF82B0074
:207FD0000AA80FF0E1F9012802D003E0807828B9002004E07F1E04F10304BED1F3200DB053
:207FF000BDE8F0832DE9F047064637680C465FEA0208ADF1180D14BF00214FF0FF3107F15E
:20801000480081460FF0A7FF002818BF0B2040F0E68000257448FC60B8F1010F057007D09A
:20803000657002200EF012FA06200EF00FFA01E0012060702078012840F29080801E012866
:2080500057D9801E01282CD9801E012800F2B88010F00FFA8246A078009021782846062974
:2080700008BF0120019001200290A068228A6368E16806F063FB0746504610F0EFFA002FAD
:2080900040F0A080B8F1000F02D00FF0EFFC02E030460EF029FB002800F0878010F0F7F983
:2080B00021E010F0E6F9012782460097A168A278606824782B46042C08BF3B1C07F0F0FE1E
:2080D0000746504610F0CAFA002F7BD1B8F1000F02D00FF0CBFC02E030460EF005FB0028A0
:2080F00063D00EF03BF93F49C1F8B0510D60074668E010F0BEF98246E08A0090E068019075
:20811000208B0290A0780390207D04900121059122782846022A08BF081CA368E178626831
:2081300002F00CF80746504610F098FA002F49D1B8F1000F02D00FF099FC02E030460EF007
:20815000D3FA002831D00EF039F9071C3AD1E078A168E28A236909F063FDC8E710F089F9D8
:208170008246E08A0090E0680190208B0290A0780390207D049001200590277807B90546DB
:20819000E1786268A368284602F054F90746504610F064FAB7B9B8F1000F02D00FF066FC58
:2081B00002E030460EF0A0FA08B9142017E00EF0EDF8071C06D1E07821690CF0E9F896E7BA
:2081D0004FF0FF37B8F1010F05D002200DF07CFE06200DF079FE484610F061F9384606B03D
:2081F000BDE8F08750450240512E00202DE9FF4705466878002840F0E98095F89A10022933
:208210001CBF0329E82095F88F108029C8BFE82095F89010092901DB0A2900DDE82095F8FB
:20823000911009B1042905DB8029C0F2CE80882980F2CB80002840F0C9806948007888421B
:2082500004D005F19101E820FEF780FB05F19001E720FEF77BFB05F18F01E120FEF776FB54
:2082700005F19C015020FEF771FBDFF87C8195F89A0002280CD04FF6FE70A8F8080405F134
:20829000920108F2FE3010F0D8F805F1920604E005F192063088A8F8080408F5FE7005F17E
:2082B00084010B220FF096FC4FF001090220A5F816903146287501A80FF0E4FA95F89E7088
:2082D000B5F89CA0686805F19E01002FA0F1010068600CBF002048464F780FB140F0020085
:2082F0008F780FB140F00400CF780FB140F008000F790FB140F040004F790FB140F0800044
:2083100069684A1E6A6008702F7D69680024481C2862781E087028892C6598F8FC32AC6524
:20833000801C002B288141D0042785F86940E88A85F86B70C00934BF98F80D0498F836046A
:2083500031460A2285F86A0005F170000FF042FC95F89A00032829D105F1700005F19201A5
:2083700010F06BF898F8110400B31E4E306810F47F0F0CD085F82C70306805F12C014A465C
:2083900000F47F002863284601F016FE306810F0FF0F0BD02A2085F83C00306805F13C010D
:2083B00000F0FF002864284606F0C4FB00942846832101AA5346FBF7EFFC071C02D12846E4
:2083D00006F01CFC381C01D106E0E82068701820287028460AF070FB0090BDE8FF87C0462F
:2083F0004306002010010000080200202DE9F0411C4615468C4208BF854282BF00230022E3
:20841000E5E0002C08BF002D0AD100290EBF00286FF000006FF0000100F0E1F8BDE8F081D0
:208430005FF000085FF0000E002C08BF8D429CBF2C1C0025070C47EA01470E0CB44208BF8B
:20845000BD429EBF5FEA044444EA15445FEA0545070A47EA01670E0AB44208BFBD429EBF2A
:208470005FEA042444EA15645FEA0525470847EAC1774E08B44208BFBD4200F29380870803
:2084900047EA81778E08B44208BFBD427CD8C70847EA4177CE08B44208BFBD4266D8070965
:2084B00047EA01770E09B44208BFBD4250D8470947EAC1674E09B44208BFBD423AD88709AA
:2084D00047EA81678E09B44208BFBD4224D8C70947EA4167CE09B44208BFBD420DD8E6011C
:2084F00046EA5566EF01B14208BFB84201D3C01BB14158EB08085EEB0E0EA60146EA9566B2
:208510004FEA8517B14208BFB84201D3C01BB14158EB08084EEB0E0E660146EAD5666F0137
:20853000B14208BFB84201D3C01BB14158EB08084EEB0E0E260146EA15762F01B14208BF62
:20855000B84201D3C01BB14158EB08085EEB0E0EE60046EA5576EF00B14208BFB84201D360
:20857000C01BB14158EB08084EEB0E0EA60046EA9576AF00B14208BFB84201D3C01BB14191
:2085900058EB08084EEB0E0E660046EAD5766F00B14208BFB84201D3C01BB14158EB08082B
:2085B0005EEB0E0EA14208BFA84201D3401BA14158EB08085EEB0E0EA34208BFAA423EBF54
:2085D0002D0A45EA0465240A89D3734642461E4617460B46024631463846BDE8F0817047D5
:2085F0002DE9F04F754C6068ADF12C0D002840F0E28004F178063068002800F0DC80DFF8A6
:20861000C89109F123000078022800F0D4806D4D281D006880470A90A06F074678B3684EE9
:208630004FF0000A4FF01D083B7D0820711E11F8012F9A421ED0401EF9D164483946524620
:208650000DF0FEF8787E30F07F0005D194F88300401E84F8830004E094F88200401E84F874
:20867000820087F8018057F80CBC384608F0A8FE5F4602E0BA4657F80C7C002FD4D13520AE
:2086900008F0B2F9A9684E46002862D1452008F0ABF9A968002856D1684601A909F090FEE7
:2086B0004A48006838B1017D252904D050F80C0C0028F8D113E090B196F89801002838D04B
:2086D0000FF0E0F900280CBF04210D21009F96F82B02401AB8421FD8012086F8950115205D
:2086F00008F082F9A968A8B10A98884760680DF10601703001F040F910BB96F82B02009966
:20871000884203D91C2002F013FA54E0002086F896010AE00A984DE0252008F065F9A9689A
:208730000A988847002086F89501042001F0B8FA41E0252008F058F9A9680A988847192053
:2087500001F0BAFD37E00A98884708200BF0B2FB31E00A98884796F8F401B8B10EF0E4FCBD
:20877000B18901B9F1893269491E89B201EB81018918D1F801100FF078FE42F21071814268
:2087900092BF00206431081AC0B200E000206968002808BF0620D9D0C6F8D80188470446F0
:2087B000D6F8E011D6F8D80106F5F4720DF024FBA968204688470BB0BDE8F08F0802002077
:2087D00044040000D0170020BC0F0020800200202DE9F04106460C467148DFF8D8C1DFF8C8
:2087F000CC81754F724902883046D12810DCD1287BD0713800F0B280401E00F0AC80401ED1
:2088100000F0A580113810D04C3800F0888007E0D23856D0401E41D0401E33D0401E28D051
:2088300030460FF0A1FBFF2802D1F420BDE8F0815C4D05EB8005A97809B9E87850B1E87831
:20885000884208BFFB2000F0A880227891426BDC904269DB544E70688047074628786A786A
:208870004146401821460FF0B5F9B1683846884792E02278022A57DA0846641C00EB8200EB
:20889000042286E021888A424EDDC8006746182200EB011039684018241D7AE02678304649
:2088B000022841DA2C2505FB0670611C102200F2A5400FF08FF9606905FB0671C1F8B804DA
:2088D0006AE02178607802292EDA02282CDA2C2200EB410502FB0173461C07EB45070222B6
:2088F00083F8A46407F204502FE02178608802291ADA824218DD2C2303FB017595F89C3410
:2089100007F26C429842A4BF431C85F89C3402EB8102D2F8901000EB40000322BBE7207853
:208930006678022800DA16B1E820BDE8F0812C21751C331801FB007282F8945458000A22E3
:2089500000EBC300C01900F59D60A41C21E01CB3084608221DE0FCB1604691E7B4B907F258
:208970006C4007F2644200F17C0100F190030227983042F82C1F53F8044B10617F1E01F19A
:208990000A0100F104009460F3D105E040465822243021460FF01EF90020BDE8F081C0461D
:2089B000901C0020AC000000D0170020740600201807002014070020080200202DE9F0479D
:2089D000064668480D4601681F461446ADF1380DBDB1B4B128784FF0010808FA00F001423D
:2089F0000FD01046002104F099F97560B4600FF040FD5D4C82462078022804DB50460FF0BF
:208A10002DFE0020ABE0002863D103F08DFC5749086840F0020008600AA80FF021FBDFF84A
:208A30005091544999F802000AAA0C9004F1A8000CF052FE0AA80FF0EBFA002519210AAB32
:208A50008DF8305099F800004B4A0B9004F14C000CF014FD0AA80FF003FB99F8030047491F
:208A70000AAA0C9004F1DC000CF036FE0AA80FF0CFFA99F801008DF830801A210AAB404ADA
:208A90000B9004F168000CF0F9FC3E492A4604F1840013460BF00CFF3B4A04F1200004214F
:208AB0002B460EF051F8A570E57025716570E560072084F890010523A3614FF4FA71C4F80A
:208AD0001811324AC4F81C11314815700FF086FB207804EB8001401CC1F81061C0B22070EA
:208AF00050460FF0BBFD44461FB903AF38460FF051F9386830607868F060387C3074B86965
:208B100074743062788A7082224DB561F5617561F86800B1B061786900B1F061B86800B150
:208B300070610021A02206F1280009F02FFA06F1400000210DF048FE68460FF039FC164954
:208B5000029606F1780000226B460BF0B1FE134906F19C0000226B460BF0AAFE30460EB0E8
:208B7000BDE8F087D4210840F823002000200940CA0B00005D7C0100353901009DF8000035
:208B9000AD1C0100B9720100194601004F2E00200DD90000CB7B0000B976010027840100CA
:208BB0002DE9FE43DFF8C081704D0E46B00958D3444604F17C074DE00178D0290EDBD029BE
:208BD00009D181783970C17879700179B97085687D60C168B9600FF0D0F948E004F15005FE
:208BF000286009F069FF28460CF03EF93FE0884794F88410491E84F88410A96888470098DE
:208C100001788DF8041020654378CBB1DC2B0DD0DD2B0BD0E42B09D0F32B07D0DE2B05D0F4
:208C3000DF2B03D0E82B18BFDB2B0BD105F068F99DF80400162805D168460CF015F901E0DF
:208C500009F03AFF9DF80400162803D004F150000CF00AF938460DF00DF8002869680090DB
:208C7000C5D1F00BA9464446C00305D0404F08F0CDFD002800909FD1700905D32E208DF8A5
:208C9000040001A809F018FF700805D325208DF8040001A809F010FFB00805D326208DF8DD
:208CB000040001A809F008FFF00805D327208DF8040001A809F000FF300905D329208DF8D7
:208CD000040001A809F0F8FEF00908D300208DF805002D278DF8047001A809F0EDFE300A56
:208CF00008D300208DF8050030278DF8047001A809F0E2FE700A08D300208DF805003527B2
:208D10008DF8047001A809F0D7FEF00A08D300208DF8050023278DF8047001A809F0CCFEA5
:208D3000B00A08D300208DF8050036278DF8047001A809F0C1FEE06CD9F8041080B18847FC
:208D5000E16C00270091D9F80810E7648847009804F15006306009F0AFFE30460CF084F8F4
:208D70000020BDE8FE83C04608020020D0170020801C00202DE9F043894614460546ADF14F
:208D90002C0D69460DF002F85FEA000800F0C580AD1C0226284602A90BF059FA071C00F0F3
:208DB000BC809DF80900814509D0ED19BF1908F10200BF1CAD1CBEB2B042EBDCADE0401E99
:208DD00005F1020500F08D80401E50D0801E33D0401E26D0401E20D0401E18BF622040F0E1
:208DF000AC80202F40F099802046294608220EF0F1FE083504F10800082229460EF0EAFEFA
:208E100005F1080704F11000082239460EF0E2FE07F10805183408220BE0022F7DD10222A8
:208E300007E0202F79DC2046002120220FF053FB3A46204629467DE0042F6ED12046294688
:208E500002220EF0C7FEAD1C15F8010BA070287800F00100E0702878C0F340002071287884
:208E7000C0F38000607128784011A07164E00A2F53DD0DF11200002116220FF02CFB20463A
:208E9000294604220EF0A6FE2D1D201D022229460EF0A0FE42F20B0004A90BF08FFBBDF8AF
:208EB0001000A188884238DCA81C10F8011BA17110F8011BE17110F8011B217210F8011B40
:208ED000C1F3C202A2720DF1120200F0B1FB20B39DF82700A0819DF81670E78104F1100010
:208EF00025E0042F19DD0DF11200002116220FF0F2FA15F8010B207015F8010B607015F841
:208F1000010BA07015F8011B0DF11202C1F3C2002071284600F08CFB08B967200DE09DF834
:208F30002700E0809DF81670278104F10A0011220DF116010EF04EFE00200BB0BDE8F08353
:208F50002DE9FC41DFF8AC810026054688F8A962687D062803DBE82088F8A902687DA97D7F
:208F70000E2905DD032803D0E82088F8A902687D032806D1B8F8540040083CBFE82088F8E1
:208F9000A90295F8280010B1E82088F8A902E87D092801DB0A2802DDE82088F8A902287E11
:208FB00008B1042806DB802801DB882802DBE82088F8A90208F52A77294638460DF03CF9DA
:208FD000291D112207F12C000EF004FE95F8280008F52A74002804BF88F8F062A87D04D0DE
:208FF00095F8290088F8F002688DA8F8E602687E88F8E802A87E88F8E902E87E822788F84C
:20901000EA02287F98F82B6488F8EB0298F83A3488F8EC72384F88F8ED6298F83B24C8F840
:20903000CC72042688F8D06205F11D0188F8EE3204F1490088F8EF220B220EF0CBFD98F800
:20905000A90200284ED1687800284BD1287E98F8AA728DF8000017B1EA2088F8A90205F120
:209070001701E720FDF772FC98F8F00228B1287E022808BF01208DF8000098F83B049DF863
:209090000010884203D0E8206946FDF75FFC1B4C98F8AA32277867B9B8F80E0418490880D0
:2090B000C3B1032B12D0052B05D0012B03D0022B01D00FF0B3F9022020700BF091FE4FF6EE
:2090D000FF70A8F80E040F49088005E00BF088FE032000E0012020702720287030460EF012
:2090F00043F901E02A202870284609F0E5FCBDE8FC81C04608020020E1800100882D002090
:20911000A41A0020B21800202DE9F04FADF1240D079003F009F9614800780DF067F9604D9C
:209130000024012808D90A380FD0801E04D0401E0ED0401E09D006E00EF02CFC022804BFF2
:2091500001210C1C06D0696805E005211F2401E0032107246960534A1068C0F38150012805
:2091700006D152F80C0C0127020E07FA02F004430EF06EFF524AFF234018401E471C28606A
:209190007F1E02F8013BFBD1079A1268002702F0FF03FE2B20D0DDF81CC096463B4601269C
:2091B0000EF0FF02FF2A10D0904205D3914203D806FA02F2144201D002206CE017430EF05E
:2091D000FF02DFF8FCE00EF802305CF804EF5B1C0EF0FF02FE2AE5D1092006F0FDFA079843
:2091F0000121A86005F128000DF0EEFA05F19806A8464FF0010A4FF0040B0025A9460AFA00
:2092100005F0044216D1074204BF05F0FF0141F4C04104D02A480799405D51F8201022487F
:2092300004F0BCFCE8B24FF0FF310EF0DBF9C6F8009001E0C6F800B0D8F800006D1C361D4E
:209250008542DCD904A80EF0E3FE184C184A2078102104AB059008F10C000CF00FF968466D
:209270000EF0FEFECDF80C906A4660681149029008F164000CF030FA0F4951F80D0C20F4CE
:20929000F85040F4005041F80D0C0C4FC1F8FFAF4846C7F800A009B0BDE8F08F502E002076
:2092B00044120020B43F0050007FC767B00B0000117601000D5201000D30094008000940BE
:2092D000881200202DE9F84F6B4C064694F86101002800F0C880B4F80E04B6F8421088428E
:2092F00040F0C18006F128000DF0A6FC002800F0BA80002594F8110484F8615110B1022006
:209310000EF032F894F8070210B101200EF02CF8307C400905D310200EF026F880200EF0C5
:20933000D7FE20200CF050FA04F5067008F07AFB72685178107804F5027A00EB0120C0F387
:209350000321C0F3003784F85D11C0F3031384F8143400F00F0184F85E7194F8370484F8EA
:2093700062110F2804D0884202DDD77807B9014684F8F51394F8F5B384F83852BBF10F0FD8
:2093900009D194F85F0102286DD10CF005FE06F07DFEBDE8F88F39480078012802D00120DE
:2093B000FCF786F9314F7868804780460DF0AAFD0CF044FC81462E4850F82B002063606368
:2093D0000AF04AFEA16A48460CF04EFE0AF01CFDB9684046884794F85F0102280FD1504645
:2093F00008F020FB94F8F52304EB4200B0F824014FF470719140091A50460DF095FD94F8DF
:209410001474308929460AF0B3F8C4F854010F2F14D094F8F51394F85D01B94208D0401C07
:209430006FF00F06B8408101A1EB8005AD1905E0401CB8408501A5EB8005A03DC4F8585141
:20945000022004F5A27584F85C01284608F0EAFA0848C4F84C01D4F8581128460DF064FD4D
:2094700010200EF035FEBDE8F88FC046D017002040010000211E0100080200203D1D00201D
:20949000F8B507466848B0F854200021930804D2B7F89E30DB0828BFE82112F0600F04D1CE
:2094B000B7F89E20920828BFE821604E3B8906F1080212889A42B8BFE82197F89C5035B9D3
:2094D00097F89850002D08BFF52100F0A880002940F0A580D7F8AC5090F8FC1215B901290C
:2094F00003D026E0002900F0998097F89840002C18BF032C05D1D7F8AC5045F00A05C7F814
:20951000AC5015F0FF0F07D02A21D7F8AC5087F83C1005F0FF01396415F47F0F07D004214F
:20953000D7F8AC5087F82C1005F47F01396390F8FC12002449B397F89850426804216DB95E
:2095500025223A754268D28AD20934BF90F80D0490F8360487F86A00801C08E015233B7581
:20957000D28AD20934BF90F80D0490F8360487F86A0087F86B100A2207F1700087F86940B7
:2095900007F190010EF026FB01E00120387597F8A050B7F89E00FD7697F8A130F8827A6869
:2095B0003B7797F82C103A622546BD650F293D650AD0B7F8A80007F12C01224600B9012281
:2095D000384600F0F9FC04462CBB97F83C00FF2801D1B86D28B107F13C01384605F0AAFAD9
:2095F0000446C4B9009597F89C10B7F89A3007F190023846FAF7D0FB041C0CD1308939890F
:20961000884203DB384605F0F9FA04E0E5207870384607F0D5FE211C01D1F8BD1821384698
:2096300007F0D8FCF8BDC046080200208C1C00202DE9F04F154601F00708C1F3C2074FEA3C
:20965000A119044683460C22ADF11C0D002168460EF041FF5FEA080034D0012879D101A8BA
:20967000594603220EF0B6FAE41C14F8010B022200F00F0021468DF808000DF10A000EF033
:20969000A9FABDF80A60A41C0721DDF804C052486E754268624507D1027A9DF808309A42AC
:2096B00002D14289B24206D0491E00F10C00F0D10020014601E0017840788DF800108DF87A
:2096D00001001FE014F8013B14F8016B41488DF8003007218DF8016010F80C2F9A4202D17C
:2096F0004278B24205D0491EF6D100200246114603E04268017A4089687501928DF808100C
:20971000ADF80A0003A806F0B7FD9DF800009DF80110B8F1000F10D0B8F1010F19D1019826
:20973000049A9DF814109DF80860424071408918BDF81600BDF80A2004E09DF80D309DF8FC
:209750000C2059405040081803D1EF701FB1022F07D000203BE0281D214602220EF03AFA3C
:20977000A41CB9F1010F27D0B9F1020F2CD1BDF80A10281DC91DCA1021460EF02BFABDF89D
:209790000A00C11D04EBE104F0B1401E811000EB5171C910C9B249190E798210012700EBDE
:2097B000527222F00702801AC0B2401C07FA00F0FF303040087107E0291D20460AF01EFDA1
:2097D000207804EB8004641CA4EB0B04A0B207B0BDE8F08F54100020601000202DE9F84FB2
:2097F0000F4680460DF0A9FE4FF6FF71814208BF682000F0B8805D4E440004EBC004A4194C
:20981000D4F8026016B9D4F8065025B3D4F80610B14208BF692000F0A6806078401E13D0ED
:20983000401E09D0801E16D13868864200F295808142C0F092800EE03888864200F28D80F3
:209850008142C0F08A8006E03878864200F285808142C0F08280464E7068804742F2020B3D
:20987000DFF8109100904046A0EB0B0001282FD90A3801281CD9C01F49D1207862784D4625
:209890000021281800F5FE700EF025FE637838460EF023FE05F5FE798342D8BF181C02DD7B
:2098B00038460EF01AFE2178024601EB090034E00DF03AFAB668398888424CDD20786278A5
:2098D0004D463946281800F5FE700EF083F928E00DF02AFA0546384629460AF061F9B66876
:2098F0002D1A5FFA85FABAF1000F34D0207862784D463946281800F5FE700EF06BF9584654
:20991000404514BF85F89BA185F89AA109E0207862784D46281800F5FE7039460EF05AF90D
:20993000B6680BF11900404504BF0020A5F884020BF11A00404513D1B5F88472B5F8820206
:20995000C119322901DC07430AD10220A5F882023027A5F884720098B0476A20BDE8F88F4E
:209970000098B0470020BDE8F88FC046D8040000D0170020BC0F00202DE9F04F80465F4C62
:2099900098F80800A7780D46ADF1140D0228CDF80C8014D1012F12D004F57A7140460222EE
:2099B0000C4620310DF0E4FA38B903208DF8080004F1160168460EF040FDCDF80CD02FB300
:2099D000DFF848B198F808904D4CDBF8040014F809A080470A266427F8340490207A4845F1
:2099F00005D15246204641460DF0C2FA20B1761E04F10C04F2D103E00027EF72A07A2873F6
:209A1000DBF8081004988847002F73D03C49DDF80CA04FF0000864278B468E6DB1F84E00D3
:209A300085F81E804446D9460AE0BAF80010761C2134B6B233E0B9F84E00641CB61DA4B29C
:209A5000A04218DDF0780028F5D0B0880AF078FC514608220DF08CFA0028ECD1F078A87774
:209A7000308800046860B08885F80B80A5F81F00B07847462873DBF85440002F3AD085F8E9
:209A90001E8042F219000DF10A010AF097FD0DF08BFB81461B480188642746468246B1422C
:209AB00028DDA07F0028C0D0B4F81F000AF048FC039908220DF05CFA0028B6D1E07A022865
:209AD00003D0E07A80B161270FE0BDF80A000E4A6168424348460EF011FA28B9A07F6C2712
:209AF00040F00800A07700E047462846214621220EF070F8384605B0BDE8F08F080200209B
:209B1000BC0F002008100020808D5B00D01700202DE9F843614C5A4D5A4EDFF870815E4FE1
:209B300094F8E4100846401E0B2864D8DFE800F07B2C43062343062343067664042907D01D
:209B500001220A2945F8212C14BF0220032004E0202045F8210C0120024684F8E200002088
:209B700045F8390C0827C5F8FF7FC5F8F37F45F8392CBDE8F883052914BF09200620002781
:209B900084F8E400376075E094F8E170383D0120002FC5F81B0004BF0620002102D00021F2
:209BB000F160032084F8E400032045F8010C3160306880085ED294F8E41033480127032924
:209BD0000ED00068456800216022052300914046A84794F8E400062814BF0A200720CFE739
:209BF00000684568002160220523022000904046A8470420C4E7FEE72548264F002601256C
:209C100006600E203D6005F001FB02200CF05CF984F8E45084F8E360BDE8F8830020386058
:209C30000C25786024E04FF08059D9F8A0010168202088472C3D0F2045F8010C41F61D5679
:209C5000C5F80360D9F8A401466800214FF4C0720723022540460095B047D9F8A401C66813
:209C700000214FF4C07207234046B0470120386084F8E45004F178000EF0EFFBBDE8F883B9
:209C900039400C4038600C40A401001000A00C402C500C4004800C4034600C405813002067
:209CB00059492DE9F8430F78002F40F0A9805F4D564C574B8846012101286E6860701F685C
:209CD00088F8001021D9801E42D0401E10D0401E30D0401E2CD10020F18A2071C90934BF52
:209CF00095F80D1495F83614A1700EF011FA55E095F83B040CF084F9C07B022802D10020E3
:209D100006F0D6FD0CF0E4F948E00021F78A2171F90934BF95F80D1495F83614A17088B969
:209D300095F8EB0370B10229C4BF0220A07009E00EF074FB96F86900207196F86A00A070B1
:209D50000027677106F028FC686840BBBDE8F883DFF8C09099F800008600F86B8047D9F8B6
:209D700004103C22401AB0FBF6F0B0FBF2F151432278401A9101A1EB8201091AF86B3C31CC
:209D90001FFA81F98047244906FB090088677C31087820F00F0040F00200087068681F49C5
:209DB000097861B960B34168087800F02000E0708878A0710878800901D20EF06FFA607830
:209DD000032818BF02281DD1154D68688047617802290CD013490F7817B913490F7837B102
:209DF000022188F80010A9688847BDE8F883832188F80010A968884709F09EF8BDE8F883DD
:209E10000EF00CFBBDE8F883572E00208C1B002078180020B01B0020701500204E2E0020C5
:209E3000D0170020532E0020552E0020080200202DE9FF470446880FC0F0B18000200AF065
:209E5000CFFA58480EF04CF901200DF0EDF957480EF0C4F9564A002140F60A00108002F164
:209E70000C0551802B7861F303032B7002F10D0751603B784FF0010A6AF303033B70A66887
:209E90004C4B7180DF788C460D4607B95546677C3D4318BFD4469046328899466546A2F64D
:209EB00002076FB141F21E02BF1A09D006F119031A7861F382021A707DB106F1180208E036
:209ED00006F111031A7861F382021A702DB106F11002138861F309131380844661743546D4
:209EF000ACF10702531C00E03D466F6837B13888844503D0824218BF8342F5D1C5F8048058
:209F100005F10D07387861F30300387009F134000EF0C1FA8068008882421BD0834219D0C4
:209F3000278DCFB104F12803E16204F1340259801078353461F30300107020786AF30300B6
:209F5000207008F10D07C8F80430387861F30300387001E0C9F80C103046694604F012F9CF
:209F700068460EF06DF80DF06FFF99F8010068B950460CF0E7FB01280ED00D3528786AF3E8
:209F90000300287008480EF029F905E00BF086FB0028FBD00EF07DFA30460EF0A1F8009040
:209FB000BDE8FF8701010E046546010039360000082E0020F82300202DE9FE4F07461046A0
:209FD000002F00910CBFE821002101910099002900F0AC800199002940F0AA8060B178683E
:209FF000401E7860F82101707868401E7860002606703889801C3881DFF83C81009C4FF05A
:20A0100000094FF0020BCDF80890C246083C14F8080F00F00F010F2900F08580012821D0C8
:20A0300004287AD19AF8FC02002876D0DAF8141360688847061C26D03889B7F84C1080198E
:20A05000801C81421FDB7868DAF818C36168029B3A46801BE047B0B178683989801B891922
:20A07000786059E0009A029804254A44D21C12F8011FFF2941D021293DD13989B7F84C303E
:20A090000B318B4202DA1A20BDE8FE8F7968B8F82434491E79601B120B707968491E79606D
:20A0B00098F824340B707968491E7960029E0E7098F826147B68197098F8223479681B01D5
:20A0D000491E796043F00F030B7098F814C498F8F5337968491E796043EA0C130B70796887
:20A0F000491E796021260E707968C01D80B2491E796005260E706D1EB9D17968C0F30122A6
:20A11000491E796042F088020A707968491E7960087039890918891C3981BBF1010B09F12C
:20A1300008097FF474AF7868B86501E0E82001900198BDE8FE8FC046080200202DE9F04FA1
:20A150008A4609AF4FF08051ADF11C0D90463D69059001F5D8700490D1F8B001D7F808B0AC
:20A170004169069327208847524C4FF00309143CC4F884970126C4F87C67C4F880970220AB
:20A19000C4F8FC06F868C4F8080430460EF031F9D4F808040008F8D2D4F88C07800F28BFAC
:20A1B000B14655D2681E41460C238DF800000DF1010011F8012B5B1E00F8012BF9D1022DE6
:20A1D00019BF0020011C98F80C1000208DF80D108DF80E008DF80F000099C4F83C15019B83
:20A1F000C4F84035029AC4F84425039BC4F848353968BAF1020F4FEAC542A1EB0A08A2F5B4
:20A21000002106D34FEA4A52A2F580026FF315021143264A0A43C4F84C258246C4F8508536
:20A23000BBF1000FC4F854A5214DC4F858B511D02E6078682060C4F808B030460EF0D9F8DF
:20A25000D4F88C078008F8D3D4F88C07000801D3CA4627E0C4F88497D4F88C0710F0030FA2
:20A27000FAD1D4F8800720F00200C4F880073F7D47B1049F3868016A2720884738680169D9
:20A2900027208847C4F87C670598C4F8806748B12E6006982060C4F80880C5F8006420622D
:20A2B000C4F82880504607B0BDE8F08FC80104200000484218400240F8B55A4C064694F87D
:20A2D000FC02002798B1D4F8342382B1D4F8540368B142F21A0069469047D4F854038047B0
:20A2F00028B19DF8000010B1E12E08BF012794F83B040BF085FEC07B02280CBF0525012558
:20A310006068002800F08C80002E71D01B2E06D1017D052903D094F86A34002B68D0E92E8F
:20A3300027D037BBE12E15D10DF016FD88B16068C18AC9080ED294F81C14817694F80A14C5
:20A350004A1C84F80A24406881702846FFF7A8FCF8BD60681C2E4CD1616A00294DD0884778
:20A370003149002009786060012959D0FBF7A0F9F8BDF1200DF093FA6768B87E48B90DF0C1
:20A39000EBFC20B16068C18AC90832D2D3E760682FE07868398907F0F5F978680088000984
:20A3B00005D394F8FC0210B10BF078FE6768F88AC00811D3387E00F07F003876387D032849
:20A3D00003D1787E40F004007876F0200DF067FAE168606888470FE014490126B87E0E700C
:20A3F000401EB876F0200DF05AFA11480078ADE70026467006F0E4FF6068C08A000A0AD34D
:20A4100094F8FC0218B994F82B040AF039F894F92A040DF0FBFC0020606010200DF058FED9
:20A43000F8BDC046080200203D1D00204E2E00208D1B00202DE9F04F894609AF4FF080515D
:20A45000ADF1240D9246059038683D69079001F5D8700490D1F8B001D7F808B041690693BD
:20A4700027208847504C4FF00308143CC4F884870126C4F87C67C4F880870220C4F8FC0650
:20A49000F868C4F8080430460DF0B3FFD4F808040008F8D2D4F88C07800F28BFB04653D2C5
:20A4B000681E51460C238DF800000DF1010011F8012B5B1E00F8012BF9D1022D19BF0020F9
:20A4D000011C9AF80C1000208DF80D10019B8DF80E0000998DF80F00029AC4F83C15B9F130
:20A4F000020FC4F84035039BC4F844254FEAC542C4F84835A2F5002106D34FEA4952A2F5D2
:20A5100080026FF315021143254A079D0A43C4F84C258146C4F85055BBF1000FC4F85495C7
:20A53000204DC4F858B511D02E6078682060C4F808B030460DF05DFFD4F88C078008F8D311
:20A55000D4F88C07000801D3C14624E0C4F88487D4F88C0710F0030FFAD1D4F8800720F03F
:20A570000200C4F880073F7D47B1049F3868016A2720884738680169272088470598C4F895
:20A59000806740B12E6006982060C5F800642062079FA760A762484609B0BDE8F08FC0465D
:20A5B000CC01042000004842184002402DE9F843584CA76B4FF0FF300DF004FA002F00F0E7
:20A5D000A080010925D2810801D3266C0EB307F1100292E86000002105400E4008BF002D0E
:20A5F00000F08F803A693E6A07F1180510403043386295E80C00E76307F1180619431043F7
:20A6100086E8030004F1A8004FF480410DF04FFF77E039693E6A41F00A010840304338629B
:20A6300007F1180696E80C004FF00008384DC4F83880002119432E1F104307F1180383E88F
:20A65000030006F108033A691868904307F11002186092E803003068091C42468843394661
:20A67000306004F1440081460AF0CCFA04F1A80002210DF01CFF206C002842D0206CF968EF
:20A69000C06888423DD1206C90F82F1097F82F00084310F0070016D000F0010100F0020776
:20A6B0000F4304D1216C2F310A78104304E0216C2F31087840F001000870216C4246484604
:20A6D0000AF0A0FA1BE0206CA063206C0169CA432A6028680142FBD1206CB16800690843C7
:20A6F000B060206C103003C8083D081CC0432860206C3768103003C8081C38433060C4F88E
:20A71000408006F0A3FE04F053FFBDE8F883C04610100440F82300202DE9FE4F4B49DFF8F9
:20A730003C81486891F8FC2200284FD0484C494FDFF824A1012A11D0606880473F7847B994
:20A750005246A16817782FB9832342461370884765E0A1680223424613706CE0894699F827
:20A770003B040BF04DFCC07B022804D14148C01C007806F09DF80BF0ABFC394D286A394E63
:20A79000016CF06888478346606880473F780290002F47D150460078002843D1D9F84813B7
:20A7B00000208847F42001A90AF00AFA2E4F9DF9040058451ADC7B79C3B9A1680298884752
:20A7D000D9F8486378787C79042801D00DF026FE04214046641C0170E0B278710EB10320F1
:20A7F000B0470320388102F0A7F925E0832140462A6A0170536CF0686A4600219847B5F93B
:20A810000600BDF90010884214BF002001200AF009FBA16802988847F8791449087008F0D0
:20A830008BFB09E0022140460170A16802988847D9F84813042088470D480078012802D026
:20A850000020FAF735FFBDE8FE8FC04608020020D0170020532E0020552E0020572E002051
:20A87000581800209C1A00208C1B00201B1D00203D1D00208D1B00202DE9FF410446666893
:20A89000A7680D460DF0F5FD3178012903D10DF0E5FE00208CE0012131700DF0DFFE287807
:20A8B00070706878B07068687060A868B060E868F06028693061287D3075687D7075A87DED
:20A8D000B075A869B061287F3077687F7077A87FB0774FF00008C6F82080C6F83080454619
:20A8F00075627563B562B56386F82C5086F82D50786804F071FF204605F024FB204606F05B
:20A91000A3F970B92C480068C16838688847786804F07CFC0DF0ADFD35700DF09FFE2C464A
:20A9300045E068460DF074FB0094387B234A0190B9686B4606F17C000AF0A0FD68460DF0FC
:20A950008FFB00941E4938696A46029006F198000AF0C2FEB07830B906F1CC0029460BF0F8
:20A9700033FF18483061707830B906F1E80029460BF02AFF1448F06068460DF019FD01955E
:20A990008DF800501149029406F582700A226B4609F08EFFB969FA6906F13C000DF0D2FA11
:20A9B0000B4A06F16800042123460CF0CDF820460090BDE8FF81C046D0010010EDB70000DE
:20A9D000C55A0100B1830100A9830100A5180100318101002DE9F04F06464FF00108ADF1ED
:20A9F000640D0922B07D8DF84C8006F117018DF84D000DF14E000DF0EDF84B4D68688047EF
:20AA1000179016A9812000F03FF9707D002840D09DF85800022817DA042000238DF80300FB
:20AA3000347D8DF802809DF858708DF8013069468DF80040781C8DF85800D220FDF7C8FEAA
:20AA5000812016A9FDF7C4FEDFF8E0A000274FF0FF0B3C46B94618E0307D69460DEB8000BC
:20AA7000C0F81090D420FDF7B3FE01E08DF824B08DF82670307D8DF8257008A98DF8200063
:20AA9000D120FDF7A5FE641CE4B2BAF80000A0422ADC307D00279DF84D208DF840000DF1D5
:20AAB0004E018DF841700DF142000DF093F88DF84B80D02010A9FDF78BFE071C0FD1307D13
:20AAD000314610228DF828000DF129000DF082F830690AA90F90D320FDF77AFE0746A968CA
:20AAF00017988847F8B21CE0307DADF8224008A980F001008DF82000D12000F0C5F80028E1
:20AB1000B4D19DF82400FF28B0D0ADF800006946D42000F0B9F800289ED0A9681798884732
:20AB3000192019B0BDE8F08FD0170020901C00202DE9F843504C80466068002800F0998060
:20AB5000DFF83891B8F1000F18BFB8F1E90F17D14D46AE892F690CF017FB06EB8606F61931
:20AB7000C6F80100A88995F8F521014601EB81017A54E989401C80B28142D8BF0020A8810C
:20AB90003F4D6868B8F11C0F37D0B8F1000F0BD099F82300032807D1B8F1E10F04D0002097
:20ABB00089F8F201072000E0052009F083F9676899F8230003280FD077B10020FE8A87F894
:20ABD0006900F00934BF94F80D0494F8360487F86A004046FFF770FB99F89701012848D172
:20ABF00068688047044607F0D3FFA96820468847002089F89701BDE8F88380470646616820
:20AC10002048C98A0078C90804D294F88310814204DB28E094F88210814224DA616804F1E4
:20AC300078000CF0C1FB6068C08AC00805D294F88300401C84F8830004E094F88200401C6B
:20AC500084F88200A968304688476068007D252819BF012089F89601012089F89501002095
:20AC70006060BDE8F883A96830468847F120FFF723FBBDE8F883C04608020020BC0F00202E
:20AC9000D01700208C1C00202DE9F04107464F480C46018838467138022840F293801338EE
:20ACB00027D0DFF834814C3877D0401E62D0401E4DD0401E3BD0DFF824C1401E2BD0401E4F
:20ACD0001AD038460DF050F90646FF2E11D0404D686880473F4A0746B000115C80184278F3
:20ACF0004346C91820460CF075FFA968384688470EE0F420BDE8F0812178022962DA6046E8
:20AD1000641C0422001D00EB810120460CF062FF0020BDE8F0812088814253DDC1006746F1
:20AD300001EB001138681822241D0918EDE72678022E47DA2C25601C05FB06811022393117
:20AD50000CF048FF05FB0680C06C6061E0E72278022A37DA60782C2303FB028393F83830F2
:20AD7000414683422EDD00EB420001EB40010222983125E02078022824DA61882C2202FB2C
:20AD9000008292F830208A421CDD08EB8008D8F8900001EB41010322C6E72178022911DAF8
:20ADB00060782C2202FB018292F828204346824208DD401841000A2201EBC001C9187C31D9
:20ADD000A41CA2E7E820BDE8F081C046901C0020D0170020AC0000007406002014070020A2
:20ADF0002DE9F8434C4E84460120002430704B484D4D04704A48DFF82C81047005F1560032
:20AE10000088B14614EA03074FF0020606EA020608BF002E13D120464FF0E04710401F4008
:20AE300008BF002803D11D2006F07CFE4FE0454695F90000401E28700CF0B4FE47E04246F7
:20AE500092F90030394E5B1E137043F20842824207D06F8F931C834203D0BA4218BFBB4275
:20AE700016D1304608300068826C60469047008843F6030181420AD004F010FE98F9000065
:20AE900000283DD098F90000002837DD3FE06F8FB5F8721043F60400884220D0B8421ED075
:20AEB000B5F8562090421AD0B1F5505F05D0080B0BD31D2006F036FE07E01D4801683046F6
:20AED00001F5C071016003F0FDFE0CF02FFE98F90000A8B198F9000000280FDD17E01548E0
:20AEF0000078022810D003280ED004F0D7FD98F9000028B198F90000002808DC0DF08EFA63
:20AF10002046FAF7D5FB02E0204606F00BFE89F80040BDE8F883C0463D1D0020741C0020A2
:20AF3000731C00207A1C002070150020701800200C0100218D1B00202DE9F04705466C78DD
:20AF5000ADF1180D002C40F08B804A48B5F89A100088884218BFE82405F1900101A888469B
:20AF70000CF090FC444E01A80BF066FE30B995F89D0030B1707820B9E82471E0002085F8F0
:20AF90009D00002C6CD195F89D0000280CBF0120052004272F754146E8820DF10E000CF070
:20AFB00071FC686895F89C40401E6860411E6960B5F89A9004702B7D69680024481C2862B7
:20AFD000581E087028892C6596F8FC22AC65801C002A288136D085F86B7005F170004146BA
:20AFF0000A220CF0F7FD95F8980005F1700A032828D105F1900150460DF01FFA96F8110496
:20B0100000B31E4E306810F47F0F0CD085F82C70306805F12C01012200F47F002863284698
:20B03000FEF7CAFF306810F0FF0F0BD02A2085F83C00306805F13C0100F0FF00286428460A
:20B0500003F078FD0094284603210DF10E024B46F8F7A2FE041C02D1284603F0CFFD2CB127
:20B070006C701A202870284607F026FD06B0BDE8F087C04616060020080200201801000033
:20B090002DE9F0474E4C4B496FF00100383CA76B087027B994F8F5030F2840F08980464865
:20B0B000DFF818810121002F8146017072D0206B7968884221DB0AF0A5FD7968884267D392
:20B0D00094F8F503A56B0F2812D1002D62D00AF099FD696888425DD3A66B706800280CD407
:20B0F000304606F09FFCB168307B8847A56BECE7002D4FD06E68002E01D50DF08FF9AA4628
:20B110002F7BAD680AF07EFDB0420DD2A06B30B1216B4068814202DD0AF030F93AE00BF020
:20B13000F1FE0020A06335E03846A8474646301D006880475546824604F1280128460CF078
:20B15000DFF920B904F12C0128460CF0D9F9A06BA84218D10027A06AA76387420BD0216B87
:20B170004068814207DD0AF04DFDA76A79688842C8BF7860A763E56A2DB11FB17868696859
:20B19000884200DDA563B16850468847A56BAFE708F03AFE464670688047044603F066FAD4
:20B1B000B168204688470CF0EFFA002089F80000BDE8F087711C00203D1D0020D017002061
:20B1D000400200202DE9F0414D4C04F1440840460DF061F9071C00F09080B86840F6030281
:20B1F0002026531C02E04068761EF6B260B15EB101888A4218BF8B42F5D1F9682CC8283137
:20B210002CC149C881E849003A6A00263E627D6835B397F82F0000F00700401E0BD0401EEB
:20B2300006D0801E18BF002308D14FF0805304E04FF0804301E04FF00053324697F82F0016
:20B25000000908D397F82F0010F0070F03D04FF08070324303437D68F868B7F92C10A84749
:20B270000DF007F90546B4F94A00401C6FF31F30A4F84A00606C80F82F6040460CF0BAFB82
:20B2900028460DF0EBF9B4F94800B4F94A10884233D1F86890F8C20000280CBF052007209C
:20B2B00005F0B8FA04F588742568F868854208BF656890F8C240002C0CBF0468341C80F8E5
:20B2D000C2604DB195F8C23023B92868A04228BF041C01E085F8C26064B1B4F1FF3F0CD016
:20B2F0000849F86809687830B4FBF1F10CF000FDBDE8F08108200AF0F5FCBDE8F081C046A5
:20B31000F8230020442E00202DE9F04FFF25ADF1140D8DF800504FF6FF79ADF80290ADF8AA
:20B3300004900AF005FEDFF81CB104900BF1020000880027001F84B2082C64DBC846464625
:20B35000C246201F02A9082280B20AF0D7FFBDF80800814508D1BDF80A10894506D1BDF83A
:20B370000C20924502D107E0BDF80A1051EA000314D1BDF80C308BB9BDF80E00C10BCB037C
:20B390000AD100F108018C4238DA0CF039FE04980CF098F9002050E0241F31E0C20BD30345
:20B3B0002AD1C20B28D3BDF80C3000F0FF02954203D1884508BF9E421ED0C5B28DF800507F
:20B3D0008846ADF802801E46ADF804609DE80600384607F005FB78B9BDF80E20A01A07F135
:20B3F0008851001F083280B292B20AF087FFBDF80E00C019083087B2BDF80E00241A083CC3
:20B41000A4B2082C9DDA09F063FC3FB10C484FF088513A460CF078FF0CF048FD04980CF09B
:20B4300051F95A46507800281CBF0020011C03D1C7F58054391DA0B2518005B0BDE8F08F54
:20B4500004E00100A01C0020F0B5494D014695F807020027ADF1140D002855D195F8EA0355
:20B47000002851D0087ACF68C0F3021600F0070100E0BF1C0846411EC9B248B17A78387879
:20B49000B5F8124400EB0220A042F2D102270FE005F57A74443400E008373046411ECEB2FB
:20B4B000A0B3204639460CF0D1F90028F4D0032795F8070240F0040085F8070202A80BF073
:20B4D000CFFB01200BF050FF05F5FE718720FFF7DBFB05F501718520FFF7D6FB05F2052156
:20B4F0008620FFF7D1FB05F206218820FFF7CCFB0120009005F5FE760196B5F80E3439462D
:20B5100002AA0520FCF75AFB002F2ED195F8F5030F282AD095F81414814226D095F811040E
:20B5300018BB95F8560000BB12480078012802D00120FAF7BDF8104C6068804795F85F110E
:20B55000022910D195F85C11FF290CD0696851B9A96F41B9A168884705F5A27006F062FAAE
:20B5700006F056FC01E0A168884705B0F0BDC046080200203D1D0020D01700202DE9F04F52
:20B59000994692460C468046ADF13C0D0BF0BCFD434D3C2205F1100108600021684606F00F
:20B5B000F5FC20686E4630606068706020893081207A032804D0022003248DF80C0002E077
:20B5D00003248DF80C40287818B105F134000CF0EFFCA88EADF80A0068781F28B4BF411C0D
:20B5F00000210027B8F1050F697040F080000BD0B8F1040F05D0B8F1020F08BF40F0600030
:20B6100004E040F0200001E040F040008DF80D00ADF828A04FF0010BCDF8249021498DF8E3
:20B630000EB00A680BA80260496841608DF8354005238DF83640B8F1050F8DF8343012D0BE
:20B65000B5F85E00B8F1040F08D0B8F1020F0FD1B5F86400401CA5F8640009E0401C80B2BC
:20B67000A5F85E0004E0B5F85800401CA5F858000D4918206A4613F0ABFDC0B258B1B8F178
:20B69000050F09D1E86A0AF011FFB5F85800401CA5F8580000E05F4638460FB0BDE8F08F14
:20B6B00058160020D90700005D6400002DE9FF470446080BC0F08480434DA8680421026AAD
:20B6D000A970D20802D3C369002298473F4905F14C0000220CF0D3FE3D480CF07FFDA8689F
:20B6F0004168886808B9C86810B13A480CF0F8FC012008F075FE38480CF0F2FCD4F808A013
:20B710000022AAF80220A0680188A1F602072FB141F21E017F1A18BF183000D1103001887E
:20B7300040F60A06F31F4FF0010962F3091103F101080180514684F8119000E039464F68A1
:20B7500037B13888864203D0834218BF8045F5D14A6001F10D06307869F30300307005F123
:20B7700034000CF098FE8068008883421BD04346834218D0208DB8B104F12800E26204F131
:20B79000340542802B78353462F303032B70237869F30303237001F10D074860387862F359
:20B7B0000300387000E02A615046694602F0EAFC68460CF045FC0CF047FB50460CF090FCFF
:20B7D0000090BDE8FF87C046F8230020D9720100393600005100070601010E042DE9F84FD3
:20B7F0008046D8F808603068D8F80450076CDFF814A147642A6C6B6CA86B17F4F06F0146A4
:20B81000A2EB030932D1F8091DD2780966D3A9B196F821205046801D845C601E814294BF02
:20B830000C1C641E404621460AF040FAA86B001BA86353D105F198000CF03BFE40464946F8
:20B850000AF0C4FE4AE00029F8D040460AF02EFA95F82D10A86311B900283FD101E0002081
:20B87000A86305F198000CF024FE37E0FA0A19D24FF000094C4602E0A86B401EA86348B3C8
:20B89000404601210AF012FA3068446814F00F04C0F80490F0D0286B401E2863686B401ED6
:20B8B000686317E0306844680022202904F00F044260CCBF4FF0200B8B46404659460AF079
:20B8D000F5F9CBF120008145C8BF8146494640460AF07CFEEC77404607F0FAFBB8090FD379
:20B8F000A96A69B10F4640460AF034FAA86238B996F820205146895C4046C91908F0E8FD7E
:20B91000BDE8F88FD00900002DE9FE4F0BF04CFC434C04F1280202901168E0624FF40050DE
:20B93000491C1160694608F049FEDFF8FCA0DFF8FC90B4F8520000285FD0A66DB4F84E00FB
:20B9500000254FF6FF7BA0462F4654E0B07F800822D3B6F81F0008F0F3FC014608226846E5
:20B970000BF006FBC0B1716802982E4A0CF0C6FA90B9B6F81F00B77709F040FBA6F81FB0BE
:20B99000DAF800008047B4F8503013B15B1EA4F85030D9F808108847B8F84C006D1C2136E5
:20B9B000ADB235E0F078800821D3B08808F0C8FC0146082268460BF0DBFAC0B1308801040E
:20B9D000184A02980CF09AFA88B9B088F77009F015FBA6F804B0DAF800008047B4F85230C9
:20B9F00013B15B1EA4F85230D9F808108847B8F84E006D1CADB2A842D4DCB4F8500048B1AF
:20BA1000A046666DB8F84C0000254FF6FF7B2F46A8429BDC04F1300008F042FCBDE8FE8F1A
:20BA3000BC0F002000A493D6D4170020D01700202DE9F04F3E4E3D4CDFF8F890F06804F1D6
:20BA5000B801ADF1140D04F1B80A814206D1494691F90000002818BF002064D1384D281DD6
:20BA7000006880473449834600200F78A4F8BA00002F07BF4FF48601021C304920228046E6
:20BA90008DF80D002F462F48324C0378CDF808809B0904D20078000938BF012000D30220CA
:20BAB0008DF80C00306A056D284B27488DE806000068514602AAA847B9680028A778B0804A
:20BAD0000D4603D55846884740462CE0494691F900001F4B002F00F10100087093F9000084
:20BAF000C6F80CA000F10100187014BF80204046B6F84C10B4F80E74B4F812344FF67F72F9
:20BB10000A40104301430822A6F84C1006F14F00A6F85A7004F22C41A6F858300CF05AF88B
:20BB30005846A847012005B0BDE8F08F70150020581800207B1C00200405002000004F8C7E
:20BB5000D0170020542E0020A81A0020DF8401007A1C002008020020B0B504464548007852
:20BB7000002800F0828094F88F00002871D13520207504F19101112204F170000CF02AF8EF
:20BB900004F13C00FF2110220CF0A5FC04F12C000F2110220CF09FFC94F8900004F13C0509
:20BBB00000283ED0401E29D0401E14D0401E5AD12A20287002272764042305F8103C4FF4D4
:20BBD00010222263032184F86B10204607F0DEFB071C3BD137E02A200A2728700423276442
:20BBF0004FF44C1205F8103C02212263204684F86B1007F0CBFB071C28D124E02A200227F6
:20BC10002870042327644FF4102205F8103C01212263204684F86B1007F0B8FB071C15D155
:20BC300011E02A2002272870042327644FF4502205F8103C00212263204684F86B1007F04E
:20BC5000A5FB071C02D1204602F0D8FF381C0DD1B0BD01280CD10848D0F80C038047002854
:20BC700008BF002002D0192000E018200CF0E2F8B0BDC04604050020080200202DE9F041C7
:20BC9000054628798028D4BF0020E82069790026092901DB0A2900DDE820A97909B104290E
:20BCB00003DB80296FDB88296DDA00286BD1394C94F8F5030F2866D0B4F80E144FF6FF704F
:20BCD000884260D0B4F8081488425CD0E87901280BD040B1FF2856D194F85F01002852D1C1
:20BCF00001273E4602E0012700E0022704F50670804605F097FE04F5027005F093FE04F5CC
:20BD1000A27005F08FFE2448001D0068804784F85F7167680246FF210020C4F85801002FE0
:20BD300084F85C110CBF0121011C84F86111012E84F8606108BF032084F8380213488168C2
:20BD500010468847A91DE820FAF700FE691DE720FAF7FCFD291DE120FAF7F8FD94F861015F
:20BD7000012802D120200CF0A3F9094894F8F5134FF47077C4F8200207FA01F000F263614A
:20BD900040460BF00FFDBDE8F081C046D0170020BD40010008020020D01700202DE9FC475B
:20BDB00005466E68D5F80880B76B002F18BF4FF0FF307CD131630024F477171C74631BD002
:20BDD00006F13C090CF055FB82466946484609F074FB00281ED450460CF040FC9DF80000E1
:20BDF000316B0870306B736B7F1E00F10100306303F101007063E5D17078726B316B01287C
:20BE1000A1EB0201316303D1F36828469847726B14464BE0B76350460CF020FC0CF029FB29
:20BE3000244D0746287820B902200AF00FFB0120287038460CF012FCD8F80010086B40F4CD
:20BE500000700863D8F80010886B40F4FA608863707808BB716806F1E80738460CF07BF854
:20BE7000B8B1B463384621460CF075F888B10CF000FB0746287818B102200AF025F82C7029
:20BE900038460CF0EBFB1027716B306BF777401A3063706BBDE8FC8796F82D0030B1706BAF
:20BEB00020B1B46306F198000CF003FB2046BDE8FC87C0464C2E002070B50546434C287834
:20BED000ADF1200D002858D1B4F8400004F150066B88ADF800003146ADF81030E2200CF00D
:20BEF0005FF80DF1120031460CF027FA698853200BF0FCFCB4F8400004F146063146ADF897
:20BF10000E004A200CF04CF801A831460CF015FA00268DF80D60B4F84400ADF8020094F8F3
:20BF300042308DF80C3030460AF0D8FA522031460BF0D0FC94F858000F2807D00120A070A9
:20BF5000B4F8441020704B200BF0D0FC606928B102681AB10DF10E0069469047032007F08C
:20BF70001FF894F85A00032818BF042827D104F10A0010210BF08AFB21E0154E01280FD072
:20BF900002280DD00020A0700BF09AFF41F288300AF0A4FAB6F85600401CA6F856000EE001
:20BFB00005200BF08DFF062006F0FAFFB6F856000021401CA6F8560052200BF08BFCA16E38
:20BFD00009B12846884708B070BDC0462417002058160020FEB50646434C3178B4F868003B
:20BFF000E1292FD0B4F86A00E92926D0B4F86C00D9B93E4D30696F6A02903FB37F692FB315
:20C01000A96A1931814221D806208DF800000422ADF802200023ADF804309DE8030002AB2E
:20C03000B84708B90298A86210E0401C80B2A4F86C002AA00CF0E6F908E0401C80B2A4F84F
:20C050006A0003E0401C80B2A4F86800717831F07F0042D001F0600040282AD1307840BBFF
:20C07000B4F85A002569401CA4F85A000BF04CF8854203D80BF048F8401B03E00BF044F839
:20C09000401B401EB4F8827080B26421B0FBF1F080B2B842A8BFA4F88200B4F85A10B4F883
:20C0B00080304A1E02FB0300B0FBF1F0A4F88000717801F06001202906D1307820B9B4F828
:20C0D0006000401CA4F86000602906D1307820B9B4F86600401CA4F86600FEBD64617461F2
:20C0F000436E663A2000C046581600206C1400202DE9F84F05464248DFF80C8181464619CF
:20C110002D3698F8FC0234780F46C0B1D8F81413A9B109EB850ADAF8CC0000F0FF0088477C
:20C130008346D8F81413DAF8CC0000F47F008847584480B218B131780818001DC4B298F8CC
:20C15000200401280AD1387A40B148447B7A067919F803002418641DE4B200E000260D2D5D
:20C1700019D0A01900F1020A50460AF0EFFE071C19D102200AF0EAFE011C09D04D4495F86E
:20C19000490008701A274F7098F8000007F0E0FA0020BDE8F88FA719F82F01DD0CF03EF929
:20C1B00007F1020A174F3846002152460CF093F907F10C00002178220CF08DF907F13C00D1
:20C1D000FF2110220CF087F907F12C000F2110220CF081F938197860022D3E810BDB0B2D50
:20C1F00009DA7868401E78606D1E05703889641EE4B2401C3881A7F84C403846BDE8F88F73
:20C210003C000000382A0020080200202DE9F04F09AF9A4616468846ADF1440D3C893D8896
:20C23000D7F8049010900020AC428DF83C0001DACA4501D30CF0F2F8002E6BD03748875DAC
:20C25000042EA4EB07044FF00000A4B2B8BF01205FEA000B0EBF2D1BA1440024314807A93A
:20C270000823ED1B2530ADB210F801295B1E01F8012BF9D14FEA186001F8010B4FEA1843E3
:20C2900001F8013B4FEA182201F8012B01F8018B0E70234E109A306C9DF83C104369F06B1F
:20C2B00098478046B8F1FF3F24D00BA9049101208DF801009DF83C308DF8023007AA019202
:20C2D0008DF800B08DF80370CDF80890CDF80CA0ADF81640316CADF818500223F06B0A6ABA
:20C2F0008DF81430694690478046306C8269F06B0FA99047B8F1000F18BFE4200BD14FB139
:20C3100009EB040138460BAA12F8013B401E01F8013BF9D1002011B0BDE8F08F40000000F9
:20C3300008020020160600202DE9FF47424C94F8E70000286ED10127384D84F8E770E87CDF
:20C3500084F8E6006E68C4F8106168460CF030F8002604F10C0001966B468DF800603049C9
:20C370000296324608F0A4FA2E4904F130006B46324608F09DFA2C4904F154006B4681467D
:20C39000324608F095FAA96838468847DFF8A48026482A7D08F104030078254D1868C0F303
:20C3B000815A22B1BAF1030F04D184F8E170BAF1030F15D0BAF1020F12D0BAF1010F0CD089
:20C3D00002200AF043F804200AF0BCF9012804D028683221B1FBF0F10DE009F09BF912E04A
:20C3F00002200AF033F8BAF1030F0CBF4FF47A7142F210712868B1FBF0F148460CF02BF8B1
:20C4100048460CF02AF840460068C00802D230460AF01CF800200090BDE8FF87EC0A000081
:20C43000A3F00000E5010100A92D0100502E0020442E0020B03F0050581300202DE9F04F4C
:20C4500006460020ADF1140D00903E4F02917868019680473C4D03902C3D286A334CC36CEE
:20C47000E06804216A469847DFF8C4A0DFF8C8B0DFF8C88026F001062AF0010AB24519D0E5
:20C490002C4820F00100B04212D19BF900102F6AE06811F1020F08D05946BA6B91F9001064
:20C4B0009047812819D1E0682F6A2549083118E00BF0B4FF98F90010E0682F6A11F1020F3F
:20C4D00081460CD04146BA6B91F900109047812804BFD4F80C902F6A01D00BF09FFF484627
:20C4F0001749FF6A029A019BB847002818D4B24507D0104921F00101B14204BF5946087011
:20C5100001E04146087001202F6A0090E068FB6C04216A4698470B4903988968884701E0EE
:20C530000BF07CFF05B0BDE8F08FC0469C1A0020B1E9000091B00000711C0020701C00208C
:20C5500070150020D0170020841800202DE9F04105463E4804780F46002DADF1280D42D068
:20C570003B48466A002F3ED08046D6B17069C0B10123ADF8223006208DF8200029460C2221
:20C5900000236846ADF8243004F0E0F903A839460E2204F0DBF9766908A803C81A226B468B
:20C5B000B047787B012668B9002C14BF0FA013A06988102208F058F9397B13A00A2208F0E1
:20C5D00053F908E0002C14BF12A017A00BF08CFC19A00BF089FC88F802600020314604F086
:20C5F000C1FF88F803600AB0BDE8F0815265737461727465643A20307800C0465374617268
:20C610007465643A203078004368616E6E656C3A2000C04644657669636520526573746143
:20C630007274656400C046C0446576696365205374617274656400C04672657175656E6335
:20C650007920486F7070696E6700C046581600206C1400202DE9FF473A4CA11D0888401C9C
:20C6700008803949082268460BF0B4FA0AF09CFD4FF000084FF6FF7746464546824618E0B3
:20C690009DF80830616D2BB902EB421040184068010403E002EB42104018416850460BF013
:20C6B000E4FE804503D29DF80890804616466D1CADB2208BA84238DC254D281D0068804728
:20C6D0008046B4F85200B9F1000F0DD1A26D7100002301EB8601401E8918CB708A888F807E
:20C6F00080B2A4F852000EE0606D06EB461600233618B377B6F81F20A6F81F70B4F8500051
:20C71000401EA4F85000114867690088121A91B2082207EBC10069460BF05CFA608BA968C6
:20C73000401E60834046884708E0284602A904F007FC02469742A3D10BF095FE0090BDE803
:20C75000FF87C046BC0F00204C040000901C0020D01700202DE9F04707467D68D7F8088059
:20C7700091460E460BF085FE8246A86A002865D105F582700BF073FE0024EC772E625046C3
:20C790006C620BF06BFF0BF074FE304E3378824623B9022009F05AFE0120307050460BF057
:20C7B0005DFFD8F80010086B40F4807008633846494609F0CFFAA862C0B93846494607F0D5
:20C7D00087FEA878D0B9A96805F1CC000BF0C3FBE8B1AC621020E8774146284605F078FDFA
:20C7F0000BF047FE8246307840B323E0D8F80010886B40F020008863A87810B12046BDE889
:20C81000F087A96805F1CC000BF0A5FB10B9686ABDE8F0873846494607F05AFE1020AC62D2
:20C830004146E877284605F053FD0BF022FE8246307818B1022009F047FB347050460BF069
:20C850000DFF4FF0FF30BDE8F087C0464D2E00202DE9F04106AF3D793E68984604460B1CEA
:20C87000ADF1180D074611D0012B15D130797379641C3870B17904F8013B337A04F8011BC1
:20C89000B17A04F8013B7389181201E03178707804F8011B04F8010B8AB9002D0CBF42F2FE
:20C8B0000C0042F20D00694607F088FE9DF80000BDF8003004F8010B181204F8010BB8F192
:20C8D000010F34D0B8F1020F39D1002D0CBF42F2020042F203000DF1020107F06FFE7589A8
:20C8F000CDB1681E01468B100DF1020201EB5371C910CBB2811000EB517121F00701401A89
:20C91000C0B20121401C01FA00F0D15CFF3080F0FF000843D054E81DC2100DF102012046B4
:20C930000BF058F97089C01D04EBE00407E0002D14BF02210121204603F008FA2418E41B30
:20C9500006B0A0B2BDE8F0812DE9F0413B4C0546207800286FD0B4F94A00B4F948108842CB
:20C9700013D0284609F0CAFA021C06D1A16B28460BF086FB00B1A26B3AB1B2F92C102846B0
:20C990004FF0E043002200F0B9FA0BF072FD804604F588700168A94219BF00264660002621
:20C9B00006602078401EC0B2207080BBA560A07802280ED1082009F095F940460BF04EFE2C
:20C9D00005F140004FF0FF310BF0C5FA0BF051FD804604F1A8000BF064FD04F14C000BF0A4
:20C9F00046FD04F1DC000BF05CFD04F168000BF03EFD04F184000BF028FD04F120000AF084
:20CA100043FC287C012802D10E2002F0FFFBA06805F14007854208BFA66040460BF01EFE97
:20CA300038460BF03AFD05F178000BF00EFD05F19C000BF00AFDBDE8F081C046F8230020D7
:20CA50002DE9F04390460A68D8F800401678814600271D463846ADF1140D531C242E0B60DD
:20CA700053D112F8016F5B1C4C2E0B600ED1AA68E41C24F00304241D54F8040C494607F07D
:20CA900009F82968EF600127091A2960462E1AD1E41C24F00304241D54F8040CE41C029028
:20CAB00024F00304241D54F8040C002749460390AA68ADF8047001A803F00EFE2968EF60B2
:20CAD0000127091A2960532E1FD1E41C24F00304241D54F8040CE861C8F80040288B0090BD
:20CAF000A968EA69D9F800004346F7F78FFED9F80040002714B12418C9F800402968D8F852
:20CB10000040091AEF6001272960662E0AD12B8B23B9E41D24F00704083403E0E41C24F04E
:20CB30000304241D1FB9E9690E700127EF60C8F8004005B0BDE8F0833B487CB500F14402C6
:20CB50001178002565F30301324E117000F17C020564117800F1480365F3030111701A78AE
:20CB7000012161F3C3021A7000F148031A7861F304121A704FF4FA520265308908B93181FC
:20CB90000846274C2549244B097894F8FC22083148431978002A01FB00F0009035D0D4F8F0
:20CBB0003C23002A31D0D4F8400300282DD0F11D684690473179B37862681A4E65281AD096
:20CBD000A8B9107D052820D194F81104E8B9606890F82C00211D042817D10968D4F8184391
:20CBF000906D096B2B46A04778B91A2000E03570FDF762FB7CBD82F8691082F86A30D4F80F
:20CC1000401335701C2088477CBD00980AF050F87CBDC0468C1B0020B01B0020191D0020A7
:20CC300008020020572E0020701500203EB542F2050002A907F0C2FC9DF80800002864D0EB
:20CC500042F20100694607F0B9FC304D95F89401002836D020200AF043F99DF80800002430
:20CC700064229DF80810C5F88001009B85F89441581A02FB00F105F5DC70C5F8BC1107F01F
:20CC90000FFB2548007868B995F8960130B920480078002839D107F033F83EBD10200BF00D
:20CCB00017FA3EBD01A808F0C9F995F82A020199451EB1FBF0F24243891A01918D4224D92B
:20CCD00017E09DF8081064204843C5F8BC0105F5DC7007F0E5FAB5F878010124401CA5F8B7
:20CCF00078010023C5F88031202085F894410AF03BFB084991F81114204621B94FF4007066
:20CD10000BF0DEF93EBD07F0D5F83EBDBC0F00203E1D00200802002019060020F8B50146B4
:20CD30000888A0F6020058B143F20402801A04D0401E64D191F8246000E00226CF6901E048
:20CD5000CE7B4F69002F5AD000213C1F052244F23805084654F8043FB3F1FF3F4FD01B0456
:20CD70001B0C9D4206D0521E01F1040100F10100F0D144E08446BCF1050F40DA7A58224BA5
:20CD90003046C2F30344401F17D01E49401E0FD0001F0BD0801E07D0C01E0AD00F381ABFE0
:20CDB000191C6031091D04E0091F02E0083900E00C390868C0F3834003E019460868C0F3D8
:20CDD00003200F2806D0A04217D922F4702242EA004210E0761F0AD0761F08D0761F06D0F4
:20CDF0000F3E1CBF22F4702242F4802203D122F4002242F4E02247F82C200020F8BD0120B6
:20CE1000F8BDC04604110050201300502C4870B50568B5F1FF3F08BF00250AF0B9FB0128B2
:20CE30004DD108F0ABF9142849DB26482649002601230660254A0B60254C136020680028CD
:20CE5000FCD1264A131D2349186820F00300014321480068C0080CD2106810F0030F0AD037
:20CE700041F003001860106800F003000328FAD101E041F001011A481960006820B119480C
:20CE900000682846F5F7ECFA174818490660184D0A686FF35B4245EA020008601549086877
:20CEB000C0F30130012806D10A681348104040F400320A60086020680028FCD170BDFEE79A
:20CED0001C130050840460425C600C40082204430C00684204000020B03F00500040034084
:20CEF00080012843000120438C210840482003400000390104000940FFFFFCFC2DE9F84364
:20CF10009946904604460E1C44BF0020011C68D40BF0C9FA054631468022204608F018FCC8
:20CF3000071C04D097F82F0030F07F0003D128460BF08CFB53E097F82F0010F00F0F46D1A3
:20CF500000200A2107F1180640EA090941EA080896E8030008EA000019EA010608BF00287D
:20CF700020D028460BF072FB07F1180003C804F1700604F1700508EA000809EA010986E8C6
:20CF9000000395E80C0007F1180696E8030007F118059943904385E80300703494E8030007
:20CFB000BDE8F88310487968884202D07968A166786004F1600080E8000328460BF046FB42
:20CFD00004F140004FF0FF310AF0C5FFE5E728460BF03CFB97F82F0010F00F0FFAD10220AA
:20CFF0000021BDE8F883C046ED3901002DE9F04F09AF3C897D6816464FF0000A0246002EE1
:20D01000ADF1440DA04610933C888DF83CA05CD0304810F80690042E03DAA8EB0900C84668
:20D030004519F868A4EB080407AB0827A4B2C01D10F801C97F1E03F801CBF9D1080E264FE8
:20D0500003F8010B080C03F8010B080A03F8010B386C03F8011B9DF83C101E704369F86B4C
:20D0700098478346BBF1FF3F2AD0042E04DA03208DF80000022002E002208DF800008DF82C
:20D09000140002959DF83C608DF8026001218DF80110386C8DF8039007ABADF816800BADA4
:20D0B000ADF81840026A0193109E04956946F86B039690478346386C8269F86B0FA9904750
:20D0D000BBF1000F18BFE42000D1504611B0BDE8F08FC046400000000802002038482DE958
:20D0F000F0410068C06B8047044606F0A1FA354F06463846DFF8D08001788F0006FB0745F0
:20D110002E4C04F160021178022363F30301117041464A78E565083292B207FB025704F144
:20D1300044052A7863F303022A7004F17C0327641A780025074665F303021A700AF0AEFC71
:20D1500028B17868216C884238BF012300D32B4698F80110387823B91C2004F0E3FCBDE86F
:20D17000F08104F160031A782F4665F303021A7004F14403E7651A7808318FB222F00F0231
:20D1900042F003021A70820004F1480302FB07F121641A78012767F3C3021A7004F14803DF
:20D1B0001A7867F304121A707043A4F856504FF4FA51216509F07CFDBDE8F081701500209D
:20D1D00078180020B01B0020181D002039482549C0F870122449C0F874122449C0F87812CC
:20D1F0002349C0F87C122349C0F88012304AC0F8E421C0F8F4212049C0F884121F49C0F8DC
:20D2100088121F49C0F88C121E49C0F890121E49C0F894121D49C0F898121D49C0F89C128C
:20D230001C49C0F8A0121C49C0F8A4121B49C0F898101B49C0F89C101A49C0F8A0101A4982
:20D25000C0F8A4101949C0F8A810002180F8041280F80712022180F8E811012180F8F81109
:20D270007047C046FD81000015400100694D010041440100A93101006D5B0100616E01005C
:20D29000AD4D0100913901004D530100F57A01002D19010015580100557B0100A1800100FF
:20D2B00029770100890D01000D320100D7840100E18001000802002070B5394D064695F87A
:20D2D000AA02ADF1180D80B995F8EC0282280CD031480068314C016C2068884709F04AFD33
:20D2F00095F8EC12D5F8C022505495F8EC02822814BF401C002005F52A7485F8EC0295F83C
:20D31000EC0204EBE00292F82C00411082F82C10400807D295F8EC02401C85F8EC02C0B2AC
:20D330008128ECDB95F8EC0281282EDA04F14401E120F9F70BFB02204FF6FF738DF81000A2
:20D3500095F8AA12ADF8083031F0020019D0012919BF0720832108208021002249340092C4
:20D3700002AA0194FAF72AFCDB2807D0E52805D0F32803D0DF2818BFE8280BD185F8A902A9
:20D3900003E0304604F006FD04E02A203070304605F092FB06B070BD78180020A81A0020F2
:20D3B000080200202DE9F04FDFF8DCA000240646ADF13C0D4FF0010B2546A0460D93189848
:20D3D0000C91DFF8C0900E9047E016F8020FA41CA4B2401E1CD0401E09D0401E04D0401E6E
:20D3F00035D1022F33D135E0032F30D132E0072F2DD1B1787078042240EA0120AAF88401AB
:20D41000F11C0AF5C4700AF0E5FB8AF899B121E0052F1CD1CDF80880B11C02A803220AF011
:20D43000D9FB0C9803A9FCF7A7FA9DF82A0088B1029BD9F80020039340F00200049200F050
:20D45000F7008DF82A0003A805F028FA02E07819801C85B2E419F619A4B23046694608F08F
:20D47000B9FE071CB1D1022C03DC44466720254600E040460D990C800E990FB00D80BDE887
:20D49000F08FC0464C110020BC0F00202DE9F84F0746344800788B4620B93846F7F746FE97
:20D4B000BDE8F88F304DE989002405E03868E989641CA4B280193860A14201DC0AF0D3FF93
:20D4D00038465946F7F732FE95F8F411002847D19BF80080D7F800A0002940D023480168A0
:20D4F000C88AC2083BD280094FF0000602D3087D152834D009F018FEAB898646002B06BF8B
:20D51000B5F80EC06346B5F80EC05B1EBCF1000F9BB224D0D5F810906146184600EB800009
:20D5300048440278904506D003B963465B1E491E9BB2F2D113E0D0F8011070460AF095FFC5
:20D5500042F21073642101FB0A018B4205D942F242706423401AB0FBF3F6002EA6D10020AD
:20D57000BDE8F88FB0110020BC0F00200C02002036492DE9F04F0822ADF1140D039001A87C
:20D590000AF028FB324C6068804780466946722009F09EFA2B4EB0884FF6FF7590B10746C1
:20D5B000002400990398091D0AF050F9012808D000987F1E04F1010400F118000090F0D110
:20D5D00000E025462249896840468847B0884FF6FF71A94218BF281C30D183461A4800F12F
:20D5F00018010F88002F08BF002425D081461849D9F81450D1F8048000263446AA4650468C
:20D6100001A9082209F0B4FC40B17F1E06F108060AF1080A04F10104F1D10DE0039970190F
:20D6300008220AF0D7FAC047B9F81A10084F491CA9F81A10B96888475C44A0B205B0BDE840
:20D65000F08FC0468C1C0020BC0F00204C040000D0170020F8B50AF0CDFD05F001FB0AF0CF
:20D67000E1FD054605F00C000C2853D0E80826D209F0B2F92A4E376804460120014609F0CB
:20D6900012FF31686143884219D22649F020B0FBF7F0241A887C18B1C868A04238BF041C32
:20D6B000214D214628460AF0CDFF28460AF0C6FF0120FAF761F8284609F0C6FE2CE0280951
:20D6D00028D21A480AF061FD0428FAD0184A690905D220B11168104621F0010103E01046F9
:20D6F000016841F001010160983210684FF0805540F003001060D5F8B801816920208847A5
:20D710000C4CD5F8B8712068B86B804701202060206801E00AF097FE0AF072FDF8BDC0467C
:20D73000E80B0000EC0A000064130020004003408C2108402C2009402DE9FE4F1E469246AD
:20D75000834600910AF095FE334A6FF001080027012592F89091019005FA07F419EA040F54
:20D770004CD0F8B20AF04EFA002847D0837A002B44D192F8901184F0FF040C4082F89041DC
:20D790008572477292F89211C0F800B0491C82F89211009B03721E4C4460017A07460129A2
:20D7B00013D002290FD190F909301A4D4DF2FC014FF4A060314000EB032000F47060084335
:20D7D00045EA00010BE0002109E097F909100A257E6107F110003D82491D81700146F9609F
:20D7F000BAF1000F18BFC7F804A0906808B93868906005F08DFE97F9098002E07F1C032F94
:20D81000AAD301980AF02AFF4046BDE8FE8FC046CB7B000001200306F82300202DE9F0410F
:20D8300017460D460AF025FE334C8046A078832635B16D1E56D06D1E4ED0681E0AD007E07E
:20D85000A06B002808BF80264FD0A06B808D4BE003264AE0386800215022054604F096FB60
:20D87000022704F5887C04F59072A5F110015CF8040B41F8100F53684B60107A087352F860
:20D890000C0B7F1E18448860F1D1A06B002808BF02200ED0A06BC068A76B286297F82E0038
:20D8B000A36B85F82C00586AA26B6862906AA8620320676BCFB1052817DAFA6801016A5053
:20D8D00097F82E206C1822737A6A6260BA6AA2603F68401C40B2EDE70021022808BF012179
:20D8F000397002E094F89001388040460AF0B6FE3046BDE8F081C046F823002038B5304C4E
:20D910000D46A8084AD2E80858D30AF02FFAE06004F134000AF0BFFDA16868B1C0680546E6
:20D9300041B18D4206D0296AC90803D3C3690421002298472946A160486822490078086049
:20D95000022008F083FD112001F046FF0120A070A168087C08B1E07818B90E2001F03CFFBC
:20D97000A1684968886808B9C86810B116480AF0B7FB1649164D072000240860154B2968CB
:20D9900015482C606A686C602A6843EA020129600AF024FC19200AF06EFD38BDFDF712FCF6
:20D9B000204644300AF077FD10B905F0B1FD38BD204645F00201A8300AF079FD38BDC046CD
:20D9D000F8230020D02108405100070600000460141004400A000040419E00002DE9F84F13
:20D9F000344C054660688846804783463248A16800F178021768894627B95846884700207D
:20DA1000BDE8F88F002682463446BC4240D0787E30F07F0038D079682B7A4878B446CA1C91
:20DA3000C0F38100834219D1022806D0032815D1491D284609F00AFF0FE0D378917801EBDD
:20DA500003212B883046994207D111785278A8EB0101B1EB022F08BF01208446BCF1000F93
:20DA700012D044B1207D012812D16168087840F0100008700CE03C46607E40F010006076B3
:20DA9000207E40F08000207657F80C7C002FBED149465846884754B19AF8FC0220B1DAF8C9
:20DAB000100308B1804701E000F0A8FC01263046BDE8F88FD0170020080200202DE9F0430B
:20DAD0002A4A2B491778ADF1140D002F44D02F48077837F07F073FD1264FC88A002407F127
:20DAF0007C06BC67401C244D244BC8823078A04668F303003070012028701978012901D01A
:20DB1000F7F7D6FD09F020FC214D281D006880470222029481468DF80D80194E8DF80C2092
:20DB3000306A1C49046D43468DE80C00154B0868703702AA3946A04717490028A1F1200197
:20DB5000088005D4104991F90000F760401C0870A9684846884706E0088B401C0883002058
:20DB7000107009F0F5FD05B0BDE8F083552E00208C1B002070150020731C00203D1D002025
:20DB900058180020892001007A1C0020572E0020D0170020A81A0020EC1A00202DE9F04784
:20DBB0000D4606465FFA85FA280824BF2E4845402E494FEA8A03C85885EA00023240C2F3DB
:20DBD00000672B4A06EA0504B043224006F4E0240243B4F5E02F01D1500E14D306F4E020FF
:20DBF000074310D002F4E027B7F5A02707D0B7F5803704BF22F4003242F4A02203E022F445
:20DC1000803242F4C022DFF86C80CA5008F1D00739680122002002FA0AF40C4218BF101C4E
:20DC30005FEA000906D1F00D04D34146C5F3805001F80A00300E0BD30AF01BFC290E34BF6E
:20DC50000021211C3A68A243114339600AF006FDB9F1000F06D0F00D04D34046C5F3805173
:20DC700000F80A10BDE8F087006000A000100840007F077F002002402DE9F84F0D460746AA
:20DC900028684FEA90092F48484502D3287A022802D00320BDE8F88F0AF0EBFBDFF8A8806D
:20DCB0008346D8F8140108F5887AB84214BF00240124A00080F004005AF8006027B107F1FB
:20DCD0009C000AF095F968B956B106F19C000AF08FF938B93046022100F03AF8064602E0F9
:20DCF000022600E00026194801686EB998F8440140F0020088F84401C8F8387158460AF028
:20DD1000ADFC0020BDE8F88F2A68A00000EBC400504402612A7A9C37B9FBF1F10276384623
:20DD300009F0E6FF58460AF099FC012E07D1D8F83C01B8F9401198F842210AF019FB83200E
:20DD5000BDE8F88F40420F00F8230020442E0020344A2DE9F0418846916B04460AF090F9CD
:20DD7000002750B1906B90F82E0041460AF0E1F83E46031C18BF976B01E03B460126506BA0
:20DD900000B3556B1CE0204629460AF079F928B195F82F0040F0080085F82F002D682AE0AB
:20DDB000204629460AF06CF948B195F82E0041460AF0BFF8002608B10BB92F4603462D683D
:20DDD000002DEDD1002E18BF022028D1002B14BF002F002023D0906B3D46A8420BD1916BA8
:20DDF00020460AF04DF930B1906B2F30017841F008010170556B002DC5D1C2F8384192F8CE
:20DE1000440140F0010082F84401BE8DC2F83C4103F00103A2F84061012082F84231BDE856
:20DE3000F081C046F82300207CB5344C054694F8F5030F285DD0697E6078890959D2297E19
:20DE5000002841F00201297639D069684A1C1078801010F0030F32D000F0030002280ED14F
:20DE7000B4F808344FF6FE70984208DD56791179002001EB0621994208BF012004E004F20F
:20DE9000FE30491D09F0E2FCC8B9687E696840F0010068764A78C2F38102022A2DD1491D36
:20DEB0004A7809784FF6FF7601EB02218E4224D1297E00F0EF0041F0200129761CE0687E28
:20DED00040F00300687694F85F01B0B994F82B048DF80000FF238DF8033094F83A648DF803
:20DEF000016094F83B548DF8025068460AF03CFA7CBD687E40F0010068767CBD0802002050
:20DF100070B5064600210B22ADF1280D0DF119000AF0E1FA2E4D3078C01E15D0801E04D01B
:20DF3000143811D0801F01282FD801208DF8180006F18F0103A80AF080FA032495F8FC02BF
:20DF50008DF8144070B113E000208DF8180006F18F0103A80AF071FA032495F8FC028DF839
:20DF7000144028B9B5F812040224ADF8020005E00DF1020005F22C410AF05FFA8DF80A4061
:20DF9000B5F80E04ADF8160017E002208DF8180006F1320103A809F07FFF0DF1020006F1FE
:20DFB000280109F079FF0B48008806F11C01ADF816000DF119000AF03DFA0B208DF8000015
:20DFD00075788DF80150684600F0B0F90AB070BD08020020160600202DE9F04F2C4C207875
:20DFF000ADF12C0D012850D101200AF059F82F4E303E306A274F436CF868022108AA9847C6
:20E010009DF82000A046002836D1DFF88CA0DAF8040080470024B946022509901F480594A3
:20E0300004A90490D9F80C008DF81850FFF724FE02948DF80C501A498DF80D40306A4C809B
:20E05000076D88F800502B468DE81800154BD9F80C0002AA8B46B84700280BD4124991F9C9
:20E0700000005746401C08700998B968C6F80CB088470AE00AF0D2F998F80000012804D1D7
:20E09000002088F8000009F075FD0BB0BDE8F08F3E1D00209C1A0020D017002000093D00E8
:20E0B00080150020FD4601007A1C0020881800202DE9F043DFF8BC808946054617464FF0CF
:20E0D000FF31ADF1140D404609F045FF2A4C04EBC504666825680AF0CCF921680968002913
:20E0F0000BD42968002905DCB9F1000F09D04FF0FF3108E0B9F1000F03D00AF0AFFA00245A
:20E1100030E02968491C29600AF0A8FA2868022828DA1FB903A80AF01FF903AF3868686059
:20E13000B768684609F074FF307B144A00946B463946019005F12C0007F0A0F905F164002C
:20E15000002108F041FB05F14800012108F03CFB706801F041FB0A4A05F1180023460421D6
:20E1700008F0F2FC40460AF09AF9204605B0BDE8F083C046D82D0020740B0000AD6D01009E
:20E190009983010080B50288A2F602073FB143F20502BF1A14BF002090F8240000E0C07B33
:20E1B0002C4AD2F88832401F0B6048D0401E3CD0001F30D0801E24D0C01E18D00F380CD06F
:20E1D000D2F890024860D2F894028860D2F8BC0220F0784040F080503AE050694860D06ADE
:20E1F0008860506C20F0784040F0704030E010694860906A8860106C20F0784040F0F0400C
:20E2100026E0D0684860506A8860D06B20F0784040F0C0401CE090684860106A8860906B3A
:20E2300020F0784040F0A04012E050684860D0698860506B20F0784040F0405008E01068E0
:20E25000486090698860106B20F0784040F02050C86080BDC41000502DE9F843324D0120C8
:20E27000002428702A48DFF8AC80DFF8B0900470294800F172010F8814EA03064FF002011D
:20E2900001EA020108BF00290FD120464FF0E04710401F4008BF002827D0424692F900003C
:20E2B000401E107009F07EFC1FE0424692F90010491E117067B901F0F1FB46464846047068
:20E2D00096F90000E8B196F90000002817DD1BE0B7F5505F07D113481149006800F5C070EB
:20E2F000086000F0EFFC09F021FC48464246047092F9000028B192F90000002804DC0AF03A
:20E310008DF82046F7F7D4F92C70BDE8F883C046741C00207A1C002070150020731C0020CB
:20E33000701800200C0100213D1D002070B50646304930780D5C401F1CD0083851D0401F77
:20E350004FD0284608F002FE041C0DD130780C2808D1706830B1301D06F086FD284608F090
:20E37000F5FD0446002C43D02A462046314609F031FC37E0B07810BB307C317A2D184C109D
:20E39000480000F00E002D1804F038002D182435E8B208F0DBFD041C2AD03146182209F0EA
:20E3B00019FC04F1180060607168242209F012FC6068243060617169327C0E46D6E70128A6
:20E3D00016D12435E8B208F0C1FD041C10D03146182209F0FFFB04F118006060716824220D
:20E3F000EBE7344624B104480078214605F0B0F970BDC0464C0B0000801C0020F8B5324DB1
:20E410006868804706462F4CA9686068002855D1E0698047A76F40F01000002F4DD0002293
:20E43000797E0140884205D03A4657F80C7C002FF6D142E004F17800394607F001FA002F79
:20E450003BD06760787E30F07F0005D194F88300401E84F8830004E094F88200401E84F837
:20E470008200A9683046884761680889C98A05F07FF8A4F8800094F83B0407F0C1FD0546B4
:20E490006068C18A090A08D3C07E05F0F9FF606890F91C0009F0BAFC6068E97B012903D0FB
:20E4B00002290DD1052005E0007E401080F0010000F00100FBF7F4FBF8BDA968304688471D
:20E4D000F8BDC04608020020D0170020F0B5324E044696F8AA02ADF13C0D022807D0012886
:20E4F00005D005281CBFE82086F8A9024CD196F8F00200284DD1002109A8182286F8A912D6
:20E5100009F0E9FFCDF828D009A8214601F0ACF896F8BE0296F8E812814222DDD6F8C05228
:20E5300070B10746BDF80A006989884204D12846694608F03BFAA0B97F1E05F12405F1D1EC
:20E5500096F8BE12D6F8C0728800242200EB41106946C01909F03EFB96F8BE02401C86F861
:20E57000BE0296F8EA0328B19DF8340010B996F8E80228B909A8FFF7D9FE96F8E80240B1A5
:20E5900096F8BE12884204D12A202070204604F093FA0FB0F0BDC046080200202DE9FE4FAE
:20E5B0008046314DDFF8BC9095F8FC02174609EB4806583634880191C0B1D5F81413A9B11F
:20E5D00009EB880BDBF8CC0000F0FF0088478246D5F81413DBF8CC0000F47F008847504416
:20E5F00083B21BB13088C018001D84B295F8200401280AD1387A40B148447B7A067919F8BE
:20E6100003000019401D84B200E00026A01980B208F09CFC95F800A0071C19D000212246F8
:20E6300009F059FF002587F8008008EB090138197D704A7D786007F1840001993E8109F0AD
:20E65000C9FA5046394605F083F82846BDE8FE8F8DF8008068461A2102F0BCFC1A20BDE84B
:20E67000FE8FC0463C000000080200202DE9FF412E482D4F00683E78C06B80477968401AFE
:20E69000B100B0FBF1F4B868FF680025A8464146BC4271EB080101DAB84206D829464246FB
:20E6B00084428A413CDA074600E0294638463246F317001BA94109F0BDFA272704464FF477
:20E6D0007A7200230D46ADF802700820ADF800002046F9F763F9019015480168684688475E
:20E6F000029843464FF0000100F6FC02A41A9D416042A94111DA0F48026829462046F9F71A
:20E710004DF90D4604464FF000016042A94104DA204606F0F3FC002000E001200649087029
:20E730000090BDE8FF81C046B01B002078180020F4170020881A0020562E00202DE9F84F85
:20E750002E4C012683461D4690468946C4F87C670320C4F880670AAFC4F88407D4F88C0773
:20E7700010F0030FFAD1387A58B14FF0805ADAF8B001016A27208847DAF8B00101692720A0
:20E7900088470220C4F8FC063868C4F80804304609F02FFED4F808040008F8D2D4F88C07AD
:20E7B000800F28BF301C26D22868C4F83C056868C4F84005A868C4F84405E8681049C4F8B7
:20E7D00048053879002814BF081D081CC4F84C05C4F850850020C4F85405C4F858050949A9
:20E7F0000E60C4F800B0C4F80880C1F80064C4F82090C4F82880BDE8F88FC0460440024046
:20E81000280000200000484203B42DE9F047304C4FF0000908AF84F801903968ADF1100D2E
:20E8300002A80160B988818002A803C89A46164608F0C6F9A046051C14D04C4686B12846F1
:20E850006946012207F05AFD1AF804009DF80010884205D1641C6D1CE4B2ADB2A642EEDC7D
:20E87000A6422ED0B8F80200F61C4FF6FC7440F6F8753440001985420ADA09F039FCFCF72D
:20E8900043FDB8F8020000198542B8BF012019DB396802A8BE88016002AD868095E80300E3
:20E8B0002246534601F0C8FE98F80100B8F80210002818BF814604D164180834A0B2A8F8F8
:20E8D0000200484604B0BDE8F04702B07047C046A01C0020F0B506460F4600251446ADF15A
:20E8F000240D8B200DF10E010095FCF7CDF98A2001A9FCF7C9F9707A00282ED1387AA0B9AC
:20E91000BDF80E104FF6FE70884205DCBDF80E10884220D101A90DE020489DF80E7004888A
:20E93000BDF80E008DF812700CE0022807D0032811D1394604A809F080FD09240BE038888A
:20E950008DF812008DF81040211200128DF8111005248DF81300284611E002280CBF052412
:20E970000924012818BF311C04D1892007A9FCF78BF907A9224604A809F02CF9B07A0DEB64
:20E990000401C8736A4604A8214603F0DDFC002814BF281C009809B0F0BDC0461606002019
:20E9B0002DE9F0410120294E294930706FF0010008702C480068C06B8047264C054621785A
:20E9D0006068A2688B002F1AB7FBF3F058433F1A8800214902FB03F8B1FBF0F0904201D2DD
:20E9F00009F01CFDED1B1D48656008EB0501FDF725FD1D4C303C206BE76AA16A404207F07F
:20EA100033FB002F08BF216B08D0216B78688142DCBF401A78603F68002FF7D1606B88422F
:20EA300002D0206305F018FB05F0EEF90C4C606880470546FFF71AFEA1682846884708F00F
:20EA5000A3FE00203070BDE8F081C0463D1D0020701C0020B01B0020FFF6C2FFB1E90000C8
:20EA7000D017002078180020380200202DE9F84316460C46074609F0FCFC2D4D8146A878D7
:20EA90004FF08308002C4AD0641E41D0641E3CD0641E37D0641E26D0641E12D0641E2ED14F
:20EAB000F0B905F1340009F0F6FCC8B9316805F1A80009F000FD316805F1DC0009F0FBFC7F
:20EAD0002FE068B905F1340009F0E5FC40B93168192009F0D6FC31681A2009F0D2FC20E0C2
:20EAF0004FF000081DE0306828B1012807D1802007F0F8F815E0802008F08CFE11E04FF082
:20EB100003080EE03068A8610BE03088788208E00120FE68787406F16000F86001E030682B
:20EB30003860484609F09AFD4046BDE8F883C046F82300202DE9FC4707460E1C14BF4FF046
:20EB500000084FF0E808002F4FD0B8F1000F4ED17868401E78603F210170BD6D002D0CBF40
:20EB7000802000207968DFF88C900224083E491E7960DFF884A008703889A7F85440801C42
:20EB9000388116F8080FFF282CD02A2828D1706830B3D9F814138847054678689AF80020BA
:20EBB000401B7860716831B9D9F818C33A460023E04750B10CE0D9F818C3786871688DF802
:20EBD00000206B463A46E04710B9EB20BDE8FC873889B7F85430401938815819A7F8540047
:20EBF000641ECED17868386501E04FF0E8084046BDE8FC87080200201A1D00202DE9F041E1
:20EC1000054609F0E5F8297E2B48090902D2297D012900D0401CDFF8A880077846467068E5
:20EC30008047264C04F178010B68002B08BF0D600CD07F1E0026FFB202E07F1E1346FFB272
:20EC500053F80C2C22B92FB143F80C5C012601E0002FF2D1D8F8081088472EB3A1692846B9
:20EC70008847E88AA168C0081AD2D8F80400804794F88310491C84F88310D8F808108847A1
:20EC900094F8FC0210B1D4F8100330B9E88A400A0FD2FFF7B3FBBDE8F0818047BDE8F0811D
:20ECB00028468847BDE8F081F1206870284602F087FBBDE8F081C0468C1C00200802002018
:20ECD000D01700202DE9F0412E482F4D08382B4CD0F80080281D0668201D07680FB909F0C5
:20ECF0009DFB404609F07EF8F860404608F006FD3882B04780461D48A9680278832A31D188
:20ED10001B4EF7782FB386210170082008F02CFB708B1949401C7083164894F83B248162F2
:20ED30001749812A09DB0978842A07DA40F6485292FBF1F101F6B83106E0097840F648526E
:20ED500092FBF1F101F2A321203008F02BFDA96808E08522027040468847002002F0E2FEB4
:20ED7000BDE8F08140468847BDE8F081572E00208C1B0020CC1A0020954701000802002089
:20ED9000B01B002078180020D01700202DE9B841804607F0C9FFC01DC51098F823000028A0
:20EDB0004AD198F87E4007F0BFFFA04244DD264A5368E1100846C91891F8701004F00704CF
:20EDD0002141CFB207E0401CC0B2C118C40091F8707088F87E4047B9691E8142F3DC506876
:20EDF000002188F87E10417029E098F97E10C0000830884226DD401A79080BD298F87E1060
:20EE1000401E4FEA670701F1010188F87E10F3D1BDE8B88198F87E000C49087098F87E0050
:20EE300088F8810098F87E00401C88F87E000320FAF736FFBDE8B881002088F87E000720ED
:20EE500005F038F8BDE8B881080200201B1D0020F8B5234E0027E82086F85C70032186F8E4
:20EE70005D7008F04FFD5220012108F033FD1D4D482205F1840406F16400214601F066FD4D
:20EE90001948C5F88800403C74611848C5F890001748C5F8B4001748C5F8A8001648C5F80F
:20EEB0008C001648184CC5F8940015481749C5F89C00144847F23052C5F8A40004F1980088
:20EED00005F086FD3946A061522008F003FD10494EF6602204F1BC0005F07AFDE061F8BD8E
:20EEF0002417002058160020C9BE0000355B01007D26010095F300001D65010069040100E4
:20EF100099110100191F01006C140020ED770100D97301002DE9F04FDFF898A001270446D5
:20EF3000DFF894908AF8007099F80000ADF1140D012802D03846F6F7BBFB204605F0B4FD5C
:20EF5000DFF87880D8F80400804704908DF80C70002402941A498DF80D401B4D4C80286AED
:20EF7000184A066D02238DE81800184B10688B4602AAB047D8F80810E88000280AD4144AF7
:20EF900092F90000401C10700498C5F80CB088473C460AE05046047004988847484600782F
:20EFB000012802D02046F6F783FB204605B0BDE8F08FC046741C00203D1D0020D0170020FF
:20EFD00090150020A81A002058180020B14601007A1C002010F47C1F7CB524D110F00F0F59
:20EFF00024D006460024012505EA0600AE436D00401E13D0401E0FD0801E0BD0001F0FD12E
:20F0100042F20500694605F0D9FA9DF8000038B1093404E0241D02E0E41D00E0641DA4B2B6
:20F03000002EE1D133E010F00F0F01D000207CBD064602244FF4803505EA0600AE436D00C8
:20F05000B0F5803018D0B0F5803013D0B0F500300ED0B0F5802009D0B0F5002004D0B0F51C
:20F0700080100FD1072008E0062006E0052004E0042002E0022000E0012000F0E1F90019E0
:20F09000801C84B2002ED7D1022CD8BF002420467CBD70472DE9FF472A4C89468246211DD2
:20F0B0000888401C088028490822684608F092FD208B4FF6FF7880B16569074600262846B5
:20F0D0005146082207F054FF30B17F1E05F1080506F10106F3D100E0B0464FF6FF754545B9
:20F0F00004D1207A401C20722E4627E0404602A901F026FF0646B542F6D09DF80800012812
:20F1100007D0A16D700000EB86004018A0F8049005E0616D06EB46104018A0F81F90606933
:20F130006946082200EBC80008F054FD074D68688047618B491E6183A968884730460090E2
:20F15000BDE8FF87BC0F00204C040000D017002030B50546ADF12C0D08F062FE002818BFD4
:20F17000FC2051D168462946112208F033FDAC7C697D8DF81240687C8DF81510EB7C8DF86A
:20F1900011002A7D8DF81330AC7D8DF81420002104B101212C7E8DF8161095F825208DF859
:20F1B0001840E87D8DF8252095F824308DF81700EC8C8DF8243005F119010B220DF1190096
:20F1D000ADF8264008F006FD687C002448B9812007F082FD0A9080B1FF21812209F07BF9FE
:20F1F0000DE09DF815000A9448B1810001EB401188B207F071FD0A9008B91A2403E00720D1
:20F21000694603F08FFC20460BB030BD2DE9B043044609F02EF981462748221892F8EF1037
:20F23000491ECFB2002F82F8EF703FD1254901EB84014A880C78904634F07F0718D1E10936
:20F250000FD24FF0805000F5DC75D0F8B8018169104688472868416B404688470228F9D153
:20F270001EE000EB8800D0F804110020884717E04FF08055D5F8B801016A10468847D5F853
:20F29000B801816A40468847D5F8B801016B404688470A4901200860094908688008FCD329
:20F2B00004F03F00132801DAFFF7B0FF484609F0D5F90020BDE8B0835813002028200860C8
:20F2D00028200840300900002DE9F0478A46804602F00107C2F3400609F0CBF8264C032527
:20F2F0008146BAF1FF3F08D1A16B404608F0C8FE00280CBF616BA16B05E051464046002236
:20F3100006F026FA014600292FD091F82F0030F07F0029D0A06B88420FD04046324600F066
:20F330006BFD08B3A07801281CD004281AD004F1A800022109F0BBF814E091F82F200120FE
:20F35000002F00FA07F040EA020081F82F0014BF0A480B4807F0E4FB26B1616B40463246BA
:20F3700000F04AFD832500E00425484609F076F92846BDE8F087C046F823002001000204CD
:20F390000100010470B505462B4C2878ADF1200DEB2829D040B3E92806D0E12843D14FF4BF
:20F3B000FA7007F06BF83EE004F15E010878401C087094F85A00032818BF042803D14FF488
:20F3D000FA7007F05BF894F85E00032809D094F85A00022827D104F10A00102108F056F9FC
:20F3F00021E005F06BFF1EE094F85A00022817D104AE6946304605F07BFD5220002108F0D8
:20F4100069FA606920B1026812B1304669469047042003F0C5FD04F10A00102108F036F986
:20F43000002084F85E0005488830016809B12846884708B070BDC0462417002024170020BC
:20F4500010B5401EADF1380D28D0401E09D0801E4FD0401E43D0401E3FD0401E3BD0002043
:20F4700048E001A800F008FF04460CA942F2090005F0A4F89DF83000002808BF002203D03E
:20F49000022007F048F9024601209DF83010009001AB204605F04FFB0A3028E001A800F008
:20F4B000EBFE04460CA942F2080005F087F89DF83000002808BF002203D0012007F02BF9BF
:20F4D000024600209DF83010009001AB204605F032FB001D0BE020200CE002200AE042F2A7
:20F4F000130004A905F06AF804A808F0F6FF80B200E004200EB010BD2DE9F84F1C469146F5
:20F510008A46054608F0B5FF834607F08FFC6FF001080AAF061C40D005F1780008F09FFF72
:20F530002248C6F808A00838B0F9481086F82E90491C6FF31F31A0F848107460B0F8481093
:20F55000B1851949F56097E818002022343006F1100722401940002406F1180387E80600FD
:20F57000214686F82F40224683E806006A46314605F048FB88B196F82F009DF8007040F0C4
:20F59000800086F82F00B08D85F8C240A5F8C0000FB108F08BFBB6F92C80584609F05EF88F
:20F5B0004046BDE8F88FC046FDEFFF9F00240020F8B52B4C04F13405284608F06CFF074645
:20F5D000012004F0A1FCA06B002848D1002F41D0A068F96888423AD1684604F0E9FC38B12F
:20F5F000009828B1206C18B9082006F07BFBF8BD082008F00FF907F1100003C81949C6437E
:20F6100001F108031E601A681042FBD10C310A6807F110061043086096E80C00181C07F191
:20F630001006C04341F80C0C96E80C0051F8082C181C104341F8080CB86807F071FA284685
:20F6500008F0D8F9A063002004F05EFCF8BD4FF4806100E0022104F1A80008F028FFF8BD13
:20F67000F823002008100440F8B505460E460520287096F849006968E870F06B4861686806
:20F6900006F1280108F008FCB6F842006968488196F84600696848746868002404761F487E
:20F6B00069680078C873686806F11C01193008F0C1FE307C69688873726812F8010B696899
:20F6D000888112F8013B6968888940EA0320888117786968F8110874204617F0070118BF62
:20F6F000012001EB410109188918491C11F8010B287200F00702E960401000F0380000EB30
:20F71000420040187268318968615318834239BF2C72211C801A091A2974F8BD4206002068
:20F7300038B504F0EDFA02F01FFD2348007820B1244808380168012088472348234D0078D7
:20F7500020B9281D224B0468187808B108F066FEA047A9681F4A194D1378022B20D1012369
:20F77000174C13706378022B12BF032B832313708847617831F0010008D0042906D0052990
:20F7900007D10020207108F0C3FC01E000F004FF6178022918BF032903D103F0CDFB00E0CF
:20F7B000884795F8FC0228B1D5F8100310B1102008F08EFC38BDC046040500200802002065
:20F7D0008C1B002070180020532E0020D0170020552E0020572E0020F8B5064608F049FE82
:20F7F000264D0746711991F8EF00421C002881F8EF203ED1224C04EB8604267806F03F0060
:20F81000132801DAFFF7E8FF648836F07F0018D1F0090FD24FF0805000F5DC75D0F8B801BB
:20F830004169204688472868416B204688470128F9D11EE005EB8405D5F80411012088472C
:20F8500017E04FF08055D5F8B801C16920468847D5F8B801416A20468847D5F8B801C16A91
:20F8700020468847074901200860074908688008FCD3384608F0F2FE0020F8BD581300208D
:20F890003009000028200860282008402DE9F0412A4C94F89101002844D000260121354605
:20F8B00094F8912101FA05F0104203D16D1C032DF6D337E094F891211020A840104218BFCC
:20F8D0000E1C08F0D6FD94F891211121A9408A4384F8912108F0C2FEE8B208F093F908B33E
:20F8F000877AFFB190F909701349456851F827100168012E884606D0017A022904D1C168DC
:20F91000490B01D302E08D6902F04AF8012E19BF391C4FF000636FF0FE014FF0007340460F
:20F930000022A84794F8910120B104F1DC00002108F0BDFDBDE8F08194300440F8230020BA
:20F950002DE9FE4F294F284D00264FF001094FF0020BB046BC1E14F8020F032819D0022861
:20F9700036D160786968022832D0304608F0EAFC8246404608F07AFC84F801B001908847FE
:20F990000090019A78685FFA8AF106F05BF800981CE0304608F0D6FC8246696860780128C1
:20F9B00005D0404608F062FC84F8019004E0484608F05CFC84F80180009088470190009A30
:20F9D00078685FFA8AF106F03DF80198A9688847761C022EBFDB07F0DFF818B107F12000B4
:20F9F00008F06BFDBDE8FE8FD0170020F0190020F8B50F4601460024381C08BF0124002365
:20FA100002B90123DFF890C0F8B1866AEEB14F6ADFB1C068CC68844208D0DCF810410CF52F
:20FA30008875844214BFEC68AC6800E00024B8086FF05047A0EB9600001B874225DDB0F156
:20FA5000704F01DB002820DD01240AB3576AFFB18E6AEEB1D068C968884208D0DCF81021DC
:20FA70000CF58871824214BFC868886800E00020C0EB97006FF05041A0EB9600814204DDCE
:20FA9000B0F1704F03DB002801DC0020F8BD01231C40E0B2F8BDC046F8230020F8B5274C16
:20FAB000607830F0010705D0042803D0032818BF05283FD104222249224D27790A7095F87C
:20FAD0000C24791CC9B221718A422FDB03282DD004F016F96078042807D195F8FC0220B10B
:20FAF000D5F8481309B102208847A07895F81914421C9142C4BF401CC1B2A1706E6831892D
:20FB1000706801F03FFE70680088000904D395F8FC0208B106F0C2FA6078052803D1207927
:20FB300008F0F6FAF8BD00F037FDF8BDE12001F0F9FFF8BD08F072FCF8BDC0468C1B0020B8
:20FB5000572E00200802002070B52348214D286522484FF08056A865D6F8D801204C036831
:20FB700001210A46ADF1400D20469847D6F8D80142680121204690471A48012606601A48D2
:20FB9000F9F7C2FA05F05AFB284607F04BFF05F118044FF4E13029462060002005F06EFBDD
:20FBB00012493C22082308600021684608F042FDF8344FF46170002307940D4908906A4647
:20FBD000069605F15C0008F031FD08F02BFD10B070BDC046200700203F840100E168010099
:20FBF0000040034004011CE2080A0000B80B0020F931000090B5044600214022ADF1440D4F
:20FC1000684602F0C3F9A0788DF80000E0788DF801009DF8000000BB616811B101A805F084
:20FC3000ABF9217A01F007028DF82820E0689DF82870C1F302118DF8301027B19DF8281008
:20FC50000B9000EB41009DF8307007B10D90207C8DF8380067690F9719E0616811B101A847
:20FC700005F08AF9677A8DF82970A37A8DF82A30207A8DF82800E27A8DF82B20217B8DF86D
:20FC90002C10677B8DF82D70E389ADF82E300348006801696846884711B090BD641C00205D
:20FCB00070B50025ADF1200D07A8ADF81C5008F07FF9254CBDF81C10B4F84000884237D1DF
:20FCD00094F85B00032811D004280DD0022810D104AE6946304605F00BF9606920B1026839
:20FCF00012B1304669469047042000E0032003F057F9206E06F0C2FB5220294607F0EAFDCB
:20FD100008F00CF8044608F009F800EB042408F005F84FF47A7200EB0420B0FBF2F151432C
:20FD3000401A0A3006F0C2FB284606F0D7FB09E0032008F0C5F8052003F032F95220294651
:20FD500007F0C8FD08B070BD24170020F0B5012904460546ADF1140D04D0022941D142F22F
:20FD7000030001E042F20200694604F027FC04B16D1C06F0D9FFC01DC010C0B2002830D040
:20FD900000230646ADF1010C1F4618461CF801EF00224EFA02F101F00101884211D028B996
:20FDB0007F1CBFB25CB102EBC30103E03CB102EBC301491E05F8011B091205F8011B80F0C4
:20FDD0000100521C082AE4DB761E03F10103DDD130B12CB1D800401E05F8010B00122870D2
:20FDF0000FB9002005E004B12770012000EB870080B205B0F0BD70472DE9F047274C814675
:20FE1000606B0F4690460025B8420AD0606B00E0006820B1016811B101688F42F8D1074684
:20FE300008E004F1340606F1100A4846394608F027F9E8B97FB3343410343968484608F0BF
:20FE50001FF988B1396891F82F0040F0040081F82F00086800223860204604F0D3FE6D1C2E
:20FE7000B8F1010F01D016E03F68002FE5D112E097F82F0040F0040087F82F00304607F067
:20FE9000B9FD50463946002204F0BCFE676B6D1CB8F1010FC9D02846BDE8F087F823002045
:20FEB0002DE9F047254C01258246984691460E46C4F87C570320C4F8805708AFC4F884073A
:20FED000D4F88C0710F0030FFAD1387858B14FF08057D7F8B001016A27208847D7F8B00186
:20FEF0000169272088470220C4F8FC06C4F80894284608F07EFAD4F808040008F8D2D4F8E6
:20FF10008C07800F28BF281C15D2B8F1010F14BF08200C20C4F84C051021C4F8501500203E
:20FF3000C4F85405064A1560C4F800A0A160C2F800542662A162BDE8F087C0460440024039
:20FF500000004842FEB54FF0805647688468D6F8D001C16820688847216821488A6B10404E
:20FF7000886340F2F27120681E4D416494F82000295C94F8210040198079084321684863AA
:20FF9000684608F064FAD6F8D001397F05EB810146680B6ABA69797F206805EB810189695A
:20FFB0001943BB7F05EB83052B6B0B430199B0472168C86A40F01000C8622168086B40F05D
:20FFD00001000863A07D0027FF2802D0E07DFF2800D11FB1086B40F440400863FEBDC046F0
:10FFF0000DF8FFFFC4090000F8B5274C06460E2295
:020000040001F9
:200000000D4604F1340000F0A9FC022084F824006888A08307F08AFE074607F087FE00EBC7
:20002000072707F083FEE26A00EB0720B0FBF2F15143401A0A3006F041FA30462946FCF7FD
:200040008DFA207801280BD0687B48B9288869882A1D03F0E5FB011C02D00BA008F0DAF979
:20006000E56807F059F8854203D807F055F8451B03E007F051F8401B451E6420E560B5FB4B
:20008000F0F0A4F87800F8BD41757468204572726F723A20307800C05816002070B5264C14
:2000A0000120002684F85C01244D6670ADF1180D84F85F61281D006884F8616180470246E0
:2000C000A06F68B1417E8B0806D341F001014176017E01F0FD01017650F80C0C0028F1D1B4
:2000E000A96810468847102007F0FAFF082007F0F7FF94F86001D8B9E0258DF80150092013
:200100008DF80000B4F80E348DF80F6094F82B24ADF8023094F83B148DF8042094F83A5428
:200120008DF8061068468DF80550FEF707F901E084F8606106B070BD08020020D017002075
:200140002DE9F041DFF8948006460C4636F07F0014D1002E3DD1224D686880471E4909682B
:2001600031F81620144321F81640A968884741461431086807F030F8BDE8F081042006F0EF
:20018000EDFE071C25D04FF6FF7038807C8008F099F841468C78A7F10C05FF2802D0C96A0B
:2001A00009184C78FF2C06D1384607F0EEFE07F0DBF9BDE8F081304607F00AFB01463A46DD
:2001C000FF20A872204605F005FE10B1384607F0DCFEBDE8F081C046482E00206C1A002020
:2001E000D01700202DE9F04108F04BF9254D214E804605F1E000007848B93446A1680220DA
:2002000088470746102004F059FE6FB31AE008F011F8C0091AD218480068C46817483421CD
:2002200001220023A04788B102F0F6FE34460020A16885F8E000022088470746102004F010
:200240003DFE8FB1A168032088470DE00C4800683221B1FBF0F101B901213035284608F0F8
:2002600002F9284608F001F9404608F0FFF9BDE8F081C046EC0A0000A401001000A00C40FA
:20028000442E002058130020F0B50446E820ADF1240D08A904F09CFC9DF82000694606F0E4
:2002A000BBFF00280CBF00981D480DF121016060E82004F08DFC9DF8210004A906F0ACFF2B
:2002C00058B90599C8200322B1FBF0F0401EB0FBF2F15143401AC0B200E00020207206F002
:2002E0002BFD002167686081072321700D4A61705568BD420CD1157A267AB54208D15589AC
:20030000854205D11078207057786770084604E05B1E02F10C02EBD1012009B0F0BDC0468D
:2003200038C40D00601000202DE9F043254C0746243C606AADF1240D00283ED0002F3CD0B3
:20034000387A002839D004F0EDFC5FEA000834D0062000250323A1468DF808002E46ADF88A
:200360000A30B5F5FA7F28DAD9F82400ADF80C5004AB02AA0469009392E803000A23002201
:20038000A047B0B9387A9DF81810814210D1022804D1BDF810103A88914207D0032807D1B7
:2003A00004A93846082206F0EBFD08B9284606E0761CB04505F10105D3DC4FF0FF3009B09C
:2003C000BDE8F08390140020F0B520480127F84201D004F005FA204D204F214EBD4206D2EC
:2003E00003CD0478A4003459401CA047F6E71D48002800D08047164D164FBD4202D210CDC4
:20040000A047FAE7F0BD03251BE0416808300A1C2A400BD11A1C2A40AB4305D004680430F4
:200420000C600431043BF9D1131C05D0047801300C700131013BF9D1021C2A4001D0A84369
:2004400004300368002BE0D17047C046FFFFFFFF000000000000000030950100909501007C
:20046000EC94010055C5011070B50546244C287800283FD1A07801283CD0281DFFF754FF3D
:20048000B0F1FF3F36D1298AC81333D001F00F010F292FD12046B0F840104FF6FF728A42CC
:2004A00003D0EA898A4205D102E0E989A0F840100121C170A97C80F84210AE88A0F8446064
:2004C000298A01F00F020F2A05D080F85820C1F3031180F8591090F858100F290AD101219B
:2004E00081700848064607F0CBFD012802D1304607F0EDFF7434216809B12846884770BD06
:20050000241700202815002003B426482DE9F041008806AF1646ADF1080D001F84B2082CE2
:2005200039DB3D78201F6946082280B2804605F0EDFEBDF80000C10B19D300F0FF008542DF
:2005400015D17888BDF80210884210D1B888BDF8041088420BD1BDF80600002E18BF40464E
:200560001AD1C0F30E00241A241FA0B214E0BDF8061008466FF30E0048B908460830844232
:2005800002DA07F045FD06E0641A083C00E0241FA4B2082CC6DA002002B0BDE8F04102B0F7
:2005A0007047C046A21C00202DE9D8410020224C8DF8000007F0D3FEA278DFF88080012183
:2005C00091404FF6FF725218024098F8FC02228128B3D8F8342312B342F21A00694690471C
:2005E000144827790678A6B19FB99DF8006086B1D8F8580368B180471149124A09781278DA
:2006000030B1278908314A43B0FBF2F17818208127799DF80010208907FB0100208160785A
:2006200018B9FCF763FDBDE8D881FCF78DFABDE8D881C0464E2E00208C1B0020080200208D
:20064000191D0020B01B002003B426482DE9F041058806AF1446ADF1080D98464FF6FF700C
:20066000ADF800000222ADF802006946ADF8040044F40040ADF80600281986B2304602F0AE
:20068000A5F8BDF80600022269466FF3DF30ADF80600304602F09AF8A1102846CAB24146F7
:2006A00002F094F8387840F44040ADF800007888ADF80200B88802226946ADF804003046DA
:2006C00002F084F8BDF80000022269466FF3DF30ADF80000304602F079F802B0BDE8F041AD
:2006E00002B07047A21C00202DE9F843002A894607464CBF47F6FF75151C002F08BF002019
:2007000033D03888002808BF002403D02A4600F0D3FB0446281B002826DD388828B1291B6D
:20072000484613A204F00EFC2418B868E0B1D7F804802E1BB8F1000F0DD0404607F0A0FB42
:20074000401DB04207DC291B48460AA2434604F0F9FB24182E1B122E06DBBB68291B4846DD
:2007600006A204F0EFFB24182046BDE8F883C0463A2000C0222573222C2000C06C696E6581
:200780002025643A200070471CB5204C04F5DC7006F07EF904F5CE7006F07AF904F5EA70BD
:2007A00006F076F90021882204F5BA7007F09BFE07F0C6FA06F0C0FA84F89A01144984F8FF
:2007C0009B011448086001200DF1010184F8F30142F2040003F0FAFE42F20500694603F02A
:2007E000F5FE0D489DF80110C4F8A80164204143C4F8A0110949C4F8C4119DF8001048431E
:20080000C4F8BC010648C4F8E0011CBDBC0F002068180020AD620100014301003DCC0000B2
:20082000D9830100F8B5044607F02BFE234D064605F5A2710878A04305F588740870206822
:20084000002808BF002706D020689C3007F0D8FB002700B10127606838B19C3007F0D0FB4F
:200860000024384318BF0124274695F8440100BB012F1ED0D5F83801F0B1016A89080BD245
:200880004469304607F0F2FED5F8380100214FF400030A46A04708E0C469304607F0E6FE44
:2008A000D5F8380102210022A0470020C5F83801F8BD304607F0DAFEF8BDC046F823002000
:2008C00010B5244C08BB04F17C021178002004F1440360F303011170197860F3030119707F
:2008E000206494F8481004F1480241F0080184F84810117860F30411F420117004F149017E
:2009000004F066F944F6206019E004F14801087840F00800087094F8480020F0100084F8F3
:20092000480004F0B3FB0A2280B24FF4FA6390FBF2F1514344F62062401A03FB0020064A49
:20094000206592F8FC1219B1D2F85C1301B1884710BDC0467015002008020020002A4AD010
:200960005FEA000C8B071CD1830722D1102A08D370B4103A78C978C0103AFBD270BC1032A5
:2009800038D0042A2CD3082A05D30C2A24BF08C908C008C908C008C908C092072AD0920F00
:2009A00022E00B780370491C401C521E22D08B07F7D1C30714D18307D8D0121F12D308C9FA
:2009C00003801B0C4380001D121FF8D20AE008C903701B0A43701B0A83701B0AC370001DFF
:2009E000121FF4D2121D05D00B780370491C401C521EF9D160467047D0B5244C04F178014B
:200A00000F68002F3FD0002215280AD13B7D0126022B08D0032B06D0052B04D0042B02D0FA
:200A200000E03B7D0026984200D016B17B7E5B0905D23A4657F80C7C002FE5D123E00846C6
:200A4000394604F005FFF88A6760000A03D397F91C0007F0E3F9387D022818BF052802D1C1
:200A6000012006F089FC6068407E30F07F0005D194F88300401E84F8830004E094F8820081
:200A8000401E84F882003846D0BDC04608020020F8B5044642F209000DF1020103F096FD04
:200AA0009DF8020050B19DF80200022833D1A08894F8271001F072FD054606E042F20D001C
:200AC000694603F083FD9DF80050154E301D0768802D01DD07F0AAFCB847124B0E490F4ABC
:200AE0001F780D701FB91778B1684FB904E01778B16837F07F0703D1884701F015F900E09F
:200B000088470020A4F87C5094F82170607017B1102007F0E5FAF8BD9C1A0020572E002093
:200B2000D01700200405002003B42DE9F04307AF97F800807C88BD88ADF1140DB8F1FF0F01
:200B40000FD14FF6FF70A0420BD1A84209D104F0C7F807F0B3F919480421801C0180002066
:200B600027E000264BF6FF790FE06946082205F0CDFBBDF800006946022209EA0000ADF8EA
:200B80000000384601F022FE3E468DF80880ADF80A4002A8ADF80C5003C80122FFF7B4FC07
:200BA000071C03D1002EDAD10A2002E0BE42DCD1022005B0BDE8F04302B07047A01C0020B8
:200BC0002DE9F843234D884606464FF0FF3105F12800814607F0C7F900200CE0FF2909D022
:200BE0002A688A4204D305EB8101D1F898700FB1002627E0401CB8F1000F03D018F8201069
:200C0000FE29EBD10024346074600127B46011E0FF280ED005EB80000B787268C0F89860B6
:200C200007FA03F0104370600A680949304605F039F9641CB8F1000F04D008EB8401087838
:200C4000FE28E5D1484607F032FC3046BDE8F883007FC76744120020B0B5456884682349E2
:200C6000607DA27DADF1180D40F000400090207D0027FF2A41EA000001904FF0020002D0F9
:200C8000E27DFF2A00D13FB1E37DA07D1943039140F0004002900420FE214DF8201005F1EE
:200CA00054006946FFF78CFF2866002808BF381C1AD0617D0F2205F079FD286E217D102215
:200CC00005F074FDA17D3846FF2902D0E27DFF2A00D140B1286E112205F068FD286EE17DB7
:200CE000122205F063FD012006B0B0BD0000C0A030B5044660684078ADF1440DC0091FD36E
:200D00001F4DB4F84200B5F80E14884218D1A878A0B995F8180498B104F1280005F094FFE7
:200D200070B9012000901C340194B5F80E3405F2FE3203210620F6F749FF1FE006F0D8FC96
:200D40000BA80021182207F0CEFB02A821460C900BA8FEF791FC2C208DF82C000BA801F042
:200D6000B3FE08485038007810B19DF83C0028B105208DF82C000BA8FDF7E0FA11B030BD02
:200D8000080200204206002038B5054695F83000032839D195F83A00032835D105F128047D
:200DA0004A202146F5F7DAFD8A202146F7F718FD6C686178207800EB0120ADF800006946E6
:200DC0005020F5F7CBFDA41C6178207800EB0120ADF8000069464B20F5F7C0FD8B206946F0
:200DE000F7F7FEFCA41CE1202146F5F7B7FD641C6178207800EB0120ADF80000694653207F
:200E0000F5F7ACFD002000E0E82004492A24087028462C7001F058FE38BDC046B104002001
:200E20002DE9F8432020EFF3118780F31188214CA068012107F0FAFB4FF001094FF0000888
:200E400065692168A4F81C906A1A2168A4F81E80461B401A904227D387F3118840462D1847
:200E6000361A4846294607F0DDFBB042F7D92021EFF3118781F31188E18B012903D14046DC
:200E8000294607F0CFFBB0F1FF3F06D0A169801B814238BF081C291801E0A069411907F06E
:200EA000BDFBA4F820902560A4F81C8087F31188BDE8F883780100207FB503461F480D466E
:200EC00001881F480088144614A6984205DB32462146284604F036F81DE0994206DB184646
:200EE00006F0CAFA0028F2D04268F1E715480088002808BF0CA2EBD00095002C48BF47F68A
:200F0000FF74114E0020114901946A46346802901846A047029800907FBDC0467B6D6F64A6
:200F2000756C652325647D007B6D6F64756C652D726F70653A25787D00C046C0720B0000C7
:200F4000CE0B00008E140000FC0B00006D660100F8B50A46034621492148B1F84E708588AE
:200F600091F809C08C6D8646ED18ADB25FB10020A41FA41DE67816B1A688B54208D07F1E83
:200F800000F10100F5D10CF10100C0B2487206E04FF6FF7484421CBF002111701CD1012080
:200FA0001070B1F84C70BEF804604C6D4A7AF01883B267B10020213C2134A67F1EB1B4F8EE
:200FC0001F50AB4208D07F1E00F10100F4D1521CD0B248724FF6FF70F8BDC046BC0F002085
:200FE0008C1C002090B50C46214A0178575CADF11C0D0B2F8DF8007034D0002F35D00C2F92
:2010000004D0112F28D106F0C0FF25E01A2C21D090F89D100190C7688DF80210038A029720
:20102000C28AADF80C30510904D21249827E0978891A00E000218DF80E10877F8DF8107025
:2010400090F91F308DF81130826A0592417F8DF80F1001E0002001908DF801406846FDF711
:201060006DF902E04470FCF753FF07B090BDC0465D000000240600202DE9F04180461E480B
:2010800000680D46416927208847012404FA05F61A4DC5F80064C5F87C470327C5F88077D1
:2010A00017480460C5F88477D5F80404012818BFC5F80444C5F8FC6312480460C5F80080C4
:2010C0001023AB60204607F09CF9D5F88C074008F8D3D5F88C17204611F0404F09D1C5F870
:2010E00084770021C5F8FC16D5F80024164218BF081CBDE8F081C046B0010010044002405E
:2011000000E04842000048422DE9F84F81460020C9F80000684602F053FF1D4EDFF874A08E
:2011200000274FF0FF354FF0190B3C468046E0B206F070FDA8B1837A9BB1017A0127022905
:2011400013D0B16896F892214069C9680BFB021105F084FBDAF80010B0FBF1F0854288BF6F
:20116000051C641C032CE2D300E00025B8F1010F02D0012F05D006E017B10098854200D96F
:20118000009DC9F8005047EA0807F8B2BDE8F88FF8230020442E002070B50646204D307838
:2011A00000BB7178E8782C46012910D0022909D003292FD100204021207104F10A0006F078
:2011C0006DFA27E028B1022006F082FE22E0012806D05220002106F085FB41F2883013E048
:2011E0002021EAE75220002106F07CFB7078032802D13178EA2905D001280BD100202C46CF
:20120000E870EAE72C46074894F85C1084F85D1005F06CF97C35296809B13046884770BD3B
:2012200024170020E09304002DE9F8438146EFF31188202080F311881E4D1A4C184F01269E
:2012400005F11C000660A4F114000660F86A016A14208847D9F81000810C14BF000C0420C6
:201260002060386802682321002090470E480F4F0660386800280CBF311C03210C480768C8
:201280000FB141F00401183C206820F4E02040EA014020602E6088F31188BDE8F883C046B5
:2012A000840100101820094080022443D80B0000DC0B00000000244370B506467468B56894
:2012C000206E06F0E9F829681C488A6B10408863304600F01BFA304601F002FF2968C86ADE
:2012E00020F01000C862296815480A6B104008636868FDF793FF04F17C0007F0C0F804F11B
:20130000980007F0D6F8A07818B904F1CC0007F0CCF8607818B904F1E80007F0C6F804F5D7
:20132000827007F09AF807F0ACF80021217007F09DF904F1680005F0AFFF70BD0DF8FFFF28
:20134000FEFCFFFF38B50C4644220546002100F025FE04F12801284606F084FB04F1320148
:2013600005F10A0006F07EFBE06B6861B4F840002883B4F842006883B4F84400A88394F8D3
:201380004600A87794F84700E87794F9480085F8200094F8490085F82100B4F850006884E9
:2013A000E06C6862A07B85F8280094F8520085F82900606D0B2204F11C01E86205F1300057
:2013C000FFF7CCFA2089A5F840006068E86338BD98B50446217D012905D0152903D0252930
:2013E00018BF352917D1207E000914D219484E30007858B160781B2806D1012005F0BCFF20
:201400004FF4806006F064FE0020607061782046FFF7E8FD98BD207EC20918D2012918BF9E
:20142000152901D100090BD267781B2F06D00A48002F0CBF1A302830405C02E0232000E028
:201440003120207002480078214602F089F998BD08020020240600205D0000002DE9F0479B
:201460001F4EDFF88090002501244FF0020A4FF01108E8B206F0CEFB071C2CD0B87A012858
:2014800029D197F90900113004FA00F0C143316071680843706097F9090004FA00F0C0B208
:2014A00006F0C0F9F868002105F0EEF9812808BF87F80AA081280ED0A9F1020000F29112CF
:2014C00097F90910137808FA01F1DC3019431170002106F0F4FF6D1C032DCAD3BDE8F0877F
:2014E00008100440FA2300207CB515460E46044600E024182046694604F074FE00282DD06D
:2015000014F8021F8E42F4D1491E04F101041FD0491E12D0491E08D0491E18BF622027D179
:2015200002281BD12078287021E0032816D114F8010B28702078687019E007280ED1617852
:201540002078042240EA01202880A11C281D0CE0052803D120780628287001DD67207CBDEF
:20156000281D002103220160611C06F03BFB00207CBD70472DE9F0411E4C024660680028DD
:2015800036D0104606F0E6FE0646084606F076FE074604292CDA50000229015504EB0002CF
:2015A00012BF032900205070134D6868804780466068F1B23A4604F04DFAA9684046884705
:2015C00005F0F2FA58B904F12000044606F058FD01280DD1204606F07AFFBDE8F08104F188
:2015E0002000044606F04CFD10B9204606F06DFFBDE8F081F0190020D0170020F8B5006856
:201600000E4617464FF0FF310446483006F0ABFC4FF0FF35092E08D0217A0120B0400842D3
:2016200011D108433546207210E0227A0721012303FA01F0104202D0491EF9D503E0227AD2
:201640000D4610432072B5F1FF3F15D0A7B1062004F004FF29463846FFF70EFD07460620B3
:2016600004F03AFC47B1217A0120A8404FF0FF3580F0FF000840207204F1480006F017FF9F
:201680002846F8BD70B51E4DAC68064606F07EF94FF47A71001B4843030C05F035FA296931
:2016A000401A48BF404240F6B831F618B14210D306280EDAE9688C420BD8286848B1114A48
:2016C000091B51438A0C02EB1141884288BF011C08E00D49486840080ED208687D2100F03B
:2016E000FF004143C82905D3B1F57A6F88BF4FF47A6103E0C82101E04FF4FA61084670BDE4
:20170000F42D002040420F00AC3F00502DE9F04106467568B46806F0B4FEA96A39B92168FA
:201720008969090903D206F0A1FFBDE8F0810027AF6206F09BFFA17D3846FF2902D0E17D68
:20174000FF2900D118B12846214600F0C9FD2168886B20F0200088632168086B20F48070A5
:20176000086306F08EFE0A4C8046207818B1022004F0B2FB2770404606F078FF686A296A4D
:20178000091A29622B696A6A30469847BDE8F0814D2E0020C8B50F46082F0BDA002F3CD004
:2017A00001787F1E91FAA1F14FEA216100F8011BF6D1C8BD414201F003017F1A4618BBB2FF
:2017C000864203F0030200EB010709D9361A0178761E91FAA1F14FEA216100F8011BF6D164
:2017E00023F003017F1887420AD9391AC91C8E100168761E91FAA1F109BA40F8041BF7D1BD
:20180000BF18874209D93F1A01787F1E91FAA1F14FEA216100F8011BF6D1C8BD2DE9F8434E
:201820001C481F4D07786868804781461A4883680026344680469C4212D013F8020C8742A6
:2018400008D134B163B138464FF40041FEF778FC13E01C4604B91E4653F80C3C002BECD15A
:201860005FB9686880470D49096831F817206FF3DF3221F81720A96888472CB108F1080011
:201880002146324603F0E4FFA968484688472046BDE8F883080200206C1A0020482E002039
:2018A000D01700202DE9F04107461E49BE687C68306809688069C0F3C00008BB06F0E1FD20
:2018C000194D8046287820B1022004F005FB00202870404606F0CAFE3168886B20F020009D
:2018E00088633168086B20F480700863606A216A091A21622369626A38469847BDE8F081BC
:201900004FF4FA70B0FBF1F1012998BF012104F58274204606F0A7FD204606F0A6FDBDE857
:20192000F081C046442E00204D2E0020F8B50546012003F051FF1D4C04F5EE7000F07AF885
:2019400004F5F67000F076F869684A78087800EB0220ADF800008F7804F5EE766FB9532006
:201960006946F4F7FBFF05F128014A20F4F7F6FF05F128018A20F6F733FF06F1200005F175
:201980001C010B2206F02EF9BDF80010384604F0F1FA94F80702800803D36878002106F0D4
:2019A0009DF8002084F80702F8BDC046080200202DE98043074606F064FD804687B3B87A59
:2019C00070B397F9092005F017FD012303FA02F15FFA81F948B1113203FA02F0134B1A6830
:2019E00082431A60C24343F8042C0020F8600246BA723A723A6003467A6007F1100080E873
:201A00000C000B4A02F5C87003781943017092F8920110B1401E82F89201484604F06AF9C0
:201A2000404606F023FEBDE88083C0460C100440F823002070B504461D480078012802D079
:201A40000120F3F73DFE194D281D006880471349064620460B46283105F05AFD20B903F195
:201A60002C01204605F054FD986BA04212D10C4C94F9000010F1020F0AD00B48094B0068E5
:201A800094F90010826B186890476FF00100207002F0C2F9A9683046884770BD080200201B
:201AA000711C0020A81A002078180020D01700203D1D00201D491E482DE9F041352751F8AE
:201AC000048B51F804EB51F804CB51F8046B51F8045B40F8048B51F8044B40F804EB51F8F8
:201AE000043B40F804CB51F8042B40F8046B40F8045B40F8044B40F8043B7F1E40F8042BE8
:201B0000DDD151F8045B51F8044B40F8045B51F8043B40F8044B51F8042B40F8043B40F80A
:201B2000042B09680160BDE8F081C0462489010000C00021F8B507461A48002606701A489F
:201B40001B4C067094F8FC02E0B1D4F840036568C0B1287D352809D168682989FFF71AFED4
:201B600068680088000901D304F0A0FAD4F84013384688470D48007801280AD03046F3F706
:201B80009FFD06E002F0C4F800F0F6FA3846F8F79BFB606810B1007D352801D005F0CEFF3C
:201BA000F8BDC0464E2E0020572E00203D1D00200802002070B51B4C05461022ADF1200DB1
:201BC00004F171016846FEF7C9FE0026049509208DF8146004F10D018DF8160001258DF80A
:201BE00015500A680DF1170002604A684260097A01720D496A4618200DF0F2FA0B4918209A
:201C00008922631D0DF0ECFA7120314606F0F0F9D520214606F0ECF95D20294605F062FE57
:201C200008B070BDCC070000E5A90000E18700002DE9F0431C4E044600271D468946A2EB13
:201C40000408ADF1140DC6F8B071012006F0D9FB3068C00FF9D3306A0090706A0190B06A0D
:201C60000290F06A039044B128462346694611F8012B5B1E00F8012BF9D10320C6F83802B3
:201C80006CB108EB09016D1E491E11F8010F15F8012F904218BF042002D1641EF5D138467C
:201CA00005B0BDE8F083C046504502402DE9F8431C4C1A48A76B06F0C3F91949054608687E
:201CC0000E6800F02000284006F4602615D0A7B107F1180191E800030346E76300201837CA
:201CE000190040EA080041EA090187E8030004F1A8004FF4005106F0E2FB16EA05000AD00F
:201D000094F8911141EA504084F89101002104F1DC0006F0D4FBBDE8F883C04620000E00C1
:201D20000C100440F823002038B518481849007818B90846007828B906E00846007830F09E
:201D40007F0001D006F072FB14490C4660688047104D2146124CEA780C3C23789A4206D178
:201D60000D4A89681278D20802D288470AE08968884705F0F1FA2078FDF7D4F8012804BF46
:201D80002078E87005F0DAFE012038BD04050020572E0020181D0020542E0020D0170020A4
:201DA000A81A00201D4938B5283991F8EC3201EBE30595F8AD42012203F0070302FA03F384
:201DC00083F0FF03234085F8AD3291F8AA3201F52A70032B18D091F8F032012B10D0022BE0
:201DE00008D0B1F8E6128A409102A1EB821101F570710EE0B1F8E6229101A1EB820108E0EF
:201E0000B1F8E6128A4001E091F81D249102A1EB82111C3005F0CEFC38BDC04630020020A2
:201E2000DFF870C098B5FF209CF85F119CF883708CF85C01012914D09CF8F5039CF814146D
:201E4000884223D014480024047005F085FA01F027FC0F480078012818D02046F3F730FCED
:201E600098BD00218CF85F1187B19CF82B148DF803009CF83A748DF800109CF83B148DF826
:201E8000017068468DF8021006F076FA98BDC0463D1D002008020020542E002000B50021AF
:201EA0002022ADF1240D684600F078F81948B0F84010ADF8181090F842108DF80B10B0F8BB
:201EC0004400ADF80E0002218DF8161009208DF80C0001218DF81F1003208DF80D000020D8
:201EE0008DF808008DF81B006A468DF81A0007498DF81D0018200DF073F90549B1F8540088
:201F0000401CA1F8540009B000BDC0462D830100581600202417002098B504462078E0282B
:201F20002CD106F077FB19490F7908610846817801290AD04FB990F85A10012905D190F81C
:201F40005C0001281AD001200CE0114AB2F86E10491CA2F86E1047B97F1CF9B2017100232A
:201F60008370022005F0B4FF08E0002004F08EFA032005F0ADFF052001F01AF80248016881
:201F800009B12046884798BDA81700202417002058160020002213460A46194671B510F0E5
:201FA000030F0BD0002A82BF00F8011BB2F1010210F0030FF6D1002A08BF71BD11F0FF0116
:201FC00041EA0121042A18D341EA0141082A0FD30E46102A08D30C460D46B2F10F0312F055
:201FE0000F0272C0103BFCD812F0080F18BF42C012F0040F18BF40F8041B12F0020F18BF60
:2020000020F8021B12F0010F18BF017071BD704738B51B4D95F8F5030F2829D095F85C1148
:20202000FF2925D095F85E0170B102290CD103F0F1FD144CD5F8541195F8EC23401A21786C
:20204000083101FB120411E003F0E4FDD5F85841B5F8803095F81424241A05EB4205B5F8C6
:202060002401E41A241A01F0EBFA241A002C01D5002038BD4FF6FF70A042C8BFA0B238BD70
:2020800008020020191D0020F8B5194E194D0120002414EA030730704FF0020000EA02002C
:2020A00008BF00280CD14FF0E04004EA0201184008BF002904D11149088C401C088403E02E
:2020C00095F90000401E287005F04AFB05F036FD0948047095F9000028B195F90000002838
:2020E00004DC06F0A3F92046F3F7EAFA3470F8BD3D1D00207A1C0020731C00208C1B00203B
:2021000070B517481749007818B90846007828B906E00846007830F07F0001D006F086F95A
:20212000114C60688047124E104DF1782A78914207D1104AA1681278D20803D288470120B4
:2021400070BDA168884705F007F92878FCF7EAFE012804BF2878F07005F0F0FC70BDC0460A
:2021600004050020572E0020D01700209C1A0020181D0020542E00209EB51B49A1F124044C
:20218000606880472146144CE288A388934220D0124B1F78EFB9124B89681F7837F07F0761
:2021A00018D1A28088471027A088ADF8007001A9ADF8040009880DF1020319800949BDF84A
:2021C00004000A4A08801068426AE068694690479EBD896888479EBD9C1A0020552E00203E
:2021E000572E00201A160020F41700207818002038B51C4C002084F8610194F8F55394F85C
:202200003802401CC0B2042884F8380224D0202003F0E2FA94F837240F2A0AD094F86201E8
:2022200094F8F513814204DD154684F8F50304F0A5F904EB4501B1F8245194F8F53394F872
:2022400038124FF4707204F502709A40491C01FB152104F071FE38BD03F0A6FEFDF71EFF33
:2022600038BDC046080200202DE9F84380461A485638077817B9174D287810B90120BDE850
:20228000F883164E243E70688047814668880124B8F1000F0ED1214603464FF6FF72B9408C
:2022A0004A40104068807BB170B9002004F0B4FD044609E018B9204604F0AEFD68882146E2
:2022C000B940084380B26880B168484688472046BDE8F8831C1D00205E020020F4170020A0
:2022E00038B50C4621680546886B20F020008863286E217D012202F02BFB286E217D0122F7
:2023000003F0A8FB286E217D002204F04FFA286EA17D002204F04AFAA878012806D005F171
:20232000CC004FF0FF3105F01EFE03E0216888690009FCD2286E217D102204F037FAA17D74
:202340000020FF2902D0E27DFF2A00D118B1286E112204F02BFA38BD2DE9F84F8346894675
:2023600017467120114604F0BBFB81206946F8F793FC4FF0F308002507E0B8F1000F23D0AF
:2023800038686D1CEDB22C3038609DF80000A8421ADD3868066890F804A0002402E0641C4B
:2023A0000A36E4B2A245E8DD737A002B0CBF052009208145F3D14A463046594604F0ECFF5C
:2023C0000128ECD14FF000084046BDE8F88F70472DE9F8431A4C05460E46201D016816480D
:2023E000007820B9002028603080BDE8F8838847DFF84880D8F804725FFA80F908F5DC7045
:2024000005F0B6FED8F880214FF47A73410001EBC001B1FBF3F129605018B8F87811286042
:202420008742318003D8C01B2860491C3180A16848468847BDE8F88354110020BC0F0020D8
:20244000D017002038B5054601201A4C68712879B0B90DF096FA2178002904BF6FF0070457
:20246000051C15D0491EC9B2217039B90DF0B3FA606804F013F90020687118E0054613E050
:202480000DF07FFA05462078FF2805D16FF0060428460DF0A0FA0BE0401CC0B20128207006
:2024A00002D1606804F011F928460DF094FA0024204638BDA81C0020154998B50F7817BB23
:2024C00019490A784968930000FB0314114B9700B3FBF7F1814214D30F480068C06B8047DE
:2024E000211AA1F54871090806D30C4A011B891A090828BF00F5487409482146F9F7A6FF5D
:2025000098BD05F093FF07490120087098BDC0463E1D0020FFF6C2FF7818002000093D0074
:2025200091B00000562E0020B01B00207CB542F2050001A902F04AF842F20100694602F0AD
:2025400045F89DF8040030B3134C0098D4F8806108B39DF80410B14209D8B04201D805F026
:202560008AFF00980021012584F8941104E001259DF8040084F89451801B642104F5DC7663
:202580004143C4F8BC11304604F082FA304601F08FFE84F898517CBDBC0F002030B504469C
:2025A0000D4642F20900ADF12C0D09A902F00EF89DF8240008B342F20B000DF10E0102F058
:2025C00005F800230094BDF80E00029300040190684602F0FBFC044604A942F2030001F0A4
:2025E000F5FF04F0A9FB024604A9B4FBF5F06843241AE0B201F09CFF06E042F20D0003A9EC
:2026000001F0E4FF9DF80C000BB030BDF8B5054605F037FF184C0126074605F19C00267179
:2026200005F025FFB4F94800B4F94A1088420ED1A07802280BD094F8440140B1384606F089
:2026400015F80720FEF7EEF805F01BFF0746B4F94800B4F94A10884218BF85F8C26006D1FC
:2026600005F1780005F003FF082003F043FB384605F0FCFFF8BDC046F8230020F0B5054648
:20268000194C2878ADF11C0DE9281CD028BB002694F85A0084F85E6002281ED104AF6946CD
:2026A000384602F02DFC5220314605F01BF92046406920B1026812B138466946904704205A
:2026C00000F076FC09E094F85E00401C84F85E00C0B2032801D102F0F9FD9434216809B12D
:2026E0002846884707B0F0BD24170020144998B50F780FBB1349144B0A789200B3FBF2F381
:20270000834217D34968114F00FB02143868C06B8047211AA1F54871090806D30C4A011B70
:20272000891A090828BF00F548740B482146F9F78DFE98BD05F07AFE06490120087098BD19
:202740003E1D0020B01B0020FFF6C2FF7818002000093D00562E0020B1E900002DE9F041E2
:2027600007461748174C0C3806786068804780461549A268087886281CD1104D05F11E023D
:202780001088401C10808720087005F08FFDA16840468847082004F0ABFBA879B04207D10A
:2027A00027B90020FFF7C6F9BDE8F0811B20F9E7E920F7E740469047BDE8F0818C1B002012
:2027C000982D0020D0170020572E00202DE9FC4716460C46054604F05FFC164F81467868BB
:2027E0008047804603F0ACFB8246B2002146484605F092FD504604F06DFF02E02D1D241D5C
:20280000ADB23046411ECEB278B128466946042203F07CFD68462146042204F0B1FB002829
:20282000ECD00549012048700870B96840468847BDE8FC87D0170020A01C00202DE9F8436B
:202840000024002B16460F468046254606D5002FC3F1000302D57F42761E2D2599463846AB
:20286000494602F0B3FD0CA0405CB7FBF9F7002F04F1010408F8010DF1D1A64205DD302129
:20288000301B401E08F8011DFBD10DB108F8015D4046BDE8F883C046303132333435363741
:2028A00038396162636465660000FEE7C8B50146184AC87AC8B9B2F84E70906D4FB3801F7E
:2028C000801DC67826B1B1F81F2083889A4202D07F1EF5D1C8BD8A7FC270CA880280B1F805
:2028E0001F208280097B8170C8BDB2F84C70506D7FB121382130867F4EB1B1F81F20B0F80C
:202900001F309A4203D1212205F06CF9C8BD7F1EF0D1C8BDBC0F002098B5164C94F8E100AC
:20292000002710B91448007860B105F0AAFD94F8E310002906BF012184F8E310012705F00B
:2029400095FE0FB1002098BD022003F087FD0E20FCF74AFF094A106848B909494020C86006
:2029600008600127D761002084F8E20098BD012098BDC04658130020010B000004800C40D9
:202980002C500C40F8B50E46044605F07AFD0546F0B205F03FF98026071C20D0B87AF0B112
:2029A0001248801C0078022806D03846FFF700F800F0B6FD832612E097F909100A4E4FF4BB
:2029C000A060002200EB012000F47F4046EA0001204603F0B9FB06463846FEF7E9FF2846C3
:2029E00005F044FE3046F8BD01000804F8230020001F06B480B280B5082802AFADF1080D59
:202A000026DBB0F5805F23DA00F18851091F0B686A46136049685160BDF80010CA0B10D3CD
:202A20003A7801F0FF018A420BD17988BDF80220914206D1B988BDF80420914208BF0120F4
:202A400007D0BDF80610401A083880B20828D8DA002002B0BDE8804002B070471FB501466B
:202A600004208DF8000048788DF80100B1F89A000DF10203ADF80C009031184604F00AFF54
:202A800004F0E2F8C0B14FF6FF7453200DF10E01ADF80E40F3F762FF0A4890F8F513A0F807
:202AA00008440F2908D00F2180F8F51304F0EAF903F07AFA05F072F86846FBF73FFC009002
:202AC0001FBDC04608020020194AF8B5044692F8560002EB8000D0F8AC30207800F07F0098
:202AE00041005D182070C918497802EB8106D6F8AC7027B182F85610207803EB400529786C
:202B00000B1102EB8302D2F8647137B90C280EDA20461821FEF766FAF8BD01F00F0157F883
:202B200021700FB905F082FC20463C46A047F8BD080200202DE9F843DFF85C90044609EBC9
:202B4000440000F15805B0F85800884604F006FA074612480678B7B12A883846002105F04E
:202B6000C2FC00253C70494664187D70627D381D414605F037F83046394600F0F1FD40B923
:202B80002846BDE8F8838DF8004068461A21FEF729FA1A20BDE8F8833C0000000802002021
:202BA0002DE9F843174C04F1780007688046632037B300261D25397D35291CD140463946E4
:202BC000324602F045FE787E30F07F0005D194F88300401E84F8830004E094F88200401E21
:202BE00084F882007D7057F80C9C3846FEF7F0FB4F46002002E03E4657F80C7C002FDAD1C9
:202C0000BDE8F8830802002098B5184B04461B1D18680004070C25D003F076FF124991F95F
:202C20000720824205DD10F1800FB8BF6FF07F00C871BC422CBF01273F1B8C88BC4210D844
:202C40000A68D3F8D40F801A801C1F2888BF1F203F1B4008C7404FF6FF70E719B84238BF03
:202C6000071C8F8098BDC0463C2E002030100940164880B507683FB315498B6803EA53002F
:202C8000C00E21D2134A106880081DD2486880081AD21068096810F0050F4FEA114101F08A
:202CA000F00101F5E0710AD1B9420DD2190F38BF40F00100D90E38BF40F0040003E0B942E7
:202CC00002D920F00500106080BDC04628500940AC3F0050000009402DE9F04180461748A0
:202CE000243007680E46ADF1300DBFB13869A8B1B8F1000F12D08EB106208DF828000125A6
:202D0000ADF82A500022ADF82C2002AC00943C690AAB93E803001A23A04708B100200AE080
:202D200002A940460C22FDF719FE05A930460E22FDF714FE28460CB0BDE8F0816C140020EF
:202D4000F8B5844640F6FF741CF8013B002210E0481B401E10F8015B7F1E01F8015BF9D110
:202D600003E01CF8010B01F8010B521C5B08082AEADA5808F5D21CF8010B1CF8015B05F0D8
:202D80000F07FF1CC5F30315122F45EA001508D11CF8016B300A24BF1CF8010B60F3DF16CF
:202DA000BF19AC42D4D1F8BD10B5042003F0D2FC022821D003281FD001281AD01148006840
:202DC000C0F38150032805D002280CBF41F28832322201E04FF47A720B490C4C09684C348C
:202DE0002046B2FBF1F105F03EFB204605F03DFB10BD02F097FC10BD02F094FC022003F067
:202E00006BF810BDB43F0050442E00206013002098B504460F46E920694601F0D9FE9DF819
:202E20000000134938B90846072200F1080105230A70082205E00846052300F108010B7038
:202E400018224272881C0222002F02704FF00007CF7003D0027842F0100202700C71054AC7
:202E6000C2F88C10A2F880300321FEF793FC98BDCC1A0020701500202DE9F041174E706886
:202E80008047144D144C2F78B1682A78012A0BD04FF0010885F8008088472078012804D099
:202EA0004046F2F70DFC00E08847F8F7C9FD804670688047B168B8F1000F08BF2F708847CB
:202EC0002078012802D00020F2F7FAFB4046BDE8F081C046721C00203D1D0020D017002090
:202EE00010B5044600212822ADF1280D6846FFF755F8134911226846FDF730FD05208DF88C
:202F000012008DF8114000218DF8151001208DF816100B228DF81700FF208DF81800092084
:202F20008DF8130003208DF814000DF11900FFF735F8044918206A460CF052F90AB010BD00
:202F4000E307000061F10000154880B50078022822D0052805D001281FD9C11E01291ED8ED
:202F60001BE004F0A3FD48B10F490E4A097812688900B2FBF1F1401A48BF00200B494F786A
:202F800047B191F8F5130F2904D018B91C20FEF7D1FD80BD052000E00220F1F763FF80BDE1
:202FA0008D1B0020C0150020B01B002008020020B0B5184C054694F85A00A8420FD084F800
:202FC0005B00052D84F85A5002D1002003F076FA606920B1C16811B194F85A008847042D7D
:202FE00018BF032D10D1276905F014FB0749C01BB0FBF1F10648B0F87A208A4204D21FB19B
:20300000A0F87A1000202061B0BDC046A0860100581600202417002038B5012003F09AFBD4
:20302000012820D0114DD5F82401C4681048342101220023A047002808BF002014D028689E
:2030400003F09EFD04F0A2FC0B4A0A4D93681168D060C01AA1EB910105FB00F3180C884227
:2030600028BF011C1160012038BDC0468000001000A00C4040420F00F42D002001461748CB
:2030800080B500688A0CC0F38367C0F38F2022D241F3072100290BD54A420021400805D1DA
:2030A0007F0806BF0127381C4FF6FF70521EF5D1002910DD4FF6FF72400040F0010082425D
:2030C00007D2780040F001070F2F92BF01200F27101C491EF0D140EA074080BD50130050CC
:2030E000F8B50646B26811687568886B20F4FA6088631168086B20F40070086305F0C1F991
:203100000F4C0746207820B1022002F0E5FE00202070384605F0AAFA05F0B3F9A96B11B961
:2031200005F0A4FAF8BD0021A96305F09FFA686B296BEB68091A29636A6B30469847F8BD44
:203140004C2E0020012898B525D1012003F002FB012820D004F032FC124C012104F1D800D0
:20316000017005F067F8800917D20D4800683222B2FBF0F707B90F46083C04F1300005F000
:2031800076F904F13000394605F06DF904F1300005F06BF901E002F06BFE002098BDC0468C
:2031A000442E00206013002010B50446012002F013FB208900280CBFEB20002012496070C8
:2031C00091F80702C20824BF20F0040081F80702820809D2400813D32B202070EB236370CB
:2031E0002046FFF771FC0BE091F8070200F0FD0081F80702217C6078C1F3001104F06EFC82
:20320000204602F0EBFE10BD0802002030B5174C054605F12801ADF1140D04F2FE3003F0EE
:20322000CDFB08B3EF2309208DF801306B688DF800005A781978181D01EB0221ADF8021064
:203240002A890178082A8DF8041014BF94F83A04C07805F11C018DF805000DF1070005F00B
:20326000F1F86846FBF76AF805B030BD0802002010B504460320ADF1180D04F128018DF8FF
:20328000020000208DF8030001A805F0DEF86068007804F11C018DF80C000DF10D0005F02D
:2032A000D1F804F1280003F0CFFC58B14FF6FF7453206946ADF80040F3F750FB04492046BA
:2032C0000A3108800DF10200FBF738F806B010BD0606002038B5124C4FF470000025E060F7
:2032E0001148A56000686560C06B80470D49C0F1FF3008600D49C868657008B90C48C8601B
:203300000C480570012001F001FF30B90F2003F035F9E068FFF7D0F838BD05F087F838BD35
:20332000B01B002008300440781800206C1A0020693D0100562E002070B5164604460D1C91
:2033400008BF052426D034F07F0001D004F00CF9002C18BF032407D155F80C0C18B915F8D5
:20336000020CFF2804D00524284604F00EFE11E0012E094805F8024C03D0294602F0CAFEF5
:2033800002E0294604F018F820464FF40041FCF7D7FE0024204670BD741A002030B5044692
:2033A000606800252062ADF1140DA5657820A4F84C0094F82C0025650F2807D004F12C01E3
:2033C00020460122F6F700FE08B116E0284694F83C10FF2901D1A16D21B104F13C01204612
:2033E000FBF7B0FB48B92B4601208DF80C30032101AA00902046F0F7D7FC05B030BD704704
:203400002DE9FC41144C154F06468846700809D320684568002101220B461FFA88F000903C
:203420003846A847B00809D3206845680021022201231FFA88F000903846A847F00809D38B
:2034400020681FFA88F600210C220223446800963846A047BDE8FC81A401001000A00C406F
:2034600010B505F00EF81549891C0978022918D005F0FCF804F082FC0D4A002304F0E2FB4F
:203480000C4C4FF090531B1820684FF07A044FEA000244EB010400215B1844EB0204241CC2
:2034A00003E005490C6805F0E1F8204610BDC04600093D00182E002004300440F823002001
:2034C0000246F8B5084611464C68203821D0401E1CD0401E18BF6FF001001ED18D6804F09E
:2034E000D0FF0E4E07463068016928688847B0F1FF3FF8D100256564206C401EA064E56426
:203500003846A56305F0B2F82846F8BD0021084601E00121002084F82D10F8BDD001001082
:2035200038B5164CA078022823D0012824D0042822D004F0A6FF05466846FDF7E5FD80B133
:20354000009949B904F1840004F091FF04F1A800042104F0B4FF08E004F1840004F0D0FB4A
:2035600003E004F1840004F082FF284605F07EF838BD192004F089FF38BDC046F8230020C1
:2035800038B504460D46E920694601F021FB13483D300078812801DB84280FDB04F10D007F
:2035A000690880B224BF04F1260080B2122CCCBF05210221401880B2C0000DE0600169081D
:2035C00000F5967080B224BF00F21E2080B2122CCCBF28210C21401880B238BD060600208F
:2035E000F8B51649144C621C0C311378114A09681778002F0CBF0969496903EB83035B18B9
:203600001D79002101E0491CC9B28D42D8BF4FF6FF700DDD1E680A4602EB4202921992F9F1
:203620000060B042EFD1B2F80100E080B2F80100F8BDC046710600209C1A002068180020FA
:2036400070B5134D114968780C880830444312480068104EC06B80477168401A31788900E1
:20366000B0FBF1F10D4802783C209040B1FBF0F242436878891A00F10803B1FBF3F25A4302
:20368000891A401A0019083070BDC046941B0020181D0020B01B0020781800201C060020A8
:2036A00070B5154D286808B104F0F4FD134C60688047103D296A0A6800261671096829626C
:2036C000A1688847094A0A49107810B90846007858B1167008460670FCF72AF80548007828
:2036E000012802D03046F1F7EBFF70BD532E0020552E00203D1D0020982D0020D0170020B0
:2037000038B5164C04F52A7005461C30FEF792F903F0C2FA042003F0EBFB94F8AA020328A1
:2037200002D194F8A902A0B105F14501E120F3F715F905F14601E720F3F710F994F83B04F7
:2037400094F8EF12884204D005F14701E820F3F705F92846FAF7F2FD38BDC046080200209D
:2037600070B502460D4632F07F0004D110460022FFF7E2FD70BD04F0A5FD104908398C7865
:20378000A5F10C06FF2802D0C96A09184C78FF2C02D103F0E9FE0DE0104604F019F8014609
:2037A0002A46FF20B072204602F014FB20B1284604F0EBFB012070BD002070BD741A00208F
:2037C00038B5044642F208000DF1020100F0FEFE9DF8020040B19DF8020002281ED12046EB
:2037E00002F072F8054606E042F20C00694600F0EDFE9DF8005094F8200068B9284600F062
:2038000047FE0020A4F87C5094F8223020702BB1102004F065FC38BD0120207038BD7047BA
:2038200000B5ADF1240DADF80000ADF80210116801A8016051684160002002460D49069077
:20384000887D8DF80C200D318DF80D000B680DF10E0003604B684360097A017218208DF8F7
:203860001C2005498DF81D206A460BF0B9FCC0B209B000BDCC0700007D5900001348144A52
:2038800014490078801E0A2807D8DFE800F019140F06140F06140F0607C0FEE710688008AD
:2038A000FCD250688008FCD2F6F73AB908688008FCD3F6F735B908688008FCD2F6F730B90E
:2038C00010688008FCD3F6F72BB9C0463C14002034600C4038600C403EB5401E4FF000047A
:2038E0000AD0401E04D0401E1CD1F6F719F919E0FFF712F8044615E0684604F061FD0194A5
:203900000B4D8DF800400849029401226B4605F1780000F0D5FF054A2C21234605F19C0006
:2039200001F0B4FD20463EBD7D380100594B00005813002038B54FF0FF3004F04BF8134CAE
:203940000F490546083CE06981420ED10D4904F14C00002204F09BFD0220A07002F096F89E
:2039600018B9FDF77BFDFBF72BFE0748284205D004F1A8004FF0005104F0A1FD38BDC046A7
:2039800039360000BDA50000020000400024002010B50446012001F01FFF1248FEF74AF800
:2039A000208900280CBFEB2000200F49607091F80702C20824BF00F0FB0081F807028008E4
:2039C0000BD391F8070200F0FD0081F80702217C6078C1F3001104F081F8204602F0FEFA11
:2039E00010BDC046E4030020080200202DE9F0410446A76E1E461546884607B1B84704F1E4
:203A0000600003C805400E4008BF002D1AD041462046802201F0A4FE04F1700181E86000B9
:203A200050B100F1180106C900F11803B243A94383E80600A16E41600020A06604F1400043
:203A400004F035FDBDE8F081154909681F280ADC1F2819D00D380FD00A380FD0001F0FD0BB
:203A6000C01E0FD01AE0253810D0001F10D0401E10D0801E10D011E0086870474868704718
:203A800088687047C8687047086970474869704788697047C8697047086A70470020704778
:203AA000F0010020F8B50646B08815460F46FDF703FA0446002D02D4281B0A2806DB3368E5
:203AC000291B38460BA201F03DFA2418B08978B1002D06D4B06804F0D3F9291B401D884267
:203AE00006DCB368291B384603A201F02BFA24182046F8BD257000C0282725732729000069
:203B000070B5124C6068F8B1124D68688047064694F883200E4861680078904206DCA968E4
:203B200030468847F120F6F7CFFB70BD04F1780003F042FC002394F88300A9686360401C4B
:203B400084F883003046884770BDC046080200208C1C0020D0170020F8B5134C60680D46CE
:203B60008047124A8446A168B2F84C70506DB7B1002421382130867F6EB1B0F81F20954214
:203B800009D1002282774FF6FF72A0F81F20604688472046F8BD7F1E04F10104EAD160461B
:203BA00088474FF6FF70F8BDD0170020BC0F0020F8B50746C81D01F00705C610002F4FF0BB
:203BC000010000FA05F0A0F1010C14BF0029002019D00020BEB17F1E33460246941B17F8A7
:203BE000011FB4F1FF3F08D10DB10CEA010104E001F1FF04401C2140C0B20029F8D15B1EC0
:203C000002F10102EAD1F8BD70B5EFF7F7FE124D68688047064603F08FFB104C94F92A0468
:203C200004F0FCF802F09EFE04F0EEF803F07AFF03F06CFFA9683046884794F82B0400F069
:203C400027FC04F211415220F2F788FE04F028FB08B9FFF73FFB70BDD017002008020020B2
:203C600038B50C4620B141680122A240114201D1022038BD914341600E480025031900EB53
:203C80008401C1F8985003F144010978FF291ABF806850F8211044F020410548F9F786FF8B
:203CA00020464FF0FF3103F0A5FC284638BDC046007FC767441200201248134908B54FF459
:203CC0002C72FCF74BFE4FF00451002081F89003012081F87903022081F87503032081F885
:203CE0007703042081F8AE03052081F8AB03062081F88103072081F84D030448C1F8C003D5
:203D000008BDC0461C04002174860100CD0500212DE990410F4C6068804780460E48007844
:203D200098B90E490F78012037F07F0707D10C490F7827B90B490F7837F07F0703D080F027
:203D40000100C0B208B103F007FBA16840468847BDE89081D0170020542E0020532E0020E4
:203D6000552E0020572E002070B5124C6068804711490025064648784D70A168820807D235
:203D8000C00814D3304688472846F1F799FC70BD3046884709480078012802D00120F1F705
:203DA0008FFC606880470646FAF768FCA1683046884770BDD0170020B01B00203D1D002061
:203DC0002DE9F041054600202860114800780E46012802D00120F1F773FC0E4C6068804728
:203DE0003768804630463FB16A687968914203DC38463F68002FF8D1056030682F60854223
:203E000001D100F009F8A16840468847BDE8F0813D1D0020D0170020B0B5144C0025284692
:203E2000A26A216BA56390420CD05268914209DD01F0F0FE0146A06A42689142C8BF4160EC
:203E4000A063216BE76A37B118B142687B689A4201DD3846A06328B14068814202DD01F0F5
:203E600095FAB0BD03F056F8A563B0BD0802002038B5046845682068002808BF4FF0FF307B
:203E80001FD004F0FEFA2168002954BF491E0021216004F0EBFB206890B904F12C0004F0B9
:203EA000EEFA04F1480004F000FB04F1640004F0FCFA6868FBF7B2F904F1180003F0ECF959
:203EC000002038BD38B5134C054694F8201094F8230081421DDD94F82110A94219DD636AA3
:203EE0003BB1294604F5BA72984794F8230094F8211084F8220001FB0051E06901EB810155
:203F00000918087884F82300D1F8011004F5BA70884738BDBC0F0020C8B506461248801EF4
:203F2000876BFFB1816B91F82F1049091AD3476BC7B1416B91F82F10490913D2416B826B7E
:203F4000C968D26891420DD1371C06D07F1E09D1816B016400278763C8BDA8304FF4004162
:203F600004F0ADFAC8BDC046FA230020B0B5134C6068628808B325880021AA42C8BF01214A
:203F80000B46AA42C6BFA91A01F58061A91A8FB297B1012B04D0121902F108013A4609E0E9
:203FA0001119C2F58062083104F0CAF9606804F108012A4604F0C4F96580B0BDB40B002036
:203FC0001249B0B5054601F134000768C7B1BA68107B012400F00F00022818BF002011D1F5
:203FE0009068FA6891F89231D268192101FB032102F034FC064909682860B0FBF1F001E0B0
:204000000020044628602046B0BDC046F8230020442E0020134910B5044691F80702ADF16D
:20402000180D40F0020081F80702012003F0A4F9607890B9211D02A803F02CFC03F042FDA0
:2040400001460120009004F110030193E38902AA0520F3F7BBFD607010B1002103F03EFD0D
:2040600006B010BD080200201048F8B5066810480068104CC06B80476168401A21788900CD
:20408000B0FBF1F0B0420ED20B4D243D686880470746A6603046FEF729FBFAF7EFFAA968A5
:2040A00038468847F8BD04F0C1F9F8BD3802002078180020B01B0020F417002010B5134C57
:2040C00094F8610194F8381240B9606860B9012084F86101202003F0F3FF05E0481CC0B263
:2040E000042884F838020BD094F8F5234FF4707104F50670914001F2636103F05BFB10BD2E
:20410000202001F069FBFBF7C9FF10BD0802002010B5134C012094F8F51384F861010F296A
:2041200018D06070202003F0CBFF0C4894F8F51394F83832C4F8200204EB4101B1F82421EF
:2041400004F50670591C5143490001F2A32102F0F3FE10BD01F028FF10BDC046F121010039
:2041600008020020C8B5071C23D079684878C61121D03A89F96400204B78C3F3C3030F2B60
:2041800008D00B78C018C918801C891C80B28242F2DC01E0801C80B2824208DB79683E8908
:2041A00009187960311A3981A7F85000C8BD0020FAE704F03BF9C8BD10B5044600211C2270
:2041C000ADF1200D6846FDF7E9FE60788DF80000A0788DF80100E0788DF8020020791122E5
:2041E000611D8DF8030001A8FCF7B8FBA07D8DF8150008B1A0690690034800688169684610
:20420000884708B010BDC046641C0020F8B504460D4608461122002104F065F994F800C01A
:20422000BCF1000F1AD0641C00214FF0010EE078A37843EA0023207809E0C610AF5D00F0D3
:204240000702401C0EFA02F2C0B23A43AA558342F3DA491C241DC9B28C45E8DCF8BD80B5DD
:2042600002465378107840EA0320C7130F7007BFC0F3062300F0FF00C0F3C323C0F30A0016
:204280004B70802848800DDA02280BDB012B0CD0022B0AD0042B08D0052B06D0062B04D0DB
:2042A000072B02D00022104600E0921C4A6080BD2DE9B841114C0546201D00688047804624
:2042C00002F04AFF6F7E0146002F08BF686806D068682A69AF68401A8018C019686029613C
:2042E000E96805F1140201F08FFD012768686F76A168A86040468847BDE8B881D0170020BC
:20430000114810B50078E8B1104C233C94F82A1264204843C4F8A00104F5CE70FFF7C8FF8B
:20432000B4F8760194F82A22D4F87C11401C80B28918A4F8760100B900210020C4F87C11A4
:20434000FFF7C0FD10BDC04619060020DF0F002038B504460F491048143009880068A14283
:2043600013DD0E4D6868804703466946722002F0B7FB0099E00000EB041009180091A968F2
:20438000184688470098001D38BD641AA1B200EBC10038BD901C0020BC0F0020D017002016
:2043A000F0B5124D00260C460746ADF1140DC5F8B061012004F025F82868C00FF9D3286AB8
:2043C0000090686A0190A86A0290E86A03903FB13846694611F8012B401E04F8012BF9D1BF
:2043E000032005B0C5F838023046F0BD5045024010B5114CA2685168496839B110B102F0C1
:20440000BFF9A268506840688047A2685168886808B9C86870B103F01FFD5168886810B175
:204420008047A0684168C86800B180470348503802F07EFB10BDC046F823002051000706B2
:2044400010B50446012001F0C7F92078212804BFEB2060700D4991F80702C20824BF20F057
:20446000040081F80702800805D22B2020702046FEF72AFB10BD91F8070200F0FD0081F837
:2044800007026078002103F029FB10BD08020020F8B5104C0646201D0568802E01DD03F08E
:2044A000C5FFA8470C4D0D49094A2F780E701FB91778A1682FB907E01778A16837F07F079E
:2044C00002D088470120F8BD8847FDF719FEF8BD572E0020D0170020040500209C1A00202B
:2044E00070B540680C46054600F5827003F0BFFF0D486A7F0168287F8018AA69C01D80B2B2
:2045000044430A4805F582766043B0FBF2F008186330B0FBF1F1491C304603F0A4FF304679
:2045200003F0A3FF70BDC046442E002040420F002DE9F84300249146884606462546274652
:2045400013E018F8011B082281F0010000F001002418E4B2601EB04206D06D1C521E4FEA65
:204560006101EDB2F0D100E00127A94502DC1FB903F081FF002FE4D02846BDE8F883FEE704
:204580000146104810B500784FF4C854812803DB8428B8BF4FF41644052909D001F038FD6C
:2045A0000949C07B0988022814BF04F57A740C4404F57A644FF47A6004F5FA64B4FBF0F0CF
:2045C00010BDC04643060020B2110020F8B50E4602F0BBFF05464FF6FF70A84208BF6820D7
:2045E00013D00C4C606880470849094A0746680000EBC5004018017889184278304603F053
:20460000F1FAA168384688470020F8BDD8040000B8110020D0170020042838B51CD1104C56
:2046200004F18400054603F0EBFCA8B1284603F018FF0A4909684843B0F5967F0CD22846B6
:2046400003F015FF052001F009FF2046012141700421A83003F033FF002038BD442E002033
:20466000F8230020084608B500F0005100F00400084314D0012002F06DF8012809D00849C5
:204680000A48096832228430B2FBF1F103F038FB08BD044803F0AAFD034803F029FD08BDC6
:2046A000442E002039360000082E0020F8230020104898B501210170022111400E4A4FF025
:2046C000E0471F4008BF002903D092F90010491E1170044692F9000028B192F900000028AD
:2046E00004DC03F0A3FE0020F0F7EAFF0020207098BDC0463D1D00207A1C002070B50120D5
:204700000E4E0F4D30702878022814D10024022114EA030001EA020108BF002901D103F0A7
:2047200085FE084991F90000401E08702C7003F029FA347070BD03F079FE70BD3D1D0020B1
:204740003E1D00207A1C002038B5EB2003F0AFF80E48002404700B480078862802D12046F6
:2047600000F018F8084D68688047094910390A6A13681C7112680A62A968884703F060F825
:2047800038BDC046572E0020D0170020552E0020982D002038B50F49104C888B401C8883CF
:2047A0006068804705460C480178862903D0A1682846884738BD8721017003F077FDA1680C
:2047C00028468847082002F093FBE920FDF7B2F938BDC0468C1B0020572E0020D0170020DE
:2047E000F8B506460F4D104F7388002417E0A20002EBC402921951689068D26852B9AF4208
:204800000BD00A7855F822200346491C08461946904701E0FCF7A2F87388641CA4B2A34256
:20482000E5DCF8BDEC940100F89401003EB5054615F8060C03281DD12B6818690090586919
:204840000190986902906C6859689A681868DB68A0472968086015F8080C01F0A7FE0446F9
:20486000012002F07BFB011C04D0422008702046FEF776FF3EBDFEE72DE9F04117468846C2
:20488000064603F0FDFA0D4C0546002128222046FDF784FB31462A462046FCF75FF84046DD
:2048A0003A46611900F0C0F8204603F00DF802A003F00AF8BDE8F0810D0A00C0B02D002077
:2048C000F0B515460E4604461F1CADF1240D08BF002308D0684600212422082303F096FEA7
:2048E000B8686B460690204631462A4603F08AFE0348044F0168204609B03960F0BDC04617
:20490000E80B0000442E002000B500211A22ADF11C0D6846FDF742FB02200B4A8DF814004A
:20492000B2F84410ADF80C10B2F840108DF818000020ADF8161005498DF8190018206A4662
:204940000AF04EFC07B000BD241700203783010038B50D460E49144664390A68AA4205D3C5
:2049600001EB8501D1F89810884201D0022038BD03F087FD074B103B1A68AC400121A94015
:204980008A4314431C6003F071FE002038BDC046A8120020E02002401049D0B50F68ADF1EB
:2049A000180DCFB17E69BEB1B0B106218DF810100226ADF812600024ADF814404388ADF803
:2049C000003042680192816802917C6904AE96E803000C226B46A04706B0D0BD9014002009
:2049E00070B50E4614460546082300212422ADF1280D684603F00AFE002006900590ADF89B
:204A00001000084800684FF47A716B46B1FBF0F080B2314604FB00F2284603F0F3FD28460A
:204A20000AB070BDE80B0000FEB50746052400266B4697FBF2F05043381AC5B20A2DACBF2A
:204A400037203020401997FBF2F51870AFB22FB1641E03F1010306F10106EAD1761C13F844
:204A60000109761E01F8010BF9D100200870FEBD70B5104D95F8F503B5F81A440F280FD04E
:204A8000D5F8586101F0C6F80019864208D895F8F5134FF4707088402418A41B04F57074C8
:204AA00005F5EE752846FCF7C5FF2146284602F081FE70BD0802002010B504460E480078FA
:204AC00001F0A6FA4268016804FB02124FF47A71B2FBF1F3094AD3854368006804FB0300A0
:204AE000B0FBF1F39BB201FB130040037D21B0FBF1F0108610BDC0464306002070150020E7
:204B00001FB5144600900A79487940EA02208A7942EA0022C87940EA022001900A78487896
